:020000040800F2
:1000000000800120D5A400081BA500081DA500083C
:100010001FA5000821A5000823A500080000000076
:1000200000000000000000000000000025A50008FE
:1000300027A500080000000029A5000801180008F5
:100040002FA5000831A5000833A5000835A5000834
:1000500037A5000839A500083BA500083DA5000804
:100060003FA5000841A5000843A5000845A50008D4
:1000700047A5000849A500084BA5000865AA000887
:100080004FA5000851A5000853A5000855A5000874
:1000900057A5000859A500085BA500085DA5000844
:1000A0005FA5000861A5000863A5000865A5000814
:1000B0007584000869A500086BA500086DA50008F7
:1000C0006FA5000871A5000873A5000875A50008B4
:1000D00077A5000879A50008E58200087DA500083D
:1000E0007FA5000881A5000883A5000885A5000854
:1000F00087A5000889A500088BA500088DA5000824
:100100008FA5000891A5000893A5000895A50008F3
:1001100097A5000899A500089BA500089DA50008C3
:100120009FA50008A1A50008A3A50008A5A5000893
:10013000A7A50008A9A50008ABA50008ADA5000863
:10014000AFA50008B1A50008B3A50008B5A5000833
:10015000B7A50008B9A50008BBA50008B946000866
:10016000BFA50008C1A50008C3A50008C5A50008D3
:10017000C7A50008C9A50008CBA50008CDA50008A3
:10018000CFA50008D1A5000810B5054C237833B9D8
:10019000044B13B10448AFF300800123237010BD5A
:1001A000A402002000000000C4FC000808B5064BB3
:1001B0001BB106480649AFF300800648036813B137
:1001C000054B03B1984708BD00000000C4FC0008BF
:1001D000A8020020A402002000000000154B002B04
:1001E00008BF134B9D46A3F5803A00218B460F466E
:1001F0001348144A121A0AF054FE0F4B002B00D079
:1002000098470E4B002B00D0984700200021040097
:100210000D000D48002802D00C48AFF300800AF012
:10022000F3FD2000290008F055FA0AF0D9FD00BFBF
:100230000000080000800120000000000000000015
:10024000A4020020F0620020000000000000000076
:1002500030B4C3787BB902784FF461435109CEF2D0
:10026000000302F01F022031012000FA02F243F8DD
:10027000212030BC70474FF46D43CEF20003457827
:10028000DA6884780378D243C2F30222C2F104010F
:10029000C9B205FA01F10F2545FA02F2C9B22240AE
:1002A0000A4303F1604303F561431201D2B283F8BC
:1002B000002302784FF461435109CEF2000302F0AB
:1002C0001F02012000FA02F243F82120D1E700BF0B
:1002D000F0B444680B680A7924F0407424F4807404
:1002E000234343EA02234360CD680C6987688A6828
:1002F0004E794FF2FD732C43CCF2FF0322433B4077
:10030000134343EA460383600B7DC26A013B22F438
:100310007002DBB242EA0353C362F0BC704700BF15
:1003200000230360037143718360C3600361012391
:100330000375704770B44FF40C5290E84200C4F259
:10034000010285685468C06843F2E0033143CFF688
:10035000FC732943234001430B43536070BC704737
:100360000023036043608360C3607047836819B9EA
:1003700023F001038360704743F0010383607047FB
:10038000092970B421D901EB41041E3CC668072538
:1003900005FA04F526EA050503FA04F445EA040320
:1003A000062AC36020D90C2A02EB82022BD9413ADB
:1003B000C46A1F2303FA02F324EA030301FA02F1D9
:1003C00043EA0102C26270BC7047066901EB410456
:1003D000072505FA04F526EA050503FA04F445EABB
:1003E0000403062A0361DED8013A02EB8202446B61
:1003F0001F2303FA02F324EA030301FA02F143EA9A
:1004000001024263DFE7233A046B1F2303FA02F37E
:1004100024EA030301FA02F143EA01020263D2E78C
:10042000836843F080438360704700BFC06C80B234
:10043000704700BF036819420CBF002001207047BD
:10044000016846F21002002321F00101C4F2020209
:100450000160036043608360C360036121239042B5
:1004600043616BD046F22803C4F2020398426CD079
:1004700046F24003C4F2020398426ED046F258039B
:10048000C4F20203984270D046F27003C4F2020331
:10049000984272D046F28803C4F20203984275D0A3
:1004A00046F2A003C4F2020398423ED046F2B803DB
:1004B000C4F20203984273D046F21043C4F202031E
:1004C000984275D046F22843C4F20203984276D08F
:1004D00046F24043C4F20203984278D046F25843B1
:1004E000C4F2020398427AD046F27043C4F2020387
:1004F00098427CD046F28843C4F2020398427FD0EF
:1005000046F2A043C4F20203984200F0838046F210
:10051000B843C4F20203984201BF4FF4C843C4F287
:1005200002034FF03D52DA6070474FF4C043C4F20B
:1005300002030022C2F23D02DA6070474FF4C0436A
:10054000C4F202033D229A6070474FF4C043C4F2E4
:1005500002034FF474629A6070474FF4C043C4F2D0
:1005600002034FF474129A6070474FF4C043C4F210
:1005700002034FF074629A6070474FF4C043C4F2B4
:1005800002033D22C2F20002DA6070474FF4C0431A
:10059000C4F202034FF47462C2F20002DA607047E0
:1005A0004FF4C043C4F202034FF03D52DA6070478B
:1005B0004FF4C843C4F202033D229A6070474FF4DF
:1005C000C843C4F202034FF474629A6070474FF458
:1005D000C843C4F202034FF474129A6070474FF498
:1005E000C843C4F202034FF074629A6070474FF43C
:1005F000C843C4F202033D22C2F20002DA6070472F
:100600004FF4C843C4F202034FF47462C2F2000212
:10061000DA6070474FF4C843C4F202030022C2F20A
:100620003D02DA60704700BFCA680B68D0F800C0AE
:100630002DE9F0014F698E69CD690C6A42EA030821
:1006400048EA07073E434B6A35432C4344EA03021A
:100650008C6A42EA04034A6B8C6B48F23F071343EF
:10066000CFF21C0723430CEA07071F4307604469C6
:100670000A6BCB6A24F007041343234343610B69DD
:1006800043604B6883608B68C360BDE8F0017047CE
:100690000023036043608360C3600361436183613F
:1006A000C361036243628362C36203634363836320
:1006B000704700BF036819B923F001030360704756
:1006C00043F0010303607047416070470B060CD58F
:1006D0004369AAB143F08003802943610FD00368C6
:1006E00001F01E01194301607047802907D0002ADC
:1006F000F5D1036801F01E0123EA01010160704792
:1007000023F0800380294361F3D1704770B44FF424
:10071000C04246F20F454FF4C84421F0F023C4F222
:100720000205C4F20204C4F2020223F0C316A84276
:1007300088BF224696B1046804F01E0404EAD1245E
:1007400089004CBF5268126823F0821313EA02003A
:1007500002D0201C18BF012070BC7047446904F00F
:100760008004EDE710B44FF4C84246F20F444FF452
:10077000C043C4F20204C4F20202C4F20203A04263
:100780008CBF1046184611F0005F21F0F02121F0D7
:10079000821114BFC160816010BC704700222DE936
:1007A000F00113460126032703E001330232102B28
:1007B0002CD00D6806FA03F42540A542F5D1D0F8F7
:1007C00000C007FA02F4E44304EA0C0CC0F800C0CD
:1007D00091F804C0D0F800800CFA02FC4CEA080C36
:1007E000C0F800C091F804C00CF1FF3CBCF1010F4F
:1007F0000FD9C5682C40C460CC79C56804FA02F4EE
:1008000001332C430232102BC460D2D1BDE8F00179
:100810007047D0F808C004EA0C0CC0F808C091F882
:1008200005C0D0F808800CFA02FC4CEA080CC0F8AD
:1008300008C0D0F804C02CEA0505456091F806C050
:1008400045680CFA03FC1FFA8CFC4CEA0505456070
:10085000CFE700BF00234FF6FF72026003714371C0
:100860008371C371704700BF036919420CBF002038
:10087000012070470AB9418370470183704700BF68
:10088000CB08083301F0070130B4890050F8235039
:100890000F2404FA01F425EA040440F8234050F838
:1008A000234002FA01F2144340F8234030BC704761
:1008B00008B54FF4A843C4F20003984218D04FF48F
:1008C000B043C4F2000398421ED04FF4B843C4F2C0
:1008D0000003984200D008BD01214FF4000000F051
:1008E00091F94FF400000021BDE8084000F08AB9FA
:1008F00001214FF4001000F085F94FF400100021A1
:10090000BDE8084000F07EB901214FF4800000F0FE
:1009100079F94FF480000021BDE8084000F072B979
:10092000F0B5044685B068460D46A68800F0E8F8A4
:10093000029A4DF68363C4F21B33A3FB021326F025
:100940003F06980C3604360C87B23E43A6802388B7
:1009500023F001031B041B0C238048F2A0612B68C9
:10096000C0F201018B4222D85B00B2FBF3F292B2DB
:1009700001372784032A98BF0422A28323889BB2CD
:1009800043F00103238023886989AA8823F48163C3
:1009900023F002031B040A431B0C13439BB2238066
:1009A0002A89AB8913439BB2238105B0F0BDEE8841
:1009B0004BF6FF718E421DBF03EB830303EB8303F2
:1009C000B2FBF3F203EB43030CBFB2FBF3F242F4CE
:1009D000804292B213051B0D0BB942F001024FF495
:1009E000967344F6D35103FB00F0C1F2620181FB20
:1009F00000318909013142F400422184BDE700BF82
:100A0000002341F28832026083804BF6FF7203813B
:100A100043814FF48043C28083817047038829B9A2
:100A200023F001031B041B0C038070479BB243F0AF
:100A300001030380704700BF038829B923F4807342
:100A40001B041B0C038070479BB243F4807303802C
:100A5000704700BF038829B923F400731B041B0CE3
:100A6000038070479BB243F400730380704700BF5C
:100A70001AB901F0FE010182704741F001010182C3
:100A8000704700BF038829B923F480631B041B0C43
:100A9000038070479BB243F480630380704700BFBC
:100AA000038819B95B045B0C038070476FEA43430A
:100AB0006FEA53439BB20380704700BF01827047C7
:100AC000008AC0B2704700BF82B000230A0F0093B3
:100AD000019301900092009B21F07F4153B1019B53
:100AE00014330193019B1B6819420CBF00200120A5
:100AF00002B07047019B1833090C0193F2E700BF65
:100B000010B44FF46053C4F202039A6802F00C026E
:100B1000042A22D0082A26D04FF41052C0F2F40240
:100B200002604FF46053C4F2020320499C68C4F38E
:100B300003140C5D22FA04F242609C68C4F3822420
:100B40000C5D22FA04F484609B68C3F34233CB5CEF
:100B500022FA03F2C26010BC70474FF49052C0F208
:100B60007A020260DDE75C68596814F4800F5C6803
:100B700015BF4FF490534FF41053C0F27A03C0F2F4
:100B8000F40301F03F01B3FBF1F24FF46053C4F200
:100B90000203C4F388145B68C3F30143013302FB0F
:100BA00004F25B00B2FBF3F20260BAE7000000203F
:100BB0004FF46053C4F202031A6B19B922EA000021
:100BC0001863704710431863704700BF4FF46053B9
:100BD000C4F202031A6C19B922EA000018647047C3
:100BE00010431864704700BF4FF46053C4F202030F
:100BF0005A6C19B922EA00005864704710435864CF
:100C0000704700BF4FF46053C4F202031A6A19B967
:100C100022EA00001862704710431862704700BF54
:100C2000002270B44FF48064C4F201020388C4F25D
:100C30000104904218BFA0429BB214BF00220122BF
:100C400008D04FF48064C4F20004B0F1804F18BFA4
:100C5000A04223D14FF68F754C881D4045EA04030E
:100C60004FF4A0564FF48055C4F20005C4F20006BC
:100C7000B04218BFA8421FBF0D894FF6FF441C4069
:100C800044EA050303804B68C3620B8803850AB1FD
:100C90008B7A03860123838270BC70474FF44065D2
:100CA0004FF40064C4F20005C4F20004A04218BF6F
:100CB000A842D5D1CEE700BF00234FF0FF314160FD
:100CC0000380038143808372704700BF038829B982
:100CD00023F080031B041B0C038070479BB243F07E
:100CE00080030380704700BF038829B923F0010304
:100CF0001B041B0C038070479BB243F0010303806D
:100D0000704700BF038C23F001031B041B0C0384FA
:100D10002DE9F001038C8D8984884F88028BB1F80E
:100D200000C02F4322F07302002523F002034FF48A
:100D3000806612041B04C4F20106C4F20105120C01
:100D40001B0CBFB2A84218BFB042A4B242EA0C02C8
:100D500047EA030316D14FF6F775B1F80EC0B1F8A4
:100D600012800F8A8E881D4045EA0C0C4FF6FB73EB
:100D70004FF6FF4548EA070725400CEA0303BCB2DB
:100D800033432C43848002838A6842630384BDE832
:100D9000F001704700230380438083808360838158
:100DA000C381038243827047038B23F008031B0433
:100DB0001B0C194301837047B0F8443021B95B0420
:100DC0005B0CA0F8443070476FEA43436FEA53432B
:100DD0009BB2A0F84430704783899BB21AB923EACA
:100DE000010181817047194381817047C94389B2EC
:100DF0000182704783899BB21AB923EA010181817C
:100E0000704719438181704770B5038ACA8823F4FB
:100E100040531B041B0C1343038283898A880446B6
:100E200008890D4623F4B0534989024323F00C038B
:100E30001B040A431B0C92B21343A381A38AAA8901
:100E400023F440731B041B0C84B01343A382684635
:100E5000FFF756FE4FF4A0524FF48053C4F2010343
:100E6000C4F201029C4218BF9442A2890CBF039BAA
:100E7000029B12B2002A21DB286803EB830303EBF9
:100E800083038000B3FBF0F148F21F53A089C5F241
:100E9000EB13A3FB0152520900B21601642500288E
:100EA00002FB151213DB12013232A3FB0253C3F310
:100EB000431333439BB2238104B070BD2A6803EB14
:100EC000830303EB83035200B3FBF2F1DCE7D200B0
:100ED0003232A3FB0213C3F342133343EAE700BFEA
:100EE0004FF41652002302600C228380C3800381DA
:100EF00042818381704700BF838929B923F400535D
:100F00001B041B0C838170479BB243F40053838105
:100F1000704700BF838919B95B045B0C83817047FC
:100F20006FEA43436FEA53439BB28381704700BF2C
:100F3000C905C90D818070478088C005C00D704704
:100F400001F01F0310B4C1F342110124A14204FABD
:100F500003F30DD002290DD014302AB9026822EA19
:100F60000303036010BC7047026813430360F9E792
:100F70000C30F2E71030F0E7C1F3421310B401F087
:100F80001F020124012B04FA02F416D0022B0CBF1D
:100F9000028A828A92B2224003880124090A04FA52
:100FA00001F19BB219420CBF00200120002A0CBFA6
:100FB000002000F0010010BC7047828992B22240EC
:100FC000EAE700BF090A012303FA01F1C94389B224
:100FD0000180704770B52A4D2C688CB0002C4BD125
:100FE0006846FFF737FC06A8FFF79AF904200121AD
:100FF000FFF7DEFD10234FF40060C4F202006946E3
:10100000009303238DF804308DF80740FFF7C6FBEB
:1010100001214FF48070FFF7E7FD02A8FFF7A0F968
:101020004FF4803302A80393029404940594FFF7CD
:1010300081F94FF400500126C4F2010006A906947C
:101040008DF81C408DF81D4008940A948DF82C6092
:10105000FFF73EF94FF400502346C4F201000E2181
:101060003246FFF78DF94FF40050C4F201003146CB
:10107000FFF77CF9034B1E6001232B600CB070BDA1
:10108000C4020020546100204FF4005008B5C4F29F
:101090000100FFF7C5F940F2C023C2F200030122AC
:1010A0001A6008BD38B50D4C236805460BB9002001
:1010B00038BD4FF40050C4F201000221FFF7BAF925
:1010C0000028F4D04FF40050C4F20100FFF7AEF94D
:1010D000002328802360012038BD00BFC00200200B
:1010E00030B448F6396301EB4105941EC3F6E303BF
:1010F0000229C1EBC501D8BF144683FB0153D8BFF9
:10110000013AC917C1EB6301201848F21F54D51CDE
:101110000818C5F2EB1484FB02340430D31732EA0A
:10112000220228BF2A46A3EB641100EBA202C3EB04
:10113000E413521842F29340D218C9F2492080FBBE
:1011400002508018D317C3EBA000C0EBC000101AE8
:1011500030BC704770B40646002922D00078F0B148
:1011600000231846F25CA2F13004E4B2092CA2F18B
:1011700041050DD9052DA2F161049CBFA2F13704F0
:10118000E4B205D9052C9ABFA2F15704E4B20024B9
:101190000133DDB204EB0010A94280B2E2D870BC8A
:1011A00070470846FBE700BF0020C4F20200202180
:1011B0000122FFF75FBB00BF0020C4F20200202124
:1011C0000022FFF757BB00BF00B583B06846FFF7AA
:1011D00041FB01200146FFF7EBFC002020220346E3
:1011E0006946C4F20200009201228DF805308DF8A4
:1011F00004208DF806308DF80730FFF7CFFAFFF79F
:10120000DBFF03B000BD00BF00B583B06846FFF749
:1012100021FB04200121FFF7CBFC4FF400600023E9
:101220004FF40052C4F20200694600928DF8043077
:101230008DF80730FFF7B2FA03B000BD4FF400603D
:1012400008B54FF40051C4F20200FFF70DFBD0F1D6
:10125000010038BF002008BDF0B412490A680346F7
:10126000E2B11148114D066811482D680768114810
:101270009D6004681048114D00682D68D8600020FA
:10128000072C08BF04465D60013F06F164059C61C0
:101290000F245D611F6118621C6008601046F0BC7D
:1012A000704700BFF0020020C8020020F8020020B2
:1012B00000030020DC020020CC020020D402002029
:1012C000F0B583B068464FF40065FFF7C3FAC4F287
:1012D000020504200121FFF76BFC00244FF400639A
:1012E0006946284600938DF805408DF804408DF836
:1012F0000740FFF753FA6846FFF7ACFA04200121D4
:10130000FFF756FC4FF480570126284669460097A0
:101310008DF805408DF804608DF806408DF8074083
:10132000FFF73CFA284639463246FFF7A3FA03B0E6
:10133000F0BD00BFF8B5A44C2368FF2B56D04FF486
:101340000060C4F202004FF40061FFF78DFA054619
:10135000002833D0FFF728FF23689B4D0120012B85
:1013600033D04AD3022B4DD0984B1A68904200F0EC
:101370008680974E186033689A1F0221122A2960CE
:1013800063D9052B94BF93489348944F06F074FF9C
:10139000934806F071FF002323603B680F2B00F099
:1013A000CC81102B6ED0FF2B3AD001333B2B3B600E
:1013B00000F0CE8134D90023236031E0FFF7FCFE3A
:1013C0002368012B2846804DCBD1804B1A6882427E
:1013D00029D01860814BFF221A607D4B002814BF72
:1013E00003200220002220601A60F8BD7D4B1A689D
:1013F000642A19D001321A60F8BD01232B60734BA7
:101400001860F8BD714B1A68904238D0704E186061
:1014100033680322782B2A6012D9704B00221A609D
:1014200000233360F8BDF8BD4FF40060C4F2020041
:101430004FF480510022FFF71DFA00232360F8BD0E
:101440004A2BEDD800232B60EAE7644F0F2B3B6853
:1014500034D8232B00F097813A2B00F085811C2B88
:101460009CD1614A1268D0079FD5604806F004FFFE
:101470005B4806F001FF002323603B688EE7544B76
:101480001A68B7E75A4A002313605A4A1360564A4B
:101490001360594A1360594A1360594A1360594AF4
:1014A0001360594A1360594A1360594A1360594AE4
:1014B0001360594A136011233B60B1E7A3F1110295
:1014C000292A3FF66BAF01A151F822F0331700082B
:1014D0009D1300089D1300089D1300082D17000898
:1014E00027170008211700081B1700081517000808
:1014F0000F17000809170008F9160008F31600086E
:10150000ED160008E7160008E1160008DB160008D3
:10151000D5160008C5160008BF160008B916000841
:10152000B3160008AF160008AB160008A71600088F
:10153000A11600089B160008951600088F160008D3
:1015400089160008831600087F1600087B1600081D
:1015500069160008571600084516000833160008DB
:1015600021160008B7150008A515000893150008F6
:1015700075150008214A126812F001057FF415AFB5
:10158000264806F079FE164806F076FE25603B6890
:1015900004E72149194A0D681068503501300D6083
:1015A0001060FEE61C49154A0D68106828350130A8
:1015B0000D601060F5E61849104A0D681068143582
:1015C00001300D601060ECE630000020E0020020E9
:1015D000F402002048BF000868BF00082C0000206B
:1015E0007CE10008FC020020D002002088BF000837
:1015F000F0020020E802002004030020D8020020AE
:10160000EC020020D4020020F8020020DC020020BE
:10161000CC02002000030020C8020020D0BF000838
:101620006549664A0D6810680A3501300D60106022
:10163000B7E66149614A0D681068083501300D60F0
:101640001060AEE65C495D4A0D68106804350130F3
:101650000D601060A5E65849584A0D6810680235BB
:1016600001300D6010609CE65349544A0D681068C3
:10167000013501300D60106093E65149D1E75049C2
:10168000D8E74F494D4ADFE74D494C4AE5E74C4919
:101690004A4AEBE74B49494AD6E74A49474ADCE719
:1016A0004849464AE2E7484986E74749B9E7464993
:1016B000C0E74549414AC7E74349404ACDE7424967
:1016C0003E4AD3E7414A126812F001057FF46DAE3D
:1016D0003F4856E73F493D4A6FE73E493B4AA1E74D
:1016E0003C493A4AA7E73B49384AADE73949374AC6
:1016F000B3E73849354AB9E7374A126812F00105AD
:101700007FF453AE35483CE73549334A4CE734491A
:10171000314A52E73249304A84E731492E4A8AE752
:101720002F492D4A90E72E492B4A96E72C492A4A01
:101730009CE72C4A0121116033E62B4B1A6822B139
:101740002A4A0121116000221A6010233B6067E6DB
:10175000274B204A196812689142264922D0204816
:1017600000681A6008605BE6144A1268D2077FF5C9
:101770001CAE214806F080FD204806F07DFD0022C9
:101780003B682A600AE6114A1268D1077FF50DAE60
:101790000F4806F071FD194806F06EFD00232B601E
:1017A0003B68FBE50E480C68006801348442D8D1E0
:1017B0000D4C01252560D4E7C8020020D802002086
:1017C00000030020DC020020CC02002004030020E3
:1017D000ACBF0008F8020020D002002088BF00083B
:1017E000D4020020EC020020E8020020F0020020D9
:1017F00008030020E4020020D0BF00087CE10008BC
:10180000034B1A6812B11A68013A1A60704700BF98
:1018100058610020064B074A1B68012B1EBF064B70
:101820001B68B0FBF3F010601368002BFCD170470D
:101830000C0300205861002038000020044B054AAA
:101840001B6803FB00F010601368002BFCD170478D
:101850003400002058610020084B094A1B684FF4EF
:101860007A7110F1FF3001FB03F106D311601368A8
:10187000002BFCD110F1FF30F8D27047340000206B
:1018800058610020012810B423D002282CD01C4B12
:1018900064221A601B4B0A221A6042F21071032064
:1018A000194B1C684EF21003CEF200034FF46D4248
:1018B000B4FBF1F1CEF2000201395960F02182F857
:1018C000231000229A6007221A60104B186010BC87
:1018D00070470B4B18600B4B44F240214FF47A7267
:1018E0001A60C0F20F01DBE7054B0A221A60054BB4
:1018F00048F2A06164221A60C0F20101D0E700BF83
:101900003800002034000020D80100200C03002003
:101910002DE9F00140F2701040F2A41540F24C01A4
:10192000C2F20000C2F20001C2F2000540F26C14E3
:1019300040F23C0240F24003C2F20002C2F2000355
:1019400090F8008090F801C087780E7848782D686C
:10195000897882F80080C2F2000482F801C0256014
:1019600097701E7058709970BDE8F001704700BF05
:1019700040F2211009F092B840F2851009F08EB8BB
:10198000F8B506460F4640F2211440F28515204670
:101990003146013409F022F9AC42F8D107B9F8BD5B
:1019A000BDE8F840FFF7E8BF30B540F24002C2F2B0
:1019B00000024CF2F433C0F60003117894785578A5
:1019C00033F8111033F8152033F8143083B08DF844
:1019D0000410014601A88DF805208DF80630FFF7A8
:1019E000CFFF03B030BD00BF00B583B00023014678
:1019F00001A88DF804308DF805308DF80630FFF71A
:101A0000BFFF03B000BD00BF30B51A4B1A4D1B68B5
:101A10008DB0EBB100232A461C46116911F0020F6C
:101A200002F1140205D00CA800EB8401013441F846
:101A30002C3C01330B2BF0D16CB9104A23461460B7
:101A400003EB830305EB83056B6898470DB030BD4E
:101A50000A4B1B68F4E709F0B9FCB0FBF4F30CAADD
:101A600003FB140002EB8003044A53F82C3C136080
:101A7000E6E700BF5804002050000020400300208B
:101A80000E2A30B436D81F4B0C789B5C48F689027E
:101A900013FB04F4C8F68802A2FB0452C2F3C70287
:101AA00002700C7814B10AB9012202704C7848F621
:101AB000890213FB04F4C8F68802A2FB0452C2F3A5
:101AC000C70242704C7814B10AB9012242708C7876
:101AD00048F6890213FB04F3C8F68802A2FB03420E
:101AE000C2F3C70282708B7813B10AB901238370E5
:101AF00030BC70470B7803704B7843708B788370E1
:101B0000F6E700BFE8C4000810B5104B104C1A6887
:101B1000104982B02046FFF7B3FF0F4B1B689BB103
:101B20000E4B2178A078627833F8111033F8122028
:101B300033F810308DF8041001A801218DF805202C
:101B40008DF80630FFF71CFF02B010BD6C010020BD
:101B5000400000203C00002074010020F4C3000875
:101B60000E4B1B68032B18D8DFE803F013100A0292
:101B70000B4B00223F2119705A709A70FFF7C4BFB7
:101B8000084B012200201A60FFF72EBF0020FFF74C
:101B90002BBF054B1868FFF707BF70472C040020C8
:101BA0003C0000205C040020740100202DE9F00FAF
:101BB0000B0682B04BD46FEA020ADFF808C1404B33
:101BC0000AF1090A072A88BF4FF0000A00F1080647
:101BD000C2F10708042703EBC10B8244CDF804804F
:101BE000B61A0124ACF14805072A16D801990BEB67
:101BF00007090346112B0CD819F8048C48FA01F890
:101C000018F0010F1ABF4FF004080CF803800CF80D
:101C1000034001330139B342ECD1BAF1110F9FBF38
:101C200007EBC708534651464FEA480801D905E07B
:101C3000194641440133112B6C54F9D901370C2F4B
:101C40000CF1120CD0D102B0BDE8F00F7047B039E2
:101C50004C2932D8DFE801F02F31313131313131C7
:101C60003131313131313131313131312D31313168
:101C700031313131313131313131313131312B315A
:101C80003131313129313127313131312D3131315A
:101C900031313131313131313131313131312B313A
:101CA000313131312900052185E7042183E7032102
:101CB00081E702217FE701217DE720217BE700BF4B
:101CC000F4BF0008A8610020B0F5907F10D248F65C
:101CD0003963C3F6E303A3FB00239B08DA0742BF83
:101CE00003EBC303C0EB83001130013008F076BF73
:101CF000704700BF70B5294B1A6882B006460AB912
:101D000001261E60264A274B11785478907833F8C4
:101D1000111033F8142033F81030234D8DF80010D3
:101D200000248DF801208DF802308DF804408DF8E4
:101D300005408DF806400BE0FFF7C6FF15F8013CA3
:101D4000013443F00103B4F5907F05F8013C16D04F
:101D500015F8013B03F00203DBB220466946002B75
:101D6000EAD1204601A9FFF7AFFF15F8013C013485
:101D700023F00103B4F5907F05F8013CE8D116B1DA
:101D80000A4B1B6833B1FFF7F3FD094B01221A60C0
:101D900002B070BD0120FFF707FEF6E74404002003
:101DA0004C000020F4C30008606100202C040020D7
:101DB0005C61002008B5064B1A6822B1002210466B
:101DC0001A60FFF797FF034B01221A6008BD00BF9E
:101DD000580400205C61002008B50D4B0D481A68BE
:101DE0000D49FFF74DFE0D4B1B68032B03D00C4B29
:101DF0001B68990708D40B4B1B6803B908BD012069
:101E0000BDE80840FFF776BFFFF782FDF3E700BFAC
:101E1000A40100204C000020700100202C040020B0
:101E200044000020740100202DE9F041864B1A681F
:101E300084B03AB985490B68002B00F0E48004B007
:101E4000BDE8F081824A81491678DFF81C824CF6A1
:101E5000CD40CCF6CC40A0FB0650002400091C600D
:101E60000C6000F0B580C8F800005578DFF8FCC1C0
:101E70004CF6CD43CCF6CC43A3FB05031B0902D1A2
:101E8000002D40F0BE80CCF800309478714F4CF6B5
:101E9000CD43CCF6CC43A3FB04231B0902D1002C79
:101EA00040F0AD806C4A3B606C4B0020107050706D
:101EB00090701E705D709C70D8F800301C4693B115
:101EC000664A1478A34240F2968014B10020107044
:101ED0000124614A5E4815780078EB18834200F2CD
:101EE000A28013700124DCF800308BB15B4842788B
:101EF00093427CD912B1002242700124564A5448C0
:101F000055784078EB18834200F292805370012498
:101F10003868002863D0514B9A78904263D912B147
:101F200000229A7001244C4D494AAF7896783818AF
:101F3000B0429CBFC0B2A87003D9B7424FD0AE70B8
:101F40003046474992F800C092F801E06C782F784B
:101F50005A781D789B7831F81C8031F8177031F869
:101F60001EC031F8122031F816E031F8133031F884
:101F7000146031F8104031F815008DF80A40394DE1
:101F80008DF804808DF805C08DF806E08DF8087096
:101F90008DF809608DF80C008DF80D208DF80E304D
:101FA000002407E0012B34D0032B37D00134B4F5E3
:101FB000907F0AD0635D022BF4D1204602A9013440
:101FC000FFF782FEB4F5907FF4D1FFF7D1FC36E73E
:101FD000002E3FF448AF0123C8F8003045E764BB4A
:101FE00001230B602BE7121A9A7001249BE7D21A87
:101FF0004270012482E7E41A1470012469E7012386
:1020000050E701233FE7DFF86080DFF860C0114F41
:1020100052E7204603A9FFF757FEC7E7204601A96C
:10202000FFF752FEC2E785421CBF107001245AE739
:1020300085421CBF507001246AE7054A064D967818
:10204000A878064B7DE700BF580400205C610020A3
:102050004C000020200400203C030020100300203E
:10206000F4C3000860610020700300205C030020BE
:1020700070B5154A154B94781178557833F81110CE
:1020800033F8152033F81430114E82B000248DF847
:10209000001005468DF801208DF802308DF80440BF
:1020A0008DF805408DF80640A35D2B42204601A91E
:1020B00018BF69460134FFF707FEB4F5907FF3D1EE
:1020C000FFF756FC02B070BD4C000020F4C30008BE
:1020D000606100202DE9F8435A4B5B4D1A682AB91C
:1020E0002E68002E00F09980BDE8F883DFF860814B
:1020F00000221A602A60C8F80020544C4FF0000EED
:102100007646A4460EEBCE00400012230CEB0009ED
:102110005A1E81186718615C11F0010F45D0112A11
:1021200000EB03064AD01CF80660F60741D421F004
:1021300001013970002A46D0023B0126002BE7D16D
:102140000EF1010EBEF1100FDCD10120FFF790FF60
:10215000002E5ED0D8F800300126012B08BF3B4C82
:10216000C2D13A4F4FF0000EB8460EEBCE00400001
:10217000002308EB000CC21804EB0209A25C02F079
:102180000601022926D00133112BF4D90EF1010EDC
:102190001237BEF1100FE8D10420FFF769FF002EBF
:1021A000A2D101232B60BDE8F8831346002BAFD1E9
:1021B000C6E713460126002BAAD1C1E721F0010191
:1021C00089F81110B8E70EF1010E0126BEF1100FCB
:1021D00098D1BAE743B302F00401C9B20029D2D1C1
:1021E00042F00402112B89F8002022D00133C218DA
:1021F000A25C02F00202D2B24AB1112B03F1010338
:1022000017D0FA5C02F00202D2B2002AF5D1012600
:10221000BAE70123C8F80030A3E7DFF83480D8F824
:102220000030002B99D168E742F004028CF80020BE
:10223000DCE70EF1010E01261237BEF1100F94D12A
:10224000AAE700BF580400205C6100206061002004
:10225000340400202DE9F00F6A4B1A6832B96A4A3B
:102260001368002B67D0BDE8F00F7047002018609E
:10227000654A664E664B1060012131601960336813
:102280008BB1644810256C1E0023C25C02F0030170
:10229000012936D00133122BF7D112382546002CF4
:1022A000F1D134603FE0DFF868A1DAF800100029CE
:1022B0003ED0DFF874B1DBF80020002A3DD0564D47
:1022C000564A29681068564A564E01EBC10400EB85
:1022D00044040131175D296027F0040701EBC105B3
:1022E00000EB450017553668145CB14244F0040514
:1022F00008BF44F00504155404BFCBF80030145453
:1023000011E004EBC400464903EB400022F0010257
:102310000F2C0A5407D005EBC50503EB4503CA5C37
:1023200042F00102CA540520BDE8F00FFFF7A0BE3D
:102330000123136097E7354EA1E740F24431C2F222
:10234000000140F238330F68324840F21831C2F2CF
:102350000003C2F20001D3F80090D1F80080944647
:102360001026A0F58775741ED30748D40023C25CDD
:1023700002F00301022905D00133122BF7D14B469D
:10238000002210E0A4B112F0010216D006EBC60242
:1023900003EB4202B046A95C41F00401A9544FF09E
:1023A000010C27460122264612388CB19946DAE7FD
:1023B000EA5C42F00502EA54F3E7BCF1000FF0D109
:1023C000E95C41F00401E9544FF0010C9046E8E764
:1023D00040F24431C2F20001CBF800C00F6040F27D
:1023E0003831C2F200010B6040F21833C2F2000330
:1023F000C3F80080002A96D1CAF8002093E74B4624
:10240000D1E700BF580400205C6100204C0400208C
:10241000500300206E6200201803002038030020C3
:102420006061002044030020CC0300202DE9F84324
:10243000694B1A6832B9694D2B68002B00F0A180F6
:10244000BDE8F88300201860654C644B206018607C
:102450004FEAC00C0CEB00035B00624A1918C0F194
:1024600012061546F3188A18EF18A846134619786D
:1024700041F0040103F8011BBB42F8D1C0F10F0E7B
:10248000431C734528BF4FEACE0C1BD20CEB000750
:10249000C0F1110300EB08014FEACE0C03EB470338
:1024A00012390CEB0E075B1901EB4707917C41F0E9
:1024B000040102F8121F997CBA4241F0040103F8AA
:1024C000121FF3D10CEB0E0205EB42020346D15C66
:1024D00041F00401D1540133B342F8D3002848D06D
:1024E000421EC0F11307BA420FD202EBC2014900EB
:1024F0000B185B197E19013B761813F8011B21F0AC
:102500000401B34203F8011CF7D1C0F110084045A3
:1025100028BF4FEAC8091DD200EBC0034FEAC80923
:1025200002EB4303511909EB080CC0F112065B19C9
:1025300001EB4C0C93F800E0991A2EF0040E83F88E
:1025400000E011F806E012332EF0040E634501F8A6
:1025500006E0EFD109EB080300EB43035B19013BF5
:1025600013F8011B013221F00401BA4203F8011CE7
:10257000F6D30420FFF77CFD236801332360BDE818
:10258000F883174C206807287FF662AF08281CBF25
:10259000144B03F5907404D119E0A34203F8010C25
:1025A0000ED013F8012B02F00201C9B242F0040070
:1025B00022F004020029F0D1A34203F8012CF0D14B
:1025C0000420FFF755FD01232B60BDE8F8830722A7
:1025D0000B27044D89E700BF580400205C610020F0
:1025E000780400206061002070B5264A26481368F0
:1025F0001BB90368002B3BD070BD00231360234D33
:10260000234A03602B6013602E6886B9214B03F5C3
:1026100090711A7822F0040203F8012B8B42F8D152
:102620000420FFF725FD2B6801332B6070BD184A8D
:10263000136801331360DA07DED5741EA4B2B4F553
:10264000907F10D213490B5D03F00202D2B22AB17F
:1026500010E00B5D03F00202D2B25AB90134A4B209
:10266000B4F5907FF5D10123036001362E6070BD73
:10267000064DC9E743F0040304200B55661CFFF721
:10268000F7FCF2E7580400205C610020640300209E
:1026900028040020606100202DE9F00F8D4A1368A6
:1026A00086B043B98C4B1A68002A00F0098106B045
:1026B000BDE8F00F704700231360884C864A236002
:1026C00013600393864F002000EBC00207EB420229
:1026D00000231178013321F00401122B02F8011BB1
:1026E000F7D101301028EFD1039B03F10109C3F1A9
:1026F0000806C4F8009001960020C2190023117842
:10270000013321F00801122B02F8011BF7D112301E
:10271000B0F5907FF1D1019A714DCDF808905342F8
:1027200093469A4600269946BAF1080F2CBFD04628
:102730004FF008084A4601990023BBF1070F34BF48
:10274000DC464FF0070C17E0082934BF0846082084
:10275000082B644603D9092A2CBF1046092004EB34
:10276000C40400EB44003C5C44F008043C540133D6
:1027700001310132122B15D0E85C00F00200C0B22A
:102780000028F4D0072EDFD9082B05D8082934BF3C
:10279000084608204446E2E7082A8CBF1046092074
:1027A0004446DCE701361235102E0AF1010A0BF11E
:1027B000010BB9D1039EDDF80CB0DDF808900023C1
:1027C00001936FF0110303FB067302936FF0120C79
:1027D0006FF023035A460CFB06FCD24303FB06F6BC
:1027E0000596CA464FF000080492039E049B0BEB2B
:1027F000CB056D00AA19019EED18F119D219ED193A
:102800004C4600231DE0082B2ED8C14509D8994518
:1028100007D8059EA81910F8126C46F0040600F8B7
:10282000126C11F8010B00F00806F6B21EB140F070
:10283000040001F8010C0133013201350134122B7F
:1028400029D012F80C00C007EBD5B8F1070FDAD980
:10285000082B16D8BAF10F0FE3D89945E1D8A87C18
:1028600040F00400A874DCE7C145DAD8112CD8D8B0
:10287000029E301910F8126C46F0040600F8126C33
:10288000CFE7BAF10F0FCCD8112C9EBFD07C40F00F
:102890000400D074C5E7019A029B08F101081232C6
:1028A0001233B8F1100F01920BF1010B02930AF1F0
:1028B000010A9AD1042006B0BDE8F00FFFF7D8BB9B
:1028C000064C2268082A03927FF6FCAE01221A60A9
:1028D000EDE600BF580400205C6100207004002079
:1028E000606100202DE9F84FA94C2368002B40F0CF
:1028F000A880A84B1B68032B12D8DFE803F07646AC
:1029000013022368002B40F0CA80A34A13683BB926
:10291000A2490B68B3F5907FC0F0C8800123136013
:10292000BDE8F88F2368002B00F0A18098499C4BEC
:1029300000220A6098491A600A609A4C02F1120556
:1029400004F112081D600021C2EB08088B1A1B1944
:1029500008EB01000DE013F8126C16F0010F9E5CFD
:1029600000F0088146F004069E540133984200F0BE
:1029700008818D42EFD993F80E6106F00206F6B297
:10298000002E00F0F6809E5CECE72368002B79D0E7
:102990007F49854A00230B607F4913600B605F1CF1
:1029A000804C17601E4603F5907C594203F11300DA
:1029B00033193A460DE05D7815F0010F5D5C00F0CB
:1029C000CB8045F0040501325D540133824200F0B2
:1029D000CB80112AEFD913F8115C05F00205EDB296
:1029E000002D00F0B8805D5CEBE72368002B33D04E
:1029F000674A6E4B00211160674A19601160481CDC
:102A0000684C18604E42C1F59077331900220EE0F1
:102A100013F8015C15F0010F5D5C00F08F8045F04C
:102A2000040501325D540133122A00F08F80904278
:102A3000EED95D7C05F00205EDB2002D7DD05D5C28
:102A4000EDE708F0C3FCC3179B0FC21802F00302A6
:102A5000D31A504A13604EE74F4A1368002B7FF495
:102A60005FAF524B196811293FF658AFC7E74A4983
:102A70000B68002B7FF454AF494B1A68B2F5907F76
:102A800009D25AE744490B68002B7FF449AF464A04
:102A90001368112B83D901230B60BDE8F88F3C4AE2
:102AA0003E49002313603C4A0B6013603D4C4FF6D7
:102AB000EE7A03F11202CFF6FF7A0A6003F5997BF2
:102AC00004F11208C3EB0A0A40F21F16A2F5907136
:102AD0000AEB02000919131902EB080510E091F83E
:102AE0002071C2EB0309FF07CC4614D519F800701A
:102AF000013347F004070131AB4209F8007014D0EC
:102B0000B242ECD90F7807F00207C2EB030CFFB218
:102B1000E146002FEAD11CF80070013327F00407CA
:102B20000131AB420CF80070EAD112325A45CDD1D6
:102B30000420BDE8F84FFFF79BBA5D5C25F0040563
:102B400001325D540133122A7FF471AF1236BE4256
:102B50007FF45BAFECE75D5C25F0040501325D546A
:102B6000013382427FF435AF123666457FF420AFE1
:102B7000DEE79E5C26F004069E54013398427FF403
:102B8000F8AE1231B1F5907F7FF4E0AED0E700BF30
:102B9000580400206C0300205C6100201C0300200E
:102BA000C003002060610020C40300207C040020DA
:102BB0002DE9F04FB24AB34E136885B033B933688C
:102BC000002B00F0968005B0BDE8F08F0023136065
:102BD000AD4AAE4C1360AE4AAE4D1360AE4A3360A0
:102BE00023602B6013602368002B43D1AB4A11781C
:102BF0001F295FD951781F2900F2C6803F228DF826
:102C000008308DF809208DF80A30A54B9E4F1A68C0
:102C100003A802A9FEF734FFA2492E689DF80C8094
:102C20009DF80DC09DF80EE09F4B38689F4A31F823
:102C3000188031F81CC031F81EE083F8008006EBE4
:102C4000C60100EB41000026194683F801C083F855
:102C500002E0167056709670FFF736F82368296800
:102C6000934A3868D15493495A1CC8542260FEF7DD
:102C70007FFEA8E72A681C2A24D98F4B03F590749D
:102C800003E0A34203F8010C0ED013F8012B02F06D
:102C90000201C9B242F0040022F004020029F0D17E
:102CA000A34203F8012CF0D10420FFF7E1F901233E
:102CB000336088E73F228DF808208DF809308DF8C1
:102CC0000A30A2E7DFF8C8E16F4FDEF80030D7F82E
:102CD00000C09A4277D0704B1B6802F00109B9F12D
:102CE000000F4AD163452DD90CF101033B602A68DE
:102CF0002FE0664C674D76E7BBF1110F19D85B46A4
:102D000008EBC80046F2601C03EB4000C2F2000C66
:102D10001CF800C01CF0010FDDF800C004D0E0E09A
:102D2000C85CC00700F1DD800133122BF8D1CDF86B
:102D300000C008F101081231B8F1100F65D11D2350
:102D4000CEF80030DEF800309A4228D301232A68FA
:102D500033600F2A2ED92368DFF854810D2B78D0E9
:102D6000544E29683A6808F803100C2BF25401D825
:102D700001332360FEF7FCFD25E76345E2D20CF149
:102D8000FF333B602A68E4E792781F2A0AD88DF85F
:102D900008308DF809303F238DF80A3035E70132CD
:102DA0002A60D6E73F228DF808308DF809208DF88B
:102DB0000A202AE738683C4902EBC20200EB4200D5
:102DC000FEF782FFC7E740F24830C2F20000036816
:102DD0009C4582D112F0010900F08B800CF1FF3B81
:102DE0009246BCF1000F02D102F1010AE346BAF1AA
:102DF0000F0FA4D846F260130AEBCA01C2F2000317
:102E000003EB4101D046CDF800C0D0455FD018F0AB
:102E100001033FF475AF112308EBC80046F2601CB4
:102E2000C2F2000C03EB40001CF80000DDF800C00B
:102E3000C00706D4002B3FF47AAF013BC85CC00743
:102E4000F8D540F24830C2F20000CEF800800360AE
:102E500045E798F80030174E0F2B2FD90023013388
:102E600008EB030218F80300F15C02F8010CF218F9
:102E70000C2B02F8011CF2D12368013B236070E7A0
:102E8000580400205C61002038040020BC030020AE
:102E9000580300204804002048030020700100204F
:102EA000A4010020F4C3000854040020740400208E
:102EB0006004002020030020606100203078114968
:102EC00003EBC30300EB4300FEF7FEFEC6E718F07A
:102ED000010F3FF411AFBBF1FF3F18BF5B469BD121
:102EE00027E740F24831C2F20001CEF800800B60C3
:102EF000F5E6BCF1100F9CBF0CF1010B92467FF67A
:102F000076AF71E7740400202DE9F04F804B814CBF
:102F10001A6885B0002A40F098802368002B57D1AA
:102F2000DFF808B2DBF800202F2A54D8DFF8F0A130
:102F3000DFF8F4819AF800009AF801109AF802205C
:102F40008DF80C008DF80D108DF80E20994658F86C
:102F5000044B182C2DD9A4F11805012D63D0A4F130
:102F60001A030F2B67D90F2D5DD904EBC407193C49
:102F7000A9F5EA730126A51E0F2C03EB470709D913
:102F80000E2D45D90136243F6B1C2C460FD0A51EB3
:102F90000F2CF5D89AF8013007F11200B3FBF6F3C5
:102FA00003A98DF80D30FEF78FFE002CE8D158F8FC
:102FB000044C09F101090134B9F1120F48F8044C2D
:102FC000C5D1FEF7D5FCDBF800300133CBF800307B
:102FD00005B0BDE8F08F504B03F5907503E0AB42B0
:102FE00003F8010C0ED013F8012B02F00201C9B254
:102FF00042F0040022F004020029F0D1AB4203F8B1
:10300000012CF0D10420FFF733F801232360DFE720
:103010009AF801303846B3FBF6F303A98DF80D306A
:10302000FEF752FEAEE705EBC50009EB40003B4959
:10303000FEF74AFE99E705EBC500A9F1240303EB6F
:1030400040003749FEF740FE8DE7364A364FD2F84A
:10305000008000261E60354B26603F25424602A8B0
:1030600069461E6010238DF806308DF800508DF8EB
:1030700001508DF805508DF802608DF80460FEF760
:10308000FFFC424603A801A9FEF7FAFC284B9DF875
:1030900008809DF809C09DF80AE09DF80C509DF845
:1030A0000D009DF80E901D491D4A33F8155033F858
:1030B000188033F81CC033F81EE033F8100033F8E2
:1030C0001930157081F8008081F801C081F802E0A4
:1030D0005070937035460DE008F078F9C3171B0F58
:1030E000C01800F00F00C31ABB5101350436122D71
:1030F0003FF413AFEA07EFD408F068F9C3171B0FCA
:10310000C01800F00F00C31A0833BB51EDE700BF31
:10311000580400205C610020606100203004002021
:1031200060030020A401002074030020500400204C
:10313000F4C3000810B582B0002914BFFF23002398
:10314000002814BFFF240024002A14BFFF220022FD
:10315000002001A98DF804408DF805308DF8062077
:1031600007F03CFD012007F099FC02B010BD00BF44
:10317000074B012003F5907113F8012B12F00202A6
:1031800014BF03F8010C03F8012C8B42F4D17047F3
:10319000606100202DE9F84F1746814688460AB93C
:1031A000BDE8F88F0020FEF7A5FD39077FD4FA06A9
:1031B00079D44B4A4B4B126803EBC20113F832B07F
:1031C00091F801A07B07EBD5474E48484B220021E0
:1031D00007F067FE06F590750122334613F8014BA0
:1031E00014F0020414BF03F8012C03F8014CAB42A5
:1031F000F4D13F4B1B68002B67D03E4B1B68D807B0
:1032000067D53A4B01225A709A703B4B374CCBEB47
:103210000B1B08EB8B0103EBC10101200023CA1833
:103220000133527812B1072BA054F8D10B782F4CF0
:103230009944B9F1180F0AEB8A0A88BFA9F1190954
:103240002E4B0AEB8A0A0AEB090003EB80000121EE
:103250000023C25C013312B1042BA154F9D1284CD4
:10326000DFF8A8C004F14B07002514F8013F93B123
:1032700005EB0C0315F80C2098785B7858B102EB3D
:10328000C202181806EB4202D15C41F00201D1548F
:1032900001338342F8D10335BC42E6D1194B0122F8
:1032A0001A60BDE8F88F0120FEF79EFB81E706F06B
:1032B00089FDC820FEF7C2FA134B1B68002B7FF470
:1032C00078AF0120FEF770FB73E7F9067FF568AF72
:1032D000E4E7B8F1000F18BFB8F11E0F95D190E7E1
:1032E00068030020ACDE000860610020D0030020ED
:1032F0007401002044000020F8C4000898D9000898
:10330000CF030020580400202C040020C8DD000852
:1033100040F24403C2F200031868704738B50B4B03
:103320000B4D1B68032B044604D0830702D52B6882
:10333000980707D5FEF714FC064B2C6001221A6093
:10334000204638BDFEF7E4FAF4E700BF2C04002065
:10335000440000205804002040F22C43C2F2000335
:1033600018687047032810B509D8074C23688342B2
:1033700003D02060FEF7F4FB2368184610BD024B13
:103380001B68184610BD00BF2C04002040F27813C3
:10339000C2F20003186870476328024B88BF64209C
:1033A000186070477801002040F2A813C2F20003B1
:1033B000186870476228024B88BF00201860704769
:1033C000A801002040F26833C2F200031868704779
:1033D0001128044B04D81860034B01221A6070476F
:1033E000186870476803002058040020064B1868CE
:1033F000102805D900201860044B01221A6070477C
:1034000001301860F8E700BF68030020580400206E
:10341000054B186828B101381860044B01221A6066
:10342000704711201860F8E7680300205804002056
:1034300040F23C43C2F2000318687047074B10B5D6
:10344000186000B110BD064B0F241C60FEF7C4FCD1
:10345000044B1C60BDE81040FEF756BB3C04002046
:10346000A40100206C01002040F2A013C2F200036E
:1034700018687047024B0A288CBF1868186070479C
:10348000A0010020044B1868092802D90020186008
:103490007047013018607047A0010020044B186885
:1034A00010B10138186070470A201860704700BFDB
:1034B000A0010020064B1B68012B00D07047054B74
:1034C00000223F2119705A709A70FEF785BC00BF28
:1034D000C80300207001002040F2C833C2F200038C
:1034E00018687047012810B5034602D9054B1868C3
:1034F00010BD044C2068984203D02360FFF7DAFF28
:10350000206810BDC8030020F0B5584B1B68012B84
:1035100083B0044642D0022B01D003B0F0BD20B9E5
:10352000534B1A68002A7AD018600020FEF75CFA24
:10353000504B1B683B2B2ED81D2B73D967081E25BB
:103540004D4A4E4B10785178927833F8100033F88A
:10355000111033F81220464B8DF804001B688DF8CB
:1035600005108DF80620002B46D1AF423CBF444EDB
:103570003C4606D339E000F2211007F02FFBAC42A5
:1035800033D2306820180134A84201A9F3D33C3863
:103590006328F4D8EFE727463C25D1E70020FEF763
:1035A00023FA344B1B683B2B48D9354B1A683C2314
:1035B000A418314AA34298BFC3EB040411782F4BDF
:1035C0009078557833F8111033F8152033F810300F
:1035D0008DF80410632C8DF805208DF8063004D882
:1035E00004F2211001A907F0F9FA264B1B68002B01
:1035F00093D0FEF7C1F990E7214E002405E000F2D8
:10360000211007F0EBFABC42EFD83368E018013420
:10361000A84201A9F3D33C386328F4D8EFE701228C
:103620001A6082E7132B7FF678AF4AF6AB27CAF60B
:10363000AA27A7FB04377F08142581E71D2B0ED886
:10364000132B7FF66AAF0E4A4AF6AB23CAF6AA23BB
:103650001268A3FB041402EB54041423A9E7084BDB
:103660001A681E2302EB5404A3E700BF2C040020B9
:103670005C0400207801002040000020F4C3000812
:10368000A80100207401002038B5814B1B680A2B6B
:103690001AD8804A804C12687AB9804D2A68C2B91B
:1036A0007F49804A03EB830301EB83031168986829
:1036B00001318142116045D238BD794A03EB830361
:1036C00002EB83035B689847744B1B68002BF3D0B5
:1036D000714C754B1B68012B1FD0744B1B68032B5F
:1036E00006D02368002BE7D1BDE8384006F088BB40
:1036F0006F4B70491A68496B0132B2EB411F1A6077
:10370000EFD36D490A680020013A1860052A3AD8BB
:10371000DFE802F059A19A938C50684B68491A6807
:1037200049690132B2EB411F1A60D6D365490A6874
:103730000020013A1860052A0CD8DFE802F0625B2D
:10374000544B70695B680021116098472B68002B0F
:10375000BED1B1E75C4A13680133072B00F09680B5
:103760005A48136002680B6001320D2A5549026005
:1037700000F083800E2AB0D1013B08BF06230B6006
:1037800000230360A9E7524A13680133072B72D064
:103790005048136002680B6001320D2A46490260EE
:1037A00060D00E2A9DD1013B08BF06230B60002389
:1037B000036096E7484B9A78002AE4D0013A9A7061
:1037C000FEF7A2F98DE7444B5A783E2ADBD8013246
:1037D0005A70F5E7414B5A78002ABBD0013A5A702B
:1037E000FEF7FAFA79E73D4B9A783E2AB2D80132D1
:1037F0009A70F5E7394B1A78002AABD0013A1A7063
:10380000EEE7364B5A783E2AA4D801325A70E7E7E1
:10381000324B9A78002A9DD0013A9A70E0E72F4BFC
:103820001A783E2A96D801321A70D9E72A4B1A78AC
:103830003E2AA8D801321A70C2E7274B5A78002ACC
:10384000A1D0013A5A70BBE7234B9A783E2A9AD806
:1038500001329A70B4E7204B1A78002A93D0013ACB
:103860001A70ADE70133072B18BF0B607FF439AF37
:1038700001230B6035E701238AE70133072B18BFCB
:103880000B607FF42AAF01230B6026E7012367E773
:10389000A001002058040020740100205C61002079
:1038A000500000201C040020C80300202C0400202D
:1038B0004C0300202C0100203003002024040020B1
:1038C0007C01002054030020340300204800002025
:1038D000140300209C0100203C0000207001002007
:1038E000064B1A783E2A07D803D13F221A70FEF7FA
:1038F00073BA02321A70FAE7704700BF70010020F5
:10390000064A137843B1012B03D100231370FEF74D
:1039100063BA023B1370FAE7704700BF70010020E2
:10392000064B5A783E2A07D803D13F225A70FEF739
:1039300053BA02325A70FAE7704700BF7001002094
:10394000064A537843B1012B03D100235370FEF78D
:1039500043BA023B5370FAE7704700BF7001002082
:10396000064B9A783E2A07D803D13F229A70FEF779
:1039700033BA02329A70FAE7704700BF7001002034
:10398000064A937843B1012B03D100239370FEF7CD
:1039900023BA023B9370FAE7704700BF7001002022
:1039A00040F27013C2F200031A7802705A78427023
:1039B0009B788370704700BF10B440F27013047896
:1039C00041788278C2F200033F2C34BF20463F206A
:1039D0003F2928BF3F213F2A28BF3F221870597036
:1039E0009A7010BCFEF7F8B940F23C03C2F2000333
:1039F0001A7802705A7842709B788370704700BFC3
:103A000010B440F23C03047841788278C2F200039B
:103A10003F2C34BF20463F203F2928BF3F213F2A6B
:103A200028BF3F22187059709A7010BCFEF76CB80E
:103A300040F2A413C2F20003186870470F2803D89D
:103A4000034B1860FEF7C8B9014B0F221A60F9E763
:103A5000A4010020034B1A6802B97047013A1A60AA
:103A6000FEF7BAB9A4010020044B1A680E2A00D947
:103A7000704701321A60FEF7AFB900BFA401002001
:103A800040F26C13C2F20003186870470F2803D885
:103A9000034B1860FEF738B8014B0F221A60F9E7A4
:103AA0006C01002070B5012682B040F2851516F039
:103AB000010F0CBF0021392116F0020F0CBF0022AC
:103AC000392216F0040F0CBF002339238DF804109F
:103AD0008DF805208DF806300024204601A9013418
:103AE00007F07CF8AC42F8D1204606F0D7FF01364B
:103AF0000320FDF7B1FE082ED9D10020FEF7FAF819
:103B0000002001460246FFF715FB02B070BD00BF62
:103B10002A4B2DE9F04103F59071012413F8012B94
:103B200012F0020214BF03F8014C03F8012C8B427F
:103B3000F4D1017800293FD08046074608260020AE
:103B4000C6F10802FEF732F898F80110013759B3B0
:103B5000112E16D83D46344601E0112C11D82046CE
:103B60000022FEF723F815F8011F09340029F4D1CB
:103B700005E02046202100220934FEF717F8112C19
:103B8000F7D90420FEF774FA3220FDF757FE013E04
:103B90000CD017F8011C0020C6F10802FEF706F849
:103BA00098F801100029D3D13446E8E718F8011F2E
:103BB0000029C3D1BDE8F081BDE8F081606100203B
:103BC000F8B5324B1B681BB1A0F114053B2D00D991
:103BD000F8BD0020FEF78EF82D4B2E4C93F8883060
:103BE000C3EB031305EB83052B4B04F5907103EB3B
:103BF000C5050120234613F8012B12F0020214BF61
:103C000003F8010C03F8012C8B42F4D1234E707998
:103C1000F278337958B102EBC202181804EB420271
:103C2000D15C41F00201D15401338342F8D1307AA2
:103C3000B279F37958B102EBC202181804EB4202D0
:103C4000D15C41F00201D15401338342F8D1002705
:103C5000EB195B78ABB103EB4303F118F25C8878A6
:103C60004B7858B102EBC202181804EB4202D15C47
:103C700041F00201D15401338342F8D10137072FBB
:103C8000E6D1074B01221A60F8BD00BF7401002085
:103C9000ACDE000860610020F8C40008C8DD000840
:103CA000580400202DE9F04FB94B1B68044693B02F
:103CB000184613B913B0BDE8F08F3F268DF8346075
:103CC0003C2603258DF82360162600230CA92A46DE
:103CD000A4208DF824600F268DF835308DF836300D
:103CE0008DF825308DF826308DF82B308DF8275043
:103CF0008DF8296000F0AEFB01220DF12101A72013
:103D000000F0A8FB01220DF12501A82000F0A2FB84
:103D100001220AA9BD2000F09DFBBE2001220DF169
:103D20002A0100F097FBB4F5843F80F0A3809DF852
:103D300021809DF822C09DF825E09DF82610B8F15D
:103D4000110F84BF4FF000088DF82180BCF1030FE4
:103D500084BF4FF0000C8DF822C0BEF10A0F84BF63
:103D60004FF0000E8DF825E0012902D900218DF8D1
:103D700026109DF828700F2F02D90F278DF8287074
:103D80009DF829600F2E71D89DF82A00012802D0D5
:103D900000208DF82A009DF82320642A009203D980
:103DA00064258DF8235000959DF82430632B02D9AB
:103DB00016238DF82430774C07932568764B0195B0
:103DC0009DF827509DF834B002959DF830509DF82D
:103DD00035A003959DF831509DF8369004959DF8D7
:103DE000325083F800B005959DF82B5083F801A060
:103DF000069540F26835C2F2000583F80290C5F8D6
:103E00000080DFF8C081029DC8F800C0DFF8B8C1AB
:103E1000624BCCF80050DFF8B4C1614ACCF800E046
:103E2000DFF8ACE11F60CEF800105E4B0399049DF3
:103E300011701E6005995C4B557091701860009A66
:103E40005A4B079D1A605A4B06991D60594B1960D1
:103E500000232360FDF758FEFDF7BEFF019A2260A4
:103E6000FFF728FBFDF77CFE012023E70F268DF8E6
:103E7000296089E7A92001220DF1260100F0EAFA64
:103E800040F6FF03C0F201039C427FF650AF0122CF
:103E90000DF12701BC2000F0DDFA0DA92A46D7203C
:103EA00000F0D8FA01220DF12901DA2000F0D2FA4F
:103EB000DB2001220DF1220100F0CCFAB4F5003F25
:103EC000FFF435AF01220DF12301DC2000F0C2FA2E
:103ED000DD20012209A900F0BDFAFF23C0F2020390
:103EE0009C427FF624AF0DF12B010122E02000F06F
:103EF000B1FA0FA90B22E52000F0ACFA0EAE0BA927
:103F0000022240F2251000F0A5FA40F235103146A9
:103F1000042200F09FFA0DF14605274B0DF13B00FE
:103F200005E042F002021A611433A84212D010F8E0
:103F3000012FFF2AF8D002F01001C9B202F00F02DF
:103F40009A601A690029ECD122F002021A61143336
:103F5000A842ECD19DF82C301848FF2B1EBF184A00
:103F600003F00F0353609DF82D30FF2B1EBF144A42
:103F700003F00F0353610023F25CFF2A1EBF00EB26
:103F8000031102F00F024A600133042BF4D1CEE694
:103F9000A0040020740100203C000020A4010020A7
:103FA000700100206C0100203C04002078010020FA
:103FB000A801002040040020500000202C01002017
:103FC0007C0100202C04002044000020A0010020DF
:103FD000C80300202DE9F04F854B1B68A3B0002BD0
:103FE00000F08B80834B844A93F8008093F801C0E3
:103FF00093F802E0814B92F800B01F68804B92F872
:1040000001A01E687F4B92F802901D687E4B8DF8D0
:1040100019501C687D4B8DF81A401B688DF820B034
:1040200000937B4B009C1B688DF81B400193794BE0
:10403000019C1B688DF821A00293774B8DF822908C
:104040001B688DF824800393744B8DF825C0186885
:10405000734B8DF826E01968724B8DF815701A684D
:104060008DF816608DF81C40029C6F4B8DF81D403A
:10407000039C8DF817008DF81E408DF81810002055
:104080008DF81F2012ACFF250A2888BF255409D8B7
:104090009A68196902F00F028907225444BF42F05E
:1040A00010022254013014334028EDD15F48002320
:1040B0000AAEFF22012B97BF00EB0311F2544968AF
:1040C00001F00F0198BFF1540133102BF2D1584980
:1040D00000230EADFF2001EB0312032B97BF5268A4
:1040E000E85402F00F02EA540133102BF3D1A4205C
:1040F00008A9032200F0C8F918B9002023B0BDE8D0
:10410000F08FA7200DF11501012200F0BDF9002864
:10411000F3D0BC200DF11901012200F0B5F90028FF
:10412000EBD0A8200DF11A01012200F0ADF9002812
:10413000E3D0A9200DF11B01012200F0A5F9002810
:10414000DBD0BD2007A9012200F09EF90028D4D0C1
:10415000BE200DF11E01012200F096F90028CCD0FE
:10416000D72009A9032200F08FF90028C5D0DA2052
:104170000DF11D01012200F087F90028BDD0DB20E0
:104180000DF11601012200F07FF90028B5D0DC20E6
:104190000DF11701012200F077F90028ADD0DD20E4
:1041A00006A9012200F070F90028A6D0E0200DF148
:1041B0001F01012200F068F900289ED0E520214669
:1041C000402200F061F9002897D040F225103146D6
:1041D000102200F059F900288FD0102240F235103B
:1041E000294600F051F9003018BF012086E700BFD2
:1041F000A00400203C000020700100206803002083
:104200002C04002044000020A0010020C80300204E
:10421000A40100206C0100203C0400207801002053
:10422000A801002040040020500000207C01002054
:104230002C01002006F0FEBC2DE9F843814688469B
:10424000174605F07BFC10B90020BDE8F883552027
:1042500005F00CFD2E48082105F030FD442005F046
:1042600005FD002443F2144505F0CAFC0134AC42BC
:1042700098BF002814BF00260126F5D043F214434E
:104280009C4227D805F05AFC0028DDD0552005F0C7
:10429000EDFC204C1E48082105F010FDBE2005F065
:1042A000E5FC0921204605F0D3FC05F047FC1A4B3C
:1042B0001B68222B13D0282B11D00923C9F80030FA
:1042C00094F90130DB0FC8F80030237801203B60FF
:1042D000BDE8F88305F032FC3046BDE8F883237969
:1042E00062782578C3F34113093302F00704C3F160
:1042F0000C00191F45FA00F004FA01F10143D2093C
:10430000C9F800300120C8F800203960BDE8F88302
:10431000940400208004002090040020F8B5A0F14F
:104320000905032D044602D900263046F8BD05F0E4
:10433000F5FC05F003FC0028F6D02E4F384605F0BA
:10434000CBFC3B782C4A13602C4A0121222B0646D9
:10435000116001D0282BE8D105F0F0FB0028E4D053
:10436000552005F083FC264F2248082105F0A6FCC5
:10437000BE2005F07BFC0921384605F069FC3B793D
:10438000C3F341130933A342CFD005F0D7FB002874
:10439000CBD0552005F06AFC0821164805F08EFCAC
:1043A0004E2005F063FC7F2005F060FC802005F0C6
:1043B0005DFC680100F0E00005F058FC05F0BEFB74
:1043C00005F0BCFB0028B0D0552005F04FFC094893
:1043D000082105F073FC482005F048FC002405F096
:1043E0000FFC0134F92C98BF0028F8D005F0A6FB8B
:1043F0009BE700BF94040020900400208C04002060
:10440000800400202DE9F04184B003F03FF8DFF88C
:10441000408000240127650045F0A0050126009793
:104420002846002132460DF10F03A419C8F80050A8
:1044300003F080F830B1082CEDD1044B186804B0BB
:10444000BDE8F081014B30461E60F8E7A004002073
:104450009C04002010B50A4B1C6882B00B4614B9AE
:10446000204602B010BD0092064A1268014610466E
:10447000012203F05FF8D0F1010038BF0020F0E71F
:10448000A00400209C0400202DE9F047144B1B6879
:1044900082B0174603B3EAB1DFF84CA0114C0646D0
:1044A000C0EB01094FF001080025DAF80000CDF853
:1044B00000803146012209EB060303F0B9F858B930
:1044C00010202368002BFCD001382560F9D101367B
:1044D000013FEAD1012000E0002002B0BDE8F087F2
:1044E000A0040020806200209C04002070B53E4B98
:1044F0001A68824288B0064674D002A81E60FCF793
:10450000A9F904A8FCF7ECFC01200146FCF750FBDC
:1045100001200146FCF74CFB20200121FCF764FB45
:104520000020C4F202000B210822FCF7A9F90020A8
:104530000822C4F202000C21FCF7A2F90223002099
:104540008DF80C30032304460125C4F2020002A9B1
:104550008DF80D304FF4006302938DF80E408DF806
:104560000F50FCF71BF920464FF48053C4F20200B1
:1045700002A90293FCF712F94FF4A050C4F2010013
:104580002946FCF7C7FC4FF4A0500C23C4F20100ED
:1045900004A9ADF81A300496ADF81440ADF81640F1
:1045A000ADF81840ADF81C40FCF72EFC4FF4A050BD
:1045B000C4F201002946FCF79FFC4FF4A050C4F25E
:1045C000010040F225512A46FCF7BAFC472301A816
:1045D0008DF804308DF805408DF806408DF80750B1
:1045E000FBF736FE08B070BDBC06002030B40F4AA1
:1045F00013687F2BFCD80E490E4D0B685C1C7F2C7A
:1046000045F8230098BF0C6001D900230B6072B6F7
:1046100013680133136062B64FF4A050C4F2010076
:1046200040F22771012230BCFCF78ABCB80600209A
:10463000B4060020AC04002010B50446007828B170
:10464000FFF7D4FF14F8010F0028F9D110BD00BF07
:1046500040F2A843C2F200031868003018BF0120DE
:10466000704700BF30B40D4B1A6882B10C490D4D34
:104670000A68541C802C55F8225018BF0C6009D0D1
:1046800072B61A68013A1A6062B6012205601046D5
:1046900030BC704700220A60F2E700BFA804002087
:1046A000A4040020C0060020024A1368002BFCD19D
:1046B000704700BFB80600204FF4A05038B5C4F2D0
:1046C000010040F22551FCF757FC00282BD14FF494
:1046D000A050C4F2010040F22771FCF74DFC00B974
:1046E00038BD4FF4A050C4F2010040F22771FCF72E
:1046F00069FC234B1A68002A38D0224A224C1168E0
:10470000481C802808BF002054F8211010601A6847
:104710004FF4A050013AC4F2010089B21A60BDE81A
:104720003840FCF705BC4FF4A050C4F2010040F241
:104730002551FCF747FC4FF4A050C4F20100FCF7F0
:10474000FBFB124B1A687F2AC1D81149114D0A6828
:10475000541CC0B27F2C45F8220098BF0C6001D9D0
:1047600000220A601A6801321A60B0E74FF4A050C4
:10477000C4F2010040F22771BDE83840FCF7E0BB0D
:10478000B8060020AC060020AC040020A8040020DD
:10479000B0060020C00600202DE9F04383B0684633
:1047A000FCF758F800260120C4F202060146012455
:1047B000FCF7FEF900254FF0800930466946CDF838
:1047C00000908DF805508DF804408DF806508DF856
:1047D0000750FBF7E3FF20462146FCF7E9F94FF0CD
:1047E000400830466946CDF800808DF805508DF8B8
:1047F00004408DF806508DF80750FBF7CFFF204698
:104800002146FCF7D5F910273046694600978DF808
:1048100005508DF804408DF806508DF80750FBF7D1
:10482000BDFF304649462246FCF724F83046414653
:104830002246FCF71FF8304639462246FCF71AF8A4
:1048400003B0BDE8F08300BFF8B5094D04460F463C
:10485000002601E02B6833B92046FFF703FF00284C
:10486000F8D00120F8BD0136BE422860F4D3F8BD6F
:10487000846200202DE9F04F85B0054603F02AFD43
:10488000FFF712FFFFF7E4FE002843D00024624F39
:10489000DFF888A10126A346294603A8FFF7D4FF25
:1048A000DFF874914FF001080346002835D0039BD0
:1048B0003E600A2B07D00D2BEED0FF2CECD80AF867
:1048C00004300134E8E70AF804B0002C32D103F0D8
:1048D00001FDE1E7514852491A4606F00EFE002854
:1048E0004CD04E484F49032206F007FE00284FD017
:1048F0004A484D49052206F000FE002855D14B4894
:104900004B49022206F0F9FD002849D10123C9F8DC
:104910000830062005B0BDE8F08F4648019303F04B
:10492000ABFC454803F0A8FC444803F0A5FC019B00
:104930001846EFE73F48019303F09EFC374803F029
:104940009BFC3E4803F098FC34483D49022206F0A7
:10495000D4FD38B131483B49052206F0CEFD18B9E7
:104960000220D7E74046D5E72C483749022206F017
:10497000C4FD019B0028ADD10320CBE709F13C0029
:1049800032490F2206F0D2FDC9F804800420C1E7A5
:1049900009F11C002E491F2206F0C8FD0520B9E7C9
:1049A0000023C9F808300620B4E71C48294905222D
:1049B00006F0A3FD98B119482749092206F09DFD8C
:1049C00010B316482549042206F097FDA8B11348F4
:1049D0002349092206F091FD40B1FF209AE72148C2
:1049E00012490F2206F0A2FD072093E71E481F4937
:1049F000FF2206F09BFD0A208CE71D481D491F225F
:104A000006F094FD092085E71B4818490F2206F09F
:104A10008DFD08207EE700BFC00800203C0A002072
:104A20005CDF000868DF00086CDF0008410A002036
:104A300074DF00083CDF000840DF000848DF0008A2
:104A40004CDF000850DF000858DF0008460A00204D
:104A50003F0A002078DF000880DF00088CDF0008B4
:104A600094DF00082C0A00200C090020450A0020D1
:104A70000C0A0020400A0020CC080020F0B583B0CA
:104A8000074606F032FD06461A4803F0F5FBBEB1B4
:104A90003C46F61904E0184603F0C8FBB4420FD0B8
:104AA00014F8013B1449A3F120055E2D68461A460F
:104AB000F1D906F0D7FC684603F0DEFBB442EFD133
:104AC0000E4803F0D9FB03F005FC3846FFF7B4FDB0
:104AD0000B48FFF7B1FDFFF7E7FD02E0022807D022
:104AE00020B10A20FFF7C6FE0128F7D103B0F0BDC0
:104AF0000020FBE7A0DF0008B4DF0008A8DF000803
:104B00007CE1000838B539B10446451814F8010BAA
:104B1000FFF76CFDAC42F9D1BDE83840FFF7C4BDEA
:104B200040F6C000C2F20000704700BF10B5002080
:104B3000C4F202008021002282B0FBF79BFE0C4AE7
:104B40000521144600201368002BFCD00139206099
:104B5000F9D10020C4F2020080210122FBF78AFE75
:104B600001A83221FFF770FE0028F9D102B010BD74
:104B70008462002008B502460B460748074906F044
:104B800071FC0548FFF77AFF20B1054B002283F83E
:104B90003C205A6008BD00BF400B0020BCDF00086D
:104BA000C008002008B502460B460748074906F032
:104BB00059FC0548FFF762FF20B1054B002283F83E
:104BC0003C205A6008BD00BF400B0020CCDF00082D
:104BD000C008002008B5024608B1037823B9074889
:104BE000BDE80840FFF74ABF0549064806F03AFC11
:104BF0000448BDE80840FFF741BF00BFF8E50008E2
:104C0000DCDF0008400B002030B54FF4E13083B00A
:104C100003F0FAFBFFF7C0FD4FF4E130FFF766FC4D
:104C20000020C4F2020010210022FBF723FE1E4CDC
:104C300000200022C4F202008021FBF71BFE0525A4
:104C40002246002321680029FCD0013D1360F9D1E0
:104C5000002080210122C4F20200FBF70BFE124962
:104C600032222368002BFCD0013A0D60F9D10020DC
:104C7000C4F2020010210122FBF7FCFD03E001A8B1
:104C800003F006FB60B901A8FFF7ECFC0028F6D0A2
:104C9000019803F0CBFA01A803F0FAFA0028F2D049
:104CA0000198FFF7A3FCEEE78462002008B50B4BE8
:104CB0001A6802B108BD01224FF4E1301A6003F016
:104CC000A3FB074803F0D8FAFFF766FD4FF4E13085
:104CD000FFF70CFCBDE80840FFF728BF900B002051
:104CE000E8DF000810B403781649FBB10022086021
:104CF0001446013005E001300E2A14DC10F8013CA6
:104D00008BB13D2B02BF01EBC20300F8014C586090
:104D1000F1D0262BEFD1013200F8014C41F83200DE
:104D200001300E2AEADD531C0F2B08DC002201EBB8
:104D3000C30011460133815008320F2BFADD10BC3D
:104D4000704700BFFC0B0020F8B50A4D0646002452
:104D500055F83430E70031461846013423B106F0E7
:104D6000B2FB18B1102CF3D10348F8BD014BDF1989
:104D70007868F8BDFC0B002004E1000808B5FFF7D7
:104D8000E3FF4EF2E001C0F6000106F09CFBD0F11B
:104D9000010038BF002008BD00B50B4685B04EF2BB
:104DA000E8010246C0F60001684606F05BFB684673
:104DB000FFF7CAFF05B000BD10B5044606F095FB2D
:104DC000014600B910BD2046BDE81040FFF79ABE6D
:104DD00010B504464EF2F000C0F60000FFF7ECFFFD
:104DE0004EF20010C0F60000FFF7E6FF4EF208108A
:104DF000C0F60000FFF7E0FF4EF21410C0F600000E
:104E0000FFF7DAFF4EF22010C0F60000FFF7D4FFE4
:104E10002046FFF7D1FF4EF22810C0F60000FFF742
:104E2000CBFF4EF23410C0F60000FFF7C5FF4EF284
:104E30004010C0F60000FFF7BFFF4EF24C10C0F666
:104E40000000FFF7B9FF2046FFF7B6FF4EF25410FF
:104E5000C0F60000BDE81040FFF7AEBF38B504460D
:104E60004EF25C10C0F600000D46FFF7A5FF20468D
:104E7000FFF7A2FF4EF26810C0F60000FFF79CFF9C
:104E80002846FFF799FF4EF26C10C0F60000BDE80F
:104E90003840FFF791BF00BF4EF204104EF2801170
:104EA00008B5C0F60000C0F60001FFF7D7FF4EF2CC
:104EB00088104EF29011C0F60000C0F60001FFF716
:104EC000CDFF4EF69C104EF29811C0F60000C0F6D1
:104ED0000001FFF7C3FF4EF2A4104EF2A811C0F676
:104EE0000000C0F60001FFF7B9FF4EF618304EF291
:104EF000AC11C0F60000C0F60001FFF7AFFF4EF2A4
:104F0000B4104EF2C011C0F60000C0F60001FFF769
:104F1000A5FF4EF2CC104EF2D811C0F60000C0F63C
:104F20000001FFF79BFF4EF2E4104EF2EC11C0F6C9
:104F30000000C0F60001FFF791FF4EF2F410C0F63A
:104F40000000BDE80840FFF737BF00BF054A1368FF
:104F500001331360DB0702D40348FFF72DBF03487A
:104F6000FFF72ABFAC0C002010E20008F8E10008AF
:104F700010B504464EF21820C0F60000FFF71CFFE3
:104F80002046FFF719FF4EF22020C0F60000BDE8D2
:104F90001040FFF711BF00BF70B584B00C46054646
:104FA0001B49164668461A4606F05CFA02A81849DC
:104FB000089A06F057FA3CB123782BB12046FFF748
:104FC000FBFE1448FFF7F8FE1348FFF7F5FE2846EE
:104FD000FFF7F2FE1148FFF7EFFE2846FFF7ECFE61
:104FE0000F48FFF7E9FE3046FFF7E6FE0D48FFF7F2
:104FF000E3FE6846FFF7E0FE0B48FFF7DDFE02A880
:10500000FFF7DAFE0948FFF7D7FE04B070BD00BF16
:1050100034ED0008C8E8000828E2000840E2000873
:105020004CE2000858E2000868E2000868E1000865
:1050300010B504464EF27420C0F60000FFF7BCFE27
:105040002046FFF7B9FE4EF2A820C0F60000FFF799
:10505000B3FE4EF2B820C0F60000BDE81040FFF7E6
:10506000ABBE00BF70B505460F480E46FFF7A4FE65
:105070000E48FFF7A1FE002E0EDD043D00240C4873
:10508000FFF79AFE55F8040FFFF796FE0134094822
:10509000FFF792FEB442F2D10748FFF78DFE074BAF
:1050A00000221A6070BD00BFC0E2000810E20008D4
:1050B000DCE20008F4E20008D4E20008AC0C0020B6
:1050C0004EF20430C0F60000FFF776BE38B5044655
:1050D0004EF21430C0F600000D46FFF76DFE20467C
:1050E000FFF76AFE4EF26810C0F60000FFF764FE9C
:1050F0002846FFF761FE4EF24030C0F60000BDE8E2
:105100003840FFF759BE00BF08B54EF25030C0F628
:105110000000FFF751FE4EF25C30C0F60000BDE823
:105120000840FFF749BE00BFF0B5044683B01F48F2
:105130001E460D461746FFF73FFE2046FFF73CFE92
:105140001B48FFF739FE2046FFF736FE1948FFF7E8
:1051500033FE002E24DD043D00240BE01648FFF74B
:105160002BFE55F8040FFFF727FE1448FFF724FE27
:10517000B44215D02246124901A806F073F911482D
:10518000FFF71AFE01A8FFF717FE0F48FFF714FEFE
:10519000BC4204F10104E1D10C48FFF70DFEDDE74C
:1051A0000B48FFF709FE03B0F0BD00BF68E300083D
:1051B00040E2000878E3000874E40008A8E300086F
:1051C00034ED00088CE3000854E200089CE300087A
:1051D00080E3000870B50E4605460E481446FFF7FA
:1051E000EBFD3046FFF7E8FD0B48FFF7E5FD2846ED
:1051F000FFF7E2FD0948FFF7DFFD14B10848FFF7AC
:10520000DBFD0848FFF7D8FD0748BDE87040FFF711
:10521000D3BD00BF18E20008B4E30008D8E30008DB
:10522000ECE3000874E4000820E200082DE9F041F6
:10523000069F079D04461646984611B10B78002B31
:1052400049D12848FFF7B8FD2046FFF7B5FD2648AD
:10525000FFF7B2FD2046FFF7AFFD2448FFF7ACFD96
:105260003046FFF7A9FD2248FFF7A6FD4046FFF7AD
:10527000A3FD2048FFF7A0FD3846FFF79DFD55B17F
:105280002B7843B11C48FFF797FD2846FFF794FDA4
:105290001A48FFF791FD1A48FFF78EFD2046FFF7E9
:1052A0008BFD1848FFF788FD2046FFF785FD16485F
:1052B000FFF782FD1548FFF77FFD2046FFF77CFDD5
:1052C0001348FFF779FD3046FFF776FD1148BDE83A
:1052D000F041FFF771BD0846FFF76EFD0E48FFF77E
:1052E0006BFDAEE7F4E3000840E200084CE2000882
:1052F00010E4000818E4000820E4000830E4000886
:1053000034E4000840E4000850E400085CE40008CD
:105310006CE4000878E40008C8E800084EF2844015
:10532000C0F600000321FFF7EDBB00BF10B5044637
:105330004EF21820C0F60000FFF73EFD4EF2884105
:105340002046C0F60001FFF7C1FE4EF2B820C0F6BD
:105350000000BDE81040FFF72FBD00BF70B5064646
:105360004EF2182082B0C0F600000D461446FFF73A
:1053700023FD4EF204114EF29043C0F60001C0F638
:1053800000033046009301912A462346FFF74EFF63
:105390004EF2B820C0F6000002B0BDE87040FFF742
:1053A0000BBD00BF38B505460C46FFF7CFFD2846BC
:1053B000FFF7DEFD2046FFF7DBFD4EF20410C0F6DE
:1053C0000000FFF7D5FD4EF2D420C0F60000BDE886
:1053D0003840FFF7F1BC00BF10B504464EF29440D0
:1053E000C0F60000FFF7E8FC2046FFF7E5FC4EF2B0
:1053F0007830C0F60000BDE81040FFF7DDBC00BF0C
:1054000010B50446FFF7A2FD2046BDE81040FFF7A7
:10541000E3BF00BF4EF2B440C0F60000FFF7CCBCC3
:1054200008B5FFF7F7FF4EF2D420C0F60000BDE844
:105430000840FFF7C1BC00BFF0B583B00E4614466C
:105440001F46089DFFF7DCFF3046FFF791FD4EF247
:105450001820C0F60000FFF7AFFC4EF20411C0F6B2
:1054600000013A462B4620460095FFF795FD4EF287
:105470002020C0F60000FFF79FFC2046FFF7D8FD74
:1054800003B0BDE8F040FFF7CBBF00BFF8B5069D05
:105490000E4614461F46FFF7B3FF3046FFF768FD80
:1054A000204639462A46FFF795FE2046FFF7C0FD05
:1054B000BDE8F840FFF7B4BF2DE9F0410F461446B0
:1054C0009846069E079DFFF79BFF3846FFF750FD65
:1054D0004EF21820C0F60000FFF76EFC414632463F
:1054E0002B462046FFF720FE4EF22020C0F600009B
:1054F000FFF762FC2046FFF79BFDBDE8F041FFF798
:105500008FBF00BF2DE9F04F83B08B46924699467E
:10551000DDF830800D9F124EFFF772FF1148FFF744
:1055200027FD1148FFF748FC00243D595BF80400B3
:105530005AF8041059F8042058F804308DE8600037
:10554000FFF774FE04340948FFF736FC0C2CECD14D
:105550000748FFF76DFD03B0BDE8F04FFFF760BFF0
:10556000D0E40008C0E40008C8E40008D4E400085F
:1055700080EB00082DE9F04F05460E46C7B0A8485D
:105580002946924602F030FF33781BB3741C4FF06B
:105590002008002706E02B2B08BF04F8018C14F824
:1055A000013BBBB1252BF6D120460221FBF7D2FDF2
:1055B000A27804F8010C002A00F04185234603F884
:1055C000012B9A781946002AF9D10F7014F8013B83
:1055D000002BE7D13146934802F006FF3046FFF733
:1055E00081FB2846904905F06EFF002842D02846EE
:1055F0008E4905F068FF0446002800F0CD83284658
:105600008B4905F060FF002800F071842846894925
:1056100005F059FF0446002800F095812846864988
:1056200005F051FF002800F06B852846834905F0FE
:105630004AFF002800F0FA872846814905F043FF19
:10564000002800F04F8228467E4905F03CFF0028E4
:1056500000F010877C48FFF7AFFB7C48FFF7ACFBFE
:105660007B48FFF7A9FB0026FFF758FE304647B0FE
:10567000BDE8F08F774C94E803001AAD04F10806FA
:1056800085E803000FCE3EAF07953D460FC596E86F
:105690000300059704F1200785E803000FCF25AD2F
:1056A00004F1340E2E460FC6BEE80F003F68089581
:1056B00004F1480C2AAD069537600FC5BCE80F0011
:1056C0002FAF48343E460FC60FCC0DF1D0084446EC
:1056D0000FC4DCF80030DEF800203360236015A929
:1056E00014A81CAC0DF1600913AE0DF1580B2A6023
:1056F0003C910994CDF8E4903A963B90CDF8F4B003
:1057000002F0C4FF0A9002F0C7FF5349C0F30742FA
:10571000C0F30723099805F0A5FE02F0C3FF426914
:10572000002A044632DB0369002B2FDBC168002905
:105730002CDB8068002829DB6568002D26DBB2F5AC
:10574000966F23DC0C2B21DC1F291FDC17281DDCA6
:105750003B2D1BDC02F26C724846404905F082FE8C
:1057600022693F490132304605F07CFEE2683C493F
:1057700014A805F077FEA268394915A805F072FE55
:1057800058463749626805F06DFE0AE000238DF83F
:1057900060308DF84C308DF850308DF854308DF8E5
:1057A00058303048FFF7D0FA0546002801F08E80C7
:1057B0002D4905F088FE002841F057802B4C4926E2
:1057C0002B48DFF8C4A0FFF703FBFFF765FB079842
:1057D0000221FFF747FC27480A99FFF7E3FDDAF8B3
:1057E0000030254A25492648002B18BF1146FFF7EF
:1057F000D9FDDAF80030002B41F03180FFF760FC72
:1058000005980621FFF72EFC1E48FFF7F9FD4FF023
:10581000000A09950594089DDDF818B039E000BF2D
:1058200068E600087CE6000894E60008BCE700088B
:1058300030E9000814EA00089CEA0008D4EB0008EC
:1058400090EC000838ED000884ED000800E1000845
:105850009CED0008FCDF000898E60008A4E60008BC
:10586000A8E60008B0E60008B8E60008ECE4000886
:1058700008E7000814E70008A0F500083CE5000868
:105880001CE7000804E10008A004002039AB5AF826
:1058900003907548FFF790FA58F80A4055F80A0047
:1058A0005BF80A1057F80A3000944A46FFF774FB79
:1058B0000AF1040A6D48FFF77FFABAF1140FE5D137
:1058C0006B48059C099DFFF7B3FBFFF7A9FDFFF7A8
:1058D000F7FB07980221FFF7C5FB6648664A674950
:1058E0001E2703460097FFF7A7FDFFF7E9FB614876
:1058F000FFF772FD62486349FFF7E8FB62486349BE
:10590000FFF7E4FB62486349FFF7E0FB6248634945
:10591000FFF7DCFBFFF77EFD44B16148FFF74CFA6F
:105920002046FFF749FA5F48FFF746FA28465A49EA
:1059300005F0C9FD0446002800F0E984FFF7E4FB08
:10594000FFF7ECFC92E6584B93E803003EAD85E888
:1059500003000595FDF76CFD80465448FFF7F4F908
:105960000546002801F00282514905F0ACFD0646CB
:10597000002801F0498128464E4905F0A4FD06465D
:10598000002801F0238028464B4905F09CFD054680
:10599000002841F0E7814948FFF7F0F910F10008CD
:1059A00018BF4FF00108CAF800804C2600238DF87C
:1059B000BC300A24FBF768FB0DF13A00FBF772FBE1
:1059C000002841F00B810A20FBF738FF013CF3D19E
:1059D00046AF3F2327F85C3D02F074FA384982B2A3
:1059E00034A805F03FFD02F073FA354982B239A8B8
:1059F00005F038FD3348FFF7EBF9FFF74DFA05984E
:105A00000221FFF72FFB30483946FFF7CBFC2F4828
:105A100034A9FFF7C7FC2E4839A9FFF7C3FC274A72
:105A20002C4B29492C48CDF80080FFF72FFDFFF7BC
:105A300047FB2948FFF7D0FC1D482849FFF746FBE4
:105A40001C482749FFF742FBFFF7E4FC002D3FF419
:105A500075AF1348FFF7B0F92846FFF7ADF91148C5
:105A6000FFF7AAF96AE700BF18E2000820E2000881
:105A7000D8E6000804E1000800E7000834E7000861
:105A8000C0E600083CE70008C8E6000848E7000850
:105A9000B8E6000854E700086CE7000878E700085B
:105AA00084E7000824E90008FCDF0008B0E60008ED
:105AB0001CEA000824EA00082CEA000830EA000882
:105AC00038EA00083CEA0008A8E100084CEA0008AF
:105AD00050EA000854EA0008A4E100086CEA000853
:105AE00084EA0008914E924D96E8070006F15003B3
:105AF00020AC84E807000FCB3EAF06F10C0E87E820
:105B00000F009EE8070025AB08930597089F06F154
:105B1000180387E8070093E807002AAB0693069F5F
:105B200006F1240387E8070093E807000DF1D00889
:105B3000303688E8070096E807002B687D4F0DF1A6
:105B4000E40989E807004BB97B4E3B6A39683A693A
:105B5000386B86E80E000123F0602B60FDF7FCFB3C
:105B60000790FDF713FC0A90FDF71EFC0B90FDF764
:105B7000CFFB00F002000C90FDF782FF0990FDF7CB
:105B800057FC0D900FA8FDF72FFF6C48FFF7DCF8CE
:105B90000546002800F01F87694905F094FC8346FC
:105BA000002801F08D802846664905F08CFC83466C
:105BB000002801F005812846634905F084FC8346EE
:105BC000002801F0C3812846604905F07CFC0646A8
:105BD000002801F0578328465D4905F074FC06460D
:105BE000002801F0F88228465A49072205F085FC72
:105BF0000646002801F0E68228465749042205F0AF
:105C00007CFC0646002801F05A832846534905F0DB
:105C10005AFC0026B34610B9DFF878B153267A6BE8
:105C20004F4915A805F01EFC4D490A9A16A805F023
:105C300019FC4B490B9A18A805F014FC11AD484902
:105C4000099A10A805F00EFC0DF1480A44499DF888
:105C50003C20284605F006FC13AF41499DF83D2045
:105C6000504605F0FFFB9DF83E203D49384605F0C3
:105C7000F9FB3C482F950325CDF8C0A03197FFF7DD
:105C8000A7F8FFF709F920462946FFF7EBF9364850
:105C90003649374A009516ABFFF7CEFB00953248E0
:105CA0003449354A18ABFFF7C7FB0C9C5CB90D9D16
:105CB000002D01F025818DE800032B480899069AF4
:105CC0002FABFFF71FFC079F2C4A1B4B26482C4984
:105CD000009704240194FFF7EFFBFFF7F1F9214649
:105CE0000598284DFFF7BEF900242B68DA0700F16C
:105CF0009E8601341035042CF7D1FFF7E1F91A48DC
:105D0000FFF76AFB15482049FFF7E0F9FFF782FB30
:105D1000BBF1000F3FF412AE1C48FFF74DF8584698
:105D2000FFF74AF81A48FFF747F807E660E000086F
:105D3000940B00202C010020980B0020B0E60008F6
:105D4000C4EA0008D4EA00089CEC0008ACEC0008A7
:105D5000BCEC0008CCEC0008DCEC000820EB0008F0
:105D600034ED0008E4EC0008CCE10008F8EC000891
:105D7000B0EC000800ED0008C0EC0008A0EC000842
:105D800018ED000838010020C8EB000884E700087F
:105D900024E9000848E60008AB4B93E803000DF146
:105DA000E409083389E8030093E807003EAD85E87D
:105DB00007000595FEF7B4FE0546A448AF68FEF758
:105DC000C3FF05F10C088246002800F0F487A049C3
:105DD00005F079FB0646002800F0548650469D49A0
:105DE00005F071FB0646002800F0018750469A49ED
:105DF00005F069FB0646002800F0188750469749D1
:105E000005F061FB002800F065852646B24604F0E7
:105E10009BFD9349024634A805F024FB9148FEF708
:105E2000D7FFFFF739F805980321FFF71BF98E48D4
:105E300005F13C01FFF7B6FA41468C48FFF7B2FA8C
:105E40008B48FFF7DDFA8B48FFF792F88A48FEF798
:105E5000B3FF4FF00F08894849463A460223FFF73F
:105E600063F987498748CDF8008005F11C0220239B
:105E7000FFF792F88448FEF79FFF14238349844A72
:105E8000844800934023FFF787F88348FEF794FF88
:105E90008248FFF7CDF8FFF7C3FA04F077FD804999
:105EA000804ACDF8008003467148FFF7C5FA032306
:105EB0007D497E4A6E48009334ABFFF7BDFAFFF789
:105EC000FFF86B48FFF788FA64487949FFF7FEF856
:105ED000FFF7A0FA002C00F00B827648FEF76CFF6B
:105EE0002046FEF769FF7448FEF766FF26E5734B10
:105EF00093E803000DF1D00888E803005348FEF74B
:105F000023FF0446002800F0F8846D4905F0DBFA11
:105F10000646002800F0588620466A4905F0D3FA64
:105F20000646002800F0AF862046674905F0CBFA08
:105F3000002840F0E284654D5726654B1B68002B16
:105F400000F06C8504F0A6FA0DF1E409044662083D
:105F50004846434905F086FAE70700F1BC86484603
:105F600005F0C3FA5B4B09EB000201469C881868F8
:105F70009B7949F8010094809371574B1B68002B63
:105F800000F0438504F01CFC3EAF0446620838462E
:105F90003349059705F066FAE40700F1A9860598EC
:105FA00005F0A3FA059C4B4B059F221801469C88DF
:105FB00018689B7978509480937104F05BFA0246DC
:105FC000002840F0818546AF07F85C0D04F048FCDE
:105FD0000246002840F0708546AC04F8700D069427
:105FE0003E48FEF7F5FEFEF757FF40460221FFF759
:105FF00039F83B484946FFF7D5F902243948059955
:10600000FFF7D0F938483949394A00943B46FFF741
:1060100013FA3849384A069B33480094FFF70CFAC4
:10602000FFF74EF83048FFF7D7F927483349FFF715
:106030004DF8FFF7EFF9002D7FF40BAD7EE421461C
:106040000F70FFF7C3BA00BF58E00008B0E60008C1
:10605000C8E7000864E8000874E8000884E800085D
:1060600034ED0008E8E700088CE8000898E800082C
:1060700088E10008ACE8000818E20008D4E700084E
:10608000B4E80008E0E70008BCE80008D0E8000831
:1060900004E10008ACF6000820E20008CCE70008A4
:1060A000D4E8000868E80008E0E8000878E800089C
:1060B000F4E8000804E9000820E90008FCDF000813
:1060C00040E9000850E9000860E9000800E600081F
:1060D0005013002078E900088C04002080E90008B3
:1060E00098E90008A8E900089CE90008B0E9000860
:1060F00044E90008D8E9000854E9000800EA00086B
:10610000B04B93E8070003F10C0425AE86E80700C6
:1061100094E807002AAD03F1180485E8070094E825
:1061200007002FAF03F1240487E8070094E8070075
:1061300030330DF1E40989E8070093E80700089679
:106140003EAE86E8070006950596FDF73BF90B90F5
:10615000FDF7DEF80546FDF7BFF90C90FDF768FC8A
:106160008046FDF765F9984C0D9015A8FDF718FCD1
:10617000236805F00102C5F3400B079253B9934A17
:106180009348191808334968902B42F8041FF8D136
:10619000012323608F48FEF7D7FD0446002800F056
:1061A00002868D4905F08FF9002800F06B832046A8
:1061B0008A4905F088F9002840F0A5858848FEF74F
:1061C000DDFD002800F01D86012645F00205099638
:1061D000CAF8005047262046824905F074F9054662
:1061E000002800F0618520467F4905F06CF9002801
:1061F00040F0A7857D4DDFF878A20A9558260DF16D
:10620000580B42467A49584605F02CF9794B7849A3
:106210005A690DF160081EA805F024F91AAD7449F9
:106220009DF85420404605F01DF91CAC70499DF8BE
:106230005520284605F016F99DF856206C49204651
:1062400005F010F90A9BCDF8D0801A683595369480
:10625000002A40F0228546AC04F8982D6648FEF7E7
:10626000B7FDFEF719FE08980321FEF7FBFE079D18
:1062700062486349634A644B0095FFF707F90B9D39
:106280005E48009512256149614A624B0195FFF70E
:1062900013F9099D594800955F49514A5F4BFFF733
:1062A000F5F80D9D002D00F0D0840C9D002D00F020
:1062B000DE8402235A4A5B495B4800932346FFF77A
:1062C000BBF8FEF7FDFE4D48FFF786F857485849E2
:1062D000FEF7FCFE57485849FEF7F8FE424857497A
:1062E000FEF7F4FE56485749FEF7F0FEFFF792F826
:1062F000BAF1000F3FF422AB5348FEF75DFD504664
:10630000FEF75AFD5148FEF757FDFFF717BB5048FF
:10631000FEF752FDA0461EAD20AC42464D49284630
:1063200005F0A0F82846FEF747FD4B48FEF744FD70
:10633000404621461022FEF78DF800283DD0002768
:106340000CE0E25D284605F08DF82846FEF734FDA6
:1063500001374248FEF730FD102F0BD007EB080342
:10636000B3F5A27F3E493F48EBD90137FEF724FD44
:10637000102FF3D13948FEF71FFD002320212E20D6
:1063800003EB0802B2F5A27F88BFE15404D8E25CB7
:10639000203A5E2A88BFE0540133102BF0D100234D
:1063A00020468DF8903008F11008FEF705FD2E48C4
:1063B000FEF702FDB8F5A87FAFD12C48FEF7FCFC34
:1063C000FFF7BCBA60E00008A80C0020A80B002072
:1063D000ACDE0008B0E60008A8EA0008B4EA00084D
:1063E000B8EA000804EB000814EB000840040020A1
:1063F00034ED00087C01002028EB000818EB0008B1
:106400003CEB0008ACEA000844EB000864EB000831
:10641000F8EA0008AC0B0020D8E1000874EB000893
:1064200008EB0008A0EB00089CE90008C0E60008A3
:106430003CE70008C8E6000848E70008B8EB000899
:1064400020EB0008C8EB000884E7000824E90008F6
:106450009CE70008A4E70008ACE70008E8E30008B0
:1064600088F40008B8E700087CE10008B0E70008FD
:1064700034E60008B34D0FCD3EAC05940FC495E84B
:106480000F0084E80F00B048FEF75EFC044630B110
:10649000AE49062205F031F8002800F03282DFF81C
:1064A00030B30DF1E409AA48FEF792FC25ACFEF7E3
:1064B000F3FC05980821FEF7D5FD1AAD08941CAC35
:1064C0004FF0000A079509942AAD20AC0695564670
:1064D0002FAF0DF1D0081EAD05940BEB0A0C48F65A
:1064E0008904DCF804209B49CDF80CC0C8F6880468
:1064F000A4FB02025209099804F0B4FFDDF80CC0B5
:106500009449DCF80420A4FB02035B09C3EB0313EA
:10651000A2EB8302284604F0A5FF8F48FEF770FF28
:1065200032468E49079804F09DFF32468C49059803
:1065300004F098FF32468B49089804F093FF3246E6
:106540008949069804F08EFF32468849384604F09F
:1065500089FF32468649404604F084FF0798FEF7DB
:1065600007FD5BF80A2083490898C2F3C012FEF7C2
:1065700031FE5BF80A207F490698C2F38012FEF7CD
:1065800029FE32467C49484604F06CFF5BF80A203D
:106590007A48C2F3C204FEF70FFC0723224678496B
:1065A0004846FEF7C1FD7748FEF706FC32467649BD
:1065B000484604F057FF5BF80A20704802F00704D1
:1065C000FEF7FAFB224607236D494846FEF7ACFD6D
:1065D0006C48FEF7F1FB02246848FEF7EDFB6549C5
:1065E000099A009423463846FEF7D6FC6548FEF724
:1065F000E3FB6248FEF7E0FB5E4900942A4623462F
:106600004046FEF7C9FC5F48FEF7D6FB0136059809
:10661000FEF70EFDFEF704FF082E0AF1080A7FF4CC
:106620005CAFFEF74DFD0026FFF788B9574F584D78
:1066300097E8070007F13C040DF1D00888E807004F
:106640000FCC3EAE503705960FC697E80F00246872
:106650002F6834600DF1E40989E80F00002F00F085
:106660002181DFF870B1FCF7FFFE0746FCF734FF2D
:1066700005463548FEF768FB0446002800F0BE8357
:10668000444904F020FF0346002800F0C28220465F
:10669000414904F018FF0346002800F071832046AA
:1066A0003E49032204F029FF0646002800F06984D1
:1066B00020463B49062204F020FF0646002800F051
:1066C000B68420463749072204F017FF0646002803
:1066D00000F0948420463449042204F00EFF06465C
:1066E000002800F056852046304904F0ECFE0026D4
:1066F000B24610B9DFF8E0A053262D48DFF8D4B039
:10670000FEF766FB0B24FEF7C7FB40460321FEF7AE
:10671000A9FC28482849294A294B019400970224BA
:10672000FEF7CAFE2749284A284B224801940095C3
:10673000FEF7C2FEFEF7C4FC05980521FEF792FCA9
:10674000002451E0C0E00008B0E6000840ED000879
:1067500058ED0008A8E60008E4E1000834ED000860
:106760006CED000874ED000878ED00087CED000881
:1067700080ED000804E1000850ED000818E2000870
:106780001000002020E2000854ED000860E000083E
:10679000A80B0020E0EB0008F0EB000804EC000878
:1067A00008EC000820EC000830EC000820EB0008A2
:1067B00038EC0008B4E1000850EC0008E4EB0008F5
:1067C0007C0C00205CEC0008F4EB0008F40B0020CB
:1067D000AC6200205000002048E6000801340B2C79
:1067E0000BF1140B00F0FB80DBF81030D807F5D567
:1067F0002246B9491AA804F035FE2246B7491CA81A
:1068000004F030FE2246B6491EA804F02BFE2246B4
:10681000B44920A804F026FEDBF80820B24918A8E5
:1068200004F020FEB148FEF7EBFDDBF80000FEF7B8
:106830009FFB18A91CA8AE4AFEF790FD1EA8FEF704
:1068400075FDDBF81020AB49C2F3400220A8FEF72B
:10685000C1FC1AA8FEF7ECFBFEF7E2FDBEE7A64876
:106860000999FEF79FFDFEF7C9BF2846A34904F02A
:106870002AFE002834D10123CAF800305026A04C4B
:10688000FEF79EBF9F48FEF779FA002800F0558278
:10689000012645F001050796CAF80050CDF824B04E
:1068A000472698E4984ADFF8C0B23B4653F80B10ED
:1068B0001433DC2B42F8041FF8D1944B94491A6826
:1068C0001B6981E80C0001232B60CCE606460446D8
:1068D000FEF776BFDFF894A24E260446FFF797BA7C
:1068E00028468C4904F0EFFD002840F01B83CAF8CD
:1068F00000005026884CFEF763BF00263546FFF7A0
:106900001CBBA01D04F068FA072804463FF6C7AD7B
:1069100001468248FEF740FA814904F0D4FD002880
:1069200000F05683DFF848B25BF8343023F0800380
:106930004BF8343021467B48FEF72EFA784904F0B4
:10694000C2FD002800F03D835BF8343023F04003A3
:106950004BF834300DF1E40922467349484604F0FF
:1069600081FD4846FEF7F0F904F036FA22466F49F9
:106970000546484604F076FD4846FEF7E5F904F082
:106980002BFA5BF83430ED0000F0070023F03F03F2
:1069900040EA030205F0380313434BF83430214634
:1069A0006348FEF7F9F904F017FA214605466148F5
:1069B000FEF7F2F904F010FA0BEBC404C5EB051571
:1069C00000EB8500606003F04FF86CE501F0A2FA7F
:1069D000594DFEF7EBBF06468346FFF720B9FEF799
:1069E0006FFB48460421FEF73DFB544D00242B6805
:1069F000D90700F1BF8001341035022CF7D1FEF722
:106A00005FFB3A48FEF7E8FC6CE44D4B93E803006B
:106A10003EAC059484E80300FFF7CFBA484B93E8F7
:106A200003000DF1E40989E80300FFF7A6BA224646
:106A300044491AA804F016FD224643491CA804F054
:106A400011FD224641491EA804F00CFD55F8082C02
:106A5000254914A804F006FD3D48FEF7D1FC55F881
:106A60000C0CFEF785FA14A93A4A1CA8FEF776FC2E
:106A70001EA8FEF75BFC1AA8FEF7DAFAFEF7D0FCB8
:106A8000FFF737B93448FEF75FF904F0A5F9074678
:106A90003248FEF759F982463148FEF755F9044667
:106AA000002F00F0B38104F020FD092800F2C88116
:106AB0002C4CB246FFF7ABB92AAC20460A490694E3
:106AC00004F0D0FCFFF78CBA2FAF3846064904F02B
:106AD000C9FCFFF77BBA00BF6CEC000810EC0008A3
:106AE00074EC000818EC000834ED0008B4E100086C
:106AF0007CEC000804E1000824E70008C0E6000878
:106B00000CE50008ACEA0008780C00207C010020AD
:106B1000F40B0020C8E6000824E5000848ED000852
:106B2000E0E000084CED000850ED000854ED0008CE
:106B3000F0E6000884F000081CE600088801002048
:106B40003CE5000828ED0008D4EC000830ED000812
:106B5000CCE100089CEB0008D4E70008E0E700085F
:106B6000ACF6000844E5000850000020ECE5000801
:106B7000AC6200202246BF4925A804F073FC2246DF
:106B8000BD492AA804F06EFC2246BC492FA804F097
:106B900069FC55F8082CBA4916A804F063FCB948FA
:106BA000FEF72EFC55F80C0CFEF7E2F916A9B64AD2
:106BB0002AA8FEF7D3FB2FA8FEF7B8FB25A8FEF7FF
:106BC00037FAFEF72DFC16E7B048FEF7BDF804F0E3
:106BD00003F903F055FC3546FFF7AFB92FAF384640
:106BE000AB49BDF83A2004F03DFCFEF7F5BEA948DC
:106BF000FEF7AAF803F0D0FE002800F0BB80344670
:106C0000DFF8E8A2FFF703B901F068F9A24DFEF73B
:106C1000CDBEA2480493FEF797F804F0DDF8CAF859
:106C20000000049B074641269A4666E59C48FEF70D
:106C30008BF804F0D1F803F08DFE002800F0AD8051
:106C40003446DFF8ACA2FFF7E2B88E48FEF7D8FB77
:106C50009448FEF78DF98C4A93485946FEF77EFB1F
:106C60009148FEF7E5F9FEF7DBFBFFF71EBB059D3C
:106C7000CDF800900195834806993A4634ABFEF76B
:106C800041FCFFF716BB8948FEF75EF804F0A4F854
:106C900003F0ECFD3546FFF750B920AC20467849AB
:106CA00004F0E0FBFFF7DABA814B82480A93FEF763
:106CB0004BF804F091F80A9CAA462060FFF79FBAAF
:106CC0007948FEF741F804F087F862260990CAF87F
:106CD0000000FEF7A4BF484604F007FC764B09EB22
:106CE000000219889B7829F800109370FFF737B9D4
:106CF000059804F0FAFB704B3A1819889B783952C2
:106D00009370FFF74CB920466C4904F0DCFB002877
:106D100000F04A8120466A4904F0D5FB002800F0C3
:106D2000BA812046674904F0CEFB002800F0598163
:106D3000CDF824B00026FFF74EBA25F001050790E4
:106D4000AAE52046604904F0BEFB002840F0098116
:106D5000574D0123CAF800305026DFF898A10A9554
:106D6000FFF74DBA26462546FEF720BE06460546E5
:106D7000FEF71CBE06460446DFF87CA1FFF747B8C5
:106D800052480493FDF7E0FF04F026F8CAF800002B
:106D9000049B054646269A46AFE406460446DFF8BD
:106DA0005CA1FFF734B8424BCDF824B006468246CA
:106DB0000A93FFF724BA064604468246FFF727B82F
:106DC0004348FDF7C1FF04F007F88DF83C00414847
:106DD000FDF7BAFF04F000F88DF83D003E48FDF7DE
:106DE000B3FF03F0F9FF8DF83E000F9B1A0CAAF8D1
:106DF00000308AF802206326FEF711BF064682465D
:106E00007BE425F002050990FFF7E2B93348FDF76E
:106E1000DFFF3348FDF7D0FFFEF776F9FEF77EFA85
:106E20004FF4FA70FAF70AFD2E4B6F6085F83C704C
:106E3000504621461F603E46FDF79CFEFEF716BCFD
:106E40002648FDF7C5FF2848FDF7B6FFFEF75CF9B9
:106E5000FEF764FA4FF4FA70FAF7F0FC214B6E601B
:106E600085F83C60504621461E60FDF79BFEFEF70C
:106E7000FDBB00BF80EC000828EC000888EC00088F
:106E800034ED000818EB00089CEB000844E900080A
:106E900038EA000868E800081CE60008E4EB00088F
:106EA00078E8000888EB0008F0F9000854E90008C9
:106EB0004004002008EB000874E90008C4EA000858
:106EC000D4EA0008F4EA0008C0E60008F4EB000881
:106ED000E0EA0008E4EA0008ECEA0008E8E7000855
:106EE000FCE70008C412002030E8000864E5000850
:106EF000ACE500080CE5000888E50008CCE50008D2
:106F0000C248FEF77DFAC248FEF732F8C14AC248CD
:106F100010A9FEF723FAC048FEF78AF8FEF780FAB8
:106F2000FEF7C9BE2846BD4904F0CDFA0B900028F3
:106F300000F0D1802846BA4904F0C5FA044600287A
:106F400000F0358100263446FEF73ABCB548FDF71F
:106F5000FBFE03F041FF64260790CAF80000FEF72D
:106F60005EBE2046B04904F0AEFA002840F03E81F3
:106F7000AE4BCAF800005026DFF800A30A93FFF7D3
:106F80003EB9E01C03F028FF0A280AD800EB800075
:106F90000BEB800BB246DBF80C30CBF80830FFF778
:106FA000ACBBB246FFF7A9BB9B48FDF7CDFE03F093
:106FB00013FF42268046CAF80000CDF824B0FFF740
:106FC0000AB95BF8343043F040034BF83430C1E485
:106FD000DFF8ACB25BF8343043F080034BF8343068
:106FE000A8E49348FDF7B0FE03F0F6FE44260B90AC
:106FF000CAF80000CDF824B0FFF7EDB8E01D03F0AB
:10700000EBFE01280446CCD802468A492AA804F09F
:1070100029FA2AA8FDF798FE03F0DEFE0F28C0D853
:10702000854B03EB0414B2466060FFF766BBA01DFE
:1070300003F0D2FE0A288246B3D802467F4920AC2C
:107040001CA804F00FFA7E495246204604F00AFAC2
:107050001CA8FDF779FE03F0BFFE431E0E2B4FEA7E
:107060008A069CBF06EB0A030BEB8303564498BFCA
:1070700098602046FDF782FE0BEB860B002800F09F
:107080002A81DBF81030002643F00203CBF81030E1
:10709000B246FFF732BB6B48FDF756FE03F09CFE8D
:1070A0008DF854006848FDF74FFE03F095FE8DF80B
:1070B00055006648FDF748FE03F08EFE8DF8560039
:1070C000159BCDF824B01A0CAAF800308AF80220DB
:1070D0004326FFF780B85E48FDF736FE03F07CFEDE
:1070E00003465C480493FDF72FFE03F075FE8446CB
:1070F0005948CDF80CC0FDF727FE03F06DFE04469D
:107100005648FDF721FE03F067FE0C905448FDF74A
:107110001BFE03F061FE049B0D901A465149484640
:1071200004F0A0F9DDF80CC04F496246304604F087
:1071300099F922464C4914A804F094F94A490C9A4A
:1071400015A804F08FF948490D9A584604F08AF9B9
:107150000C9E049BDDF80CC0CAF808600D9ECAF8AE
:107160000C40CAF804600B9EA3F26C710CF1FF3264
:10717000CAF81C10CAF81020CAF800602046614600
:107180001A46F9F7ADFF5426CAF818000B9CFEF713
:1071900017BB201D03F020FE01283FF602AF264B4F
:1071A00003EB0013B2469A685A60FFF7A6BA2F485D
:1071B000FDF7CAFD1E220146504604F0B7F97026BD
:1071C000FEF7FEBAE81D03F007FE0328054664D962
:1071D000B346FEF724BD2648FDF7B6FD03F0FCFDDF
:1071E000FCF7E8F8B3460B90FEF719BD20460F4CAC
:1071F00020490A9404F067F91F4B00280CBF9A46F7
:107200004FF0000A08BF5326FEF7F9BFCCE1000893
:1072100088EB00089CEB0008F0F90008D4E60008B1
:10722000FCE60008A0EC0008C8E6000840040020C6
:10723000F8EA000828EC00087C01002010EC0008A7
:1072400018EC0008E0EA0008E4EA0008ECEA0008AC
:10725000E4E60008ECE60008F4E600089CF9000803
:10726000F8E60008A4E60008A8E6000800E7000821
:10727000C0EC000820EB000848E6000824E5000800
:10728000AC6200201948FDF75FFD03F0A5FDFCF797
:1072900083F8B3460A90FEF7C2BC024614491CA804
:1072A00004F0E0F81CA8FDF74FFD03F095FD0F2852
:1072B0008ED807EB0515B3466860FEF7B0BC281DF5
:1072C00003F08AFD032883D807EB0013B3469A68BE
:1072D0005A60FEF7A4BCDBF8103023F00203064628
:1072E000CBF810308246FFF708BA00BFB0EC0008B8
:1072F000D4EC000830B585B04FF480446846F9F707
:107300007FFB0022200448F2A063C0F201030121A8
:10731000ADF80420ADF8082040F4B8404FF4806286
:107320004BF6FF75ADF80650ADF80A20ADF80C40ED
:107330000093F9F773FB200440F4B8406946F9F76D
:10734000EFFA05B030BD00BF10B54FF4B844C4F239
:10735000000420460121F9F77DFB20460121F9F7C1
:107360009FFB20460021F9F79BFB2046F9F7A0FA86
:10737000BDE81040FFF7BEBF70B505460E4643F2AC
:10738000010401E0013C13D04FF4B8402946C4F297
:107390000000F9F799FB0028F4D04FF4B840C4F28C
:1073A00000003146F9F790FB0028EBD0012070BDBA
:1073B000FFF7CAFF204670BD38B5054619B1BDE8D4
:1073C0003840FFF7D9BF43F2010401E0013C0AD085
:1073D0004FF4B840C4F200002946F9F775FB0028C5
:1073E000F4D0012038BDFFF7AFFF204638BD00BF05
:1073F000F8B507464FF4B840C4F200000E4601212C
:1074000015461C46F9F718FB0120C1F200000021C7
:10741000FFF7D2FF002832D04FF4B840C4F200008A
:1074200034BB0121F9F72EFB4FF4B844C4F2000439
:107430002046F9B20022F9F71BFB0220C1F200003E
:107440000021FFF7B9FFB8B18020C1F20000002190
:10745000238BFFF7B1FFA8B125B1C6F30721204662
:10746000F9F72CFB2046F1B2F9F728FB0020F8BD14
:107470000021F9F707FBD7E76FF00100F8BD4FF0E7
:10748000FF30F8BD6FF00200F8BD00BF30B5284BEB
:107490001C6883B00CB103B030BD012568461D6087
:1074A000F9F7D8F929464FF40000F9F78FFB284681
:1074B0002946F9F77DFB04202946F9F779FB29468F
:1074C0004FF40000F9F79EFB21464FF40000F9F756
:1074D00099FB002008210422C4F20200F9F7D0F938
:1074E0004FF4006004220921C4F20200F9F7C8F940
:1074F0000223002069468DF804308DF80530C4F26F
:1075000002004FF4807300938DF806508DF8074009
:10751000F9F744F94FF400604FF40073C4F202002D
:1075200069460093F9F73AF9FFF7E4FEB3E700BFC5
:10753000B00C00202DE9F041069D6F1E1E467B42D7
:107540007B418046FFF754FF074610B13846BDE83F
:10755000F08180200421C1F20000C1F20001FFF798
:107560000BFF00285BD04FF4B844C4F2000420465F
:107570000121F9F761FA0120C1F200003946FFF755
:107580001BFF00284ED020465FFA88F10122F9F750
:107590006FFA0220C1F200003946FFF70DFF002804
:1075A00043D0238B8DB33C4611E040200021C1F233
:1075B0000000FFF701FF18B34FF4B840C4F2000019
:1075C000F9F77EFA3219AC4202F8010C1DD00134F1
:1075D000AC42EAD14FF4B840C4F200000021F9F700
:1075E00051FA4FF4B840C4F200000121F9F732FA21
:1075F00040200021C1F20000FFF7DEFE0028DBD1B1
:107600006FF006073846BDE8F0814FF4B840C4F289
:1076100000000121F9F736FA3846BDE8F0816FF035
:10762000030793E76FF0040790E76FF005078DE716
:1076300070B51C460023FFF7DBFE064608B1304656
:1076400070BD8020C1F200003146FFF7B5FE28B3BF
:10765000049BD3B1049BE51801E0AC4215D04FF474
:10766000B84014F8011BC4F20000F9F727FA802093
:107670000421C1F20000C1F20001FFF77DFE0028E5
:10768000EBD16FF00306304670BD4FF4B840C4F242
:1076900000000121F9F7DEF9304670BD6FF00206F7
:1076A000CDE700BF70B43A4A3A49546A0B689C422D
:1076B00007D8956AAB4204D2D56B002D4FD0364D1A
:1076C00013E0D46A324DA34208D21268032A15D0BF
:1076D000052A20D001330B6070BC70472E6BB3427B
:1076E000F3D2ED6B002D40D02C4D2E681C1B00FA00
:1076F00004F426432E601268032AE9D1102BE9D93D
:10770000142BE7D8264AA3F11105146800FA05F0F6
:1077100004431460DEE7A3F11402032A16D9A3F18F
:107720001804032C27D81F4C256800FA02F21543D1
:107730002560DA0810BB1C4803F00704855C0126AD
:1077400006FA04F425EA04048454C3E7134AA3F1B7
:107750000805146800FA05F52C431460E9E70E4C9F
:10776000256840EA45052560AFE70C4C256840EAEE
:1077700045052560A9E72F2BACD8DAE70A4803F0C6
:107780000704855C012606FA04F42C438454A1E71F
:10779000DC0C0020C40C0020200D00203C0D00203B
:1077A000340D0020380D0020B40C002000B583B04B
:1077B0006846F9F74FF804200121F9F7F9F94FF479
:1077C000006000234FF48062C4F202006946009218
:1077D0008DF804308DF805308DF806308DF80730BF
:1077E000F8F7DCFF03B000BD70B4294A1368002B22
:1077F0002BD028490B68022B17D0032B264B26D001
:10780000264C0E682168264DA0F8011019680670F4
:10781000A0F803102E680021196046712160012034
:1078200029600023136070BC70471B4B1D681C68E7
:10783000E443E4B2B4EB152F1BD0184C266848F291
:10784000EE75AE421AD00020EBE71846EBE71D6854
:107850001C68E443E4B2B4EB152FF4D11D680F4C5F
:10786000EDB21D600F4D2E681D6845EA06251D60AE
:10787000C7E71D68094CEDB21D60C2E70B250D601E
:107880001D68C5F3072525601D68EDB21D60B8E7CA
:10789000440D0020BC0C0020C00C0020280D00204E
:1078A0002C0D0020CC0C00202DE9F0474FF4006097
:1078B0009E4CC4F202004FF48061F8F7D5FF2368B4
:1078C00093B99B4E356895B99A4B002800F0C28059
:1078D0001B68002B40F00C81974B1A684FF6FE7125
:1078E0008A4201D801321A602068BDE8F087934FC0
:1078F0003A68002A70D0002800F0B280904A1178CF
:107900000131C9B2E929117000F206818D4B8E490F
:107910005A6B09688A42E7D1996B0029E4D1DFF8F4
:1079200068828A49D8F800C00D68AC4500F07881BB
:107930008748002707601B68012B00F06481052B36
:1079400000F079810A2B18BF292B03D10068C007EA
:1079500000F155810120022B206040F09C81002A1B
:1079600040F0028274480368B3F5E16F80F016823C
:10797000784D794FD5F800903B68DFF8F4A1C1F855
:1079800000C049F00109C5F80090CAF80030026053
:107990006546724A3B6002201060714A1360714B69
:1079A0001A68714B1D60714B1A60236863B10B68D4
:1079B0009C4500F0BA816E4A5F481568664FC8F86A
:1079C000003000233D6003605A4A002313605C4A84
:1079D00033600B60137087E7664F3B68002B00F045
:1079E0008180584B002840F0D1801A68032A00F0AB
:1079F0005581DFF84C81DFF83C915A68D9F80010C6
:107A000050488A420BD88268914208D898F800C042
:107A1000C268944503D30269944540F2B3815B691F
:107A2000484A99420BD39369994208D898F80010B4
:107A3000D369994203D3136A994240F2A981002580
:107A4000356088F800500123C9F80030002D3FF45C
:107A50004BAF5BE71A6801321A602068BDE8F08717
:107A6000DFF8D090DFF8D880D9F80030A3F11F02FA
:107A70000A2A17D898F80020052A13D90A2A11D8FB
:107A80003D493048442203F003FA2F4A0023136093
:107A90000122C9F8002088F800303B60002D3FF437
:107AA00023AF33E7A3F15E02532A08D898F80020E9
:107AB0002D2A00F29F80162A01D93049E1E7A3F16F
:107AC0003C020F2A40F28980283B162B00F28F805F
:107AD00098F80030122B40F28A801F2B00F287802A
:107AE0002749CEE7E8B9134B1A6801321A600DE74F
:107AF000204B124A1D6001231360144A3360156045
:107B00001B4A15601F4A1560164A15600E4AFF2170
:107B100011600B4A1370E7E6064933600B6013707F
:107B2000E2E6074A01233B601370EFE6440D0020B4
:107B3000C80C0020400D0020D00C0020240D002097
:107B4000D80C0020DC0C0020C40C00203C0D0020D0
:107B5000300D00202C0D0020B0010020BC0C0020B6
:107B6000280D0020340D0020C00C0020CC0C00207B
:107B7000200D0020D40C00203CEE000808EF000887
:107B800080EE0008380D0020AC0100208C49D3F8AD
:107B90003490D1F800C0E14500F09180DFF85482C4
:107BA0001A6898F800A087480AF1010A5FFA8AFA71
:107BB000012A88F800A000F09A80BAF1E90F7FF658
:107BC00045AF09F1FF32944500F0C4807E4A00239E
:107BD0003360136088F8003086E698F800203B2A6E
:107BE0007FF672AF4B2A3FF66FAF784949E7002521
:107BF00035604AE7592A3FF662AF754941E7754853
:107C000000230360D1E60268013A012A88BF23609D
:107C1000F5D9714A714812680360714B1A60BEE66B
:107C20006C480068B0F5966FBFF482AE6D48076887
:107C3000013707607FE60368012BE0D00123236052
:107C4000694B1F7858789A7887EA000909F00F097C
:107C500089EA171787EA101002F00F09814501D051
:107C60000020206093F803901F79587982EA090375
:107C70007B40984201D0002323605C4B5C4A1F6824
:107C80001068554A38431860544B12680520186034
:107C9000534B1A6083E6052BD2D0BAE748490A68ED
:107CA000102A7FF4A6AEDFF82091D9F80020053A1B
:107CB000072A79D94F4B306018700546C3E6986B98
:107CC00001287FF46BAFDFF800915869D9F80010F4
:107CD000884205D89869814298BF9A637FF6B6AE0C
:107CE000444A00233360C9F800301370FCE5BAF150
:107CF0000B0F7FF6ABAEBCF10A0F7FF65EAFDFF87D
:107D0000D890C16AD9F80020ACF10B0A614442EA6C
:107D10000A220CF1010C0131C9F800200A22C0F836
:107D200034C0016388F8002065E62B48324F0568AF
:107D30003A682848AA427FF442AE026840F6C90C6D
:107D400062459FBF294AD2F800C04CF0010CC2F82E
:107D500000C034E69B6B002B7FF438AFC1F8009075
:107D6000002D3FF4C1ADD1E51B4B234F1B6810E63E
:107D70000A200F3A2021186010200F2AD8621963B8
:107D8000596305D80120FFF78DFC00233B605AE6BC
:107D90000020FFF787FC00233B6054E6174B164F8B
:107DA0001A600D4B1B68F4E5124A12783B2ADFD9A2
:107DB0004B2ADDD800233B6011230B6043E600BF54
:107DC000C40C0020DC0C0020400D00204CEF00080B
:107DD000C4EE0008D00C0020200D0020BC0C0020B8
:107DE000280D0020300D0020B40C00202C0D0020A8
:107DF000380D0020D80C0020B0010020440D0020D8
:107E0000F9F742B910B582B004460DF10600F9F752
:107E100049F978B1084B09491B88BDF80620098843
:107E2000D21AC2EB0212CB1A92FBF3F30F2B28BF2C
:107E30000F23236002B010BD480D00204A0D002022
:107E400008B50F4B1B686BB1FF23C0F202039842C9
:107E50000AD80C4B00221A800B4B40F2FF321A80DA
:107E6000012008BD184608BD02220649E120FCF7A2
:107E7000F1FAE32004490222FCF7ECFA012008BDE4
:107E8000A0040020480D00204A0D002008B50A4B30
:107E90001B680BB9002008BDE12008490222FCF74D
:107EA000F3FA0028F6D00222E3200549FCF7ECFAA9
:107EB000003018BF012008BDA0040020480D00209C
:107EC0004A0D002040F64853C2F20003188870475C
:107ED00040F64A53C2F200031888704710B582B0CA
:107EE000F9F7D2F80A240DF10600F9F7DBF840B9EA
:107EF0000A20F9F7A3FC013CF5D1054C208802B01B
:107F000010BD034CBDF806302380FFF7BFFFF5E737
:107F1000480D002010B582B0F9F7B6F80A240DF12B
:107F20000600F9F7BFF840B90A20F9F787FC013CD1
:107F3000F5D1054C208802B010BD034CBDF80630C9
:107F40002380FFF7A3FFF5E74A0D0020F9F742B8B9
:107F5000F0B507468DB00A20FCF78CFC092828D024
:107F60000A2813D0072803D0002420460DB0F0BD06
:107F7000FCF7D6FD0A2201A900F5B67003F004FC57
:107F80000146384602F01AFD7424EEE7FCF7C8FDFE
:107F900000F14C042021204603F088FA014610B17C
:107FA000002301F8013B20463A46FDF7E3FA044678
:107FB000DBE7FCF7B5FD01AE00F5A674002502E095
:107FC00002340A2D12D0237820460221002B7BD0C8
:107FD0006378002B78D0F9F7BDF8A37846F8040F42
:107FE0000135202BECD103340A2DECD1029CA4F1F5
:107FF00041032F2BB8D801A252F823F0BD8000080E
:10800000BD80000817810008BD800008697F000856
:10801000BD800008BD800008697F0008697F0008F6
:10802000697F0008697F0008BD800008697F00083B
:10803000D1800008697F0008BD800008697F0008C2
:10804000697F0008D1800008F1800008697F00087E
:10805000697F0008D1800008697F0008697F0008F7
:10806000697F0008697F0008697F0008697F000850
:10807000697F0008697F0008697F0008697F000840
:10808000BD80000817810008BD800008697F0008D6
:10809000697F0008697F0008697F0008697F000820
:1080A000697F0008697F0008697F0008697F000810
:1080B000697F0008697F0008D9800008022D7FF4DD
:1080C00053AF039B3B6050E7002D3FF44DAF8DE76E
:1080D000012D7FF449AF48E73846202300F8013BE3
:1080E0000DF109011E2203F021FA0023FB773CE782
:1080F000072D7FF439AF059BFB60039B03F16402FE
:10810000049B7A61013B3B61069BBB60079B7B60E4
:10811000089B3B6029E7042D7FF426AF039B3B704F
:10812000049B7B70059BBB701FE700BF70B53E4B87
:108130001A68824288B0064673D002A81E60F8F71B
:1081400089FB04A8F8F7CCFE01200146F8F730FDC2
:1081500001200146F8F72CFD4FF400300121F8F71B
:1081600035FD0020C4F2020002210722F8F788FB47
:1081700000200722C4F202000321F8F781FB02234A
:1081800000208DF80C30032304460125C4F20200C0
:1081900002A98DF80D30042302938DF80E408DF85E
:1081A0000F50F8F7FBFA20460823C4F2020002A998
:1081B0000293F8F7F3FA4FF48840C4F2000029461E
:1081C000F8F7A8FE4FF488400C23C4F2000004A97D
:1081D000ADF81A300496ADF81440ADF81640ADF87D
:1081E0001840ADF81C40F8F70FFE4FF48840C4F279
:1081F00000002946F8F780FE4FF48840C4F20000E2
:1082000040F225512A46F8F79BFE262301A88DF857
:1082100004308DF805408DF806408DF80750F8F7CA
:1082200017F808B070BD00BF640F002030B40F4ACB
:1082300013687F2BFCD80E490E4D0B685C1C7F2CFD
:1082400045F8230098BF0C6001D900230B6072B67B
:1082500013680133136062B64FF48840C4F2000023
:1082600040F22771012230BCF8F76ABE600F00208F
:108270005C0F0020540D002010B50446007828B192
:10828000FFF7D4FF14F8010F0028F9D110BD00BF8B
:1082900030B40D4B1A6882B10C490D4D0A68541C5C
:1082A000802C55F8225018BF0C6009D072B61A689D
:1082B000013A1A6062B601220560104630BC704770
:1082C00000220A60F2E700BF500D00204C0D002094
:1082D000680F0020024A1368002BFCD1704700BFD2
:1082E000600F00204FF4884038B5C4F2000040F21F
:1082F0002551F8F741FE00282BD14FF48840C4F2F5
:10830000000040F22771F8F737FE00B938BD4FF48E
:108310008840C4F2000040F22771F8F753FE234B67
:108320001A68002A38D0224A224C1168481C80283A
:1083300008BF002054F8211010601A684FF48840DC
:10834000013AC4F2000089B21A60BDE83840F8F77B
:10835000EFBD4FF48840C4F2000040F22551F8F719
:1083600031FE4FF48840C4F20000F8F7E5FD124BEF
:108370001A687F2AC1D81149114D0A68541CC0B22D
:108380007F2C45F8220098BF0C6001D900220A60BA
:108390001A6801321A60B0E74FF48840C4F2000056
:1083A00040F22771BDE83840F8F7CABD600F0020E1
:1083B000540F0020540D0020500D0020580F0020B5
:1083C000680F002010B541F26814C2F200040246A2
:1083D0000B4620464FF4807103F000FD2046BDE8B7
:1083E0001040FFF749BF00BF0FB400B583B004AB26
:1083F00053F8040B19460193FFF7E4FF03B05DF84F
:1084000004EB04B0704700BFFFF790BE10B584B016
:1084100001A8F8F751FC01200146F8F7D7FB00232B
:10842000ADF80C30ADF80630072301A902934FF0E8
:10843000804003F52D73ADF80430F8F7F1FB01210E
:108440000A464FF08040F8F7C7FC01240F23684626
:108450001C228DF800208DF803408DF801308DF836
:108460000230F7F7F5FE4FF080402146F8F73CFC6C
:1084700004B010BD38B54FF080400121F8F7B6FCCC
:108480006A4B1C68002C34D0694B1A6843F698215B
:1084900001328A421A6000D038BD664C6649674A8C
:1084A000012020600C6824180C6011680918116004
:1084B000146800213C2C1960EED1614B11601A68E0
:1084C00012181A605F4A10601A683C2AE4D15E4AAA
:1084D000196013681B1813601368182BDCD15B4BF1
:1084E00011601A6812181A601A68072AD4D1196024
:1084F00038BDFFF7D9F950490B68012B07D9544B08
:108500001A6840F6A660013282421A6043D0514B8D
:108510001A680132EA2A1A6054D04F4B1A680132A5
:10852000962A1A6048D04D4B1A680132962A1A6072
:108530003CD04B4B1A6801320F2A1A6030D03C4BAA
:108540001A6843F69820013282421A60A4D1394C4D
:108550003A4A012020600C6824180C601168091840
:108560001160116800242D291C6031D01268334B32
:108570003C2A38D01B681E2B53D03A4B1A68002A6D
:108580008AD01A68013A1A601B68002B84D1364BD6
:1085900001221A6080E71C60344B01221A60B6E7A2
:1085A000334A0120106000221A60C8E7314A0120D6
:1085B000106000221A60BCE72F4A012010600022E0
:1085C0001A60B0E72D4A0120106000221A60A4E76B
:1085D0002B4B1B491C680D68AC421FBF0968196012
:1085E000284B1860C2E7164A00211960136801334E
:1085F0001360144B0120186013683C2BBDD1124B43
:1086000011601A6812181A601A68182AB5D10F4A30
:10861000196013681B1813601368072B08BF1160DB
:10862000ABE7194B01221A60A7E700BFB412002084
:108630009012002070120020BC1200207C1200203A
:10864000C812002084120020A01200207412002002
:10865000B0120020B8120020AC12002068120020D6
:108660006C120020B401002094120020A4120020FB
:1086700080620020846200209C120020C012002032
:10868000C00100208C120020881200204EF690704D
:10869000C0F60000704700BF40F2B813C2F20003FA
:1086A0001868704741F2A02141F2C82241F27C23B0
:1086B000C2F20001C2F20002C2F2000346F28820B8
:1086C000C2F20000096812681B68816042600360A2
:1086D000704700BF2DE9F04F9FB001F07FFF02F01F
:1086E00025F84FF4E130FFF78FFEFFF75FF801F058
:1086F0003DFB01F067FBFFF789FE0120F9F7C2F8A7
:10870000F8F762FDF8F780FD01F01AFDFBF77AFE3D
:10871000F8F794FD002841F00A81BE48DFF8309355
:10872000FFF7AAFDBC48FFF7A7FDBC48FFF7A4FD73
:10873000B948FFF7A1FDBA48FFF79EFDB948FFF71A
:108740009BFDB548FFF798FDD9F80030002B01F0EC
:108750009680B548FFF790FDAF48FFF78DFDB34D0C
:10876000FBF768FD2B68002B01F08080B048FFF715
:1087700083FDA948FFF780FD2B68002B41F0B480F2
:10878000AC4CAD482168FFF72FFE226822F47F032E
:1087900023F47F43EBB940F2FF43C0F201039A4256
:1087A00001F2E38040F2FF632268C0F201039A42C3
:1087B00001F2D180A148FFF75FFD9748FFF75CFD0C
:1087C000206802F013F8206801F01AFE2068FFF715
:1087D00037FBFFF7BBFBF8F773FD01F0ADF941F292
:1087E000B420C2F200000123036002F049F841F214
:1087F000B421C2F2000100260E60FAF7B9FCFAF7C4
:10880000E1FD41F27822C2F2000241F2982A1060A2
:10881000FAF72AFE41F2A823C2F20003C2F2000ACC
:108820001860FAF759FECAF80000FAF701FE41F2A3
:10883000802EC2F2000E2B68CEF8000083B34FF4F6
:10884000807523687B4FC0F20205AB4228D07C487C
:108850002946FFF7C9FD754B3D601B68002B41F0B1
:10886000B7807848FFF708FD6B48FFF705FD01F07A
:108870001FFC002801F0A480FBF7ACFB002801F0EE
:10888000978002F033F8002801F08A8001F0ECF8BC
:10889000002801F058804FF48073C0F20203236077
:1088A00041F28C21C2F2000141F2BC220120C2F24D
:1088B000000208601468014602460334FAF73AFCE5
:1088C00041F2BC25C2F200050BA82B689C421ED9C0
:1088D000FEF78AFF0028F3D000210A460120FAF7AC
:1088E00029FC0120F8F7B8FF0BA8FEF77DFF002058
:1088F00001460246FAF71EFC5348FFF7BDFC464806
:10890000FFF7BAFC01F0DAFA08B101F0D1FB002060
:108910000146024606460890FAF70CFCFCF7C6F939
:10892000FCF7FEF84FF0010A0696089ECDF81CA051
:10893000DFF82081454F059600F13C0A8346042567
:108940003446CDF824A015A8FFF702FB8246002884
:1089500040F02D81D8F800303BB141F28022C2F2C4
:1089600000021368002B40F02F86069E002E40F078
:108970009783DBF80030002B40F0D3853348F8F7BD
:108980006BFC002840F0A08341F28C20C2F2000072
:1089900003685BB1D9F80030002B40F0CC8541F280
:1089A0008C2EC2F2000E0023CEF80030D8F8003032
:1089B0006BB141F28020C2F2000003683BB141F28A
:1089C000A421C2F200010B68002B40F08E8641F218
:1089D0009422C2F20002136893B1DBF80430002B3A
:1089E00040F0318641F29426C2F2000640F2B41AF9
:1089F0000023C2F2000A336040F6D863CAF80030A0
:108A000041F2842EC2F2000EDEF80030002B40F05E
:108A1000A38321E098EF00087CE10008B8EF00088C
:108A2000D8EF000890EF0008E4EF0008A004002051
:108A300004F00008B801002018F00008D0F0000889
:108A40000CF1000830F10008F0F100088862002005
:108A5000501300205C61002041F28820C2F2000027
:108A60000368002B00F0708240F2404AC2F2000A14
:108A7000AF4ADAF8003000211160002B00F0648268
:108A800041F2C82EC2F2000EDEF80020B2FBF3F174
:108A900003FB1123002B40F0578240F28C40C2F2BE
:108AA00000000368002B40F0B185D9F80030002B9E
:108AB00000F01F8501F0EEFC9E4B9F4A064616F023
:108AC000010F9E484FEA560118BF1A46FFF78CFC6B
:108AD000FF2E0AD03046FBF773F841F2BC2EC2F2EB
:108AE000000EDEF8003006330893002D40F040827F
:108AF00041F2C025C2F200052B68002B40F07182C4
:108B000041F2702AC2F2000ADAF80030002B40F07D
:108B10007B8241F29C20C2F200000368002B40F0EF
:108B2000868201F089F9FF28054600F08B8200213A
:108B30000A460120FAF7FEFA132D00F2A886DFE8B4
:108B400015F0B901E301D101F0018401B0019601F2
:108B50006A0132011301EA00DD00D000C300A90060
:108B6000B60094007F00A60614007548FFF784FB4A
:108B70007448FFF781FB0126322405960025069EE6
:108B8000DDF81CA016EA0A0F52D1002C3FF4DBAE30
:108B9000013C7FF4D8AE204621462246FAF7CAFAB5
:108BA00015A8FFF7D5F9824600283FF4D3AE00217F
:108BB00001200A46AAF1410AFAF7BCFABAF1330FCA
:108BC00000F21883DFE81AF060044D044804320410
:108BD00016037B04FD0316030B0316031603DC03C5
:108BE00016039D0316038503160316037A03220357
:108BF00016031603D103C603160316031603160342
:108C000016031603160316031603BB03AC036F0308
:108C1000160316031603160316031603160316038C
:108C2000160316031603640316031603160319032B
:108C3000F8F704FB002840F0148501260796A4E706
:108C40004148FFF719FB3F48FFF716FB41F280262A
:108C5000C2F200063368002B40F0CF850025FAF7FA
:108C600003FF32240595022589E73848FFF704FB06
:108C70003448FFF701FB41F28026C2F20006336858
:108C8000002B40F0AB850025FAF7E4FE3224059571
:108C9000022574E72E48FFF7EFFA2A48FFF7ECFAAF
:108CA0000025FAF76DFE32240595022567E729486D
:108CB000FFF7E2FA2348FFF7DFFA0026FAF750FE43
:108CC0003224059602255AE72348FFF7D5FA1D48B6
:108CD000FFF7D2FA0026FAF723FE32240596022582
:108CE0004DE71E48FFF7C8FA1648FFF7C5FA0025FA
:108CF000FAF726FE32240595022540E71848FFF7CB
:108D0000BBFA1048FFF7B8FA0026FAF7E9FD32245B
:108D10000596022533E71348FFF7AEFA0948FFF737
:108D2000ABFA0025FAF7ECFD32240595022526E77B
:108D30008812002074E9000804E1000850F60008D9
:108D4000A0F800087CE1000884F8000868F8000832
:108D500028F8000848F8000804F80008E0F70008C0
:108D6000C0F70008A0F70008B848FFF785FAB84830
:108D7000FFF782FA41F2C823C2F200031A68B54B2A
:108D80003A2A00F2E0841A6801321A6041F27C2427
:108D9000C2F2000400232360D9F80060FEB9322437
:108DA00005960425EBE6AC48FFF766FAA848FFF7FE
:108DB00063FA41F2C821C2F20001A64B0A68002AF8
:108DC00000F0CD841A68013A1A6041F27C22C2F2A6
:108DD0000002D9F8006000231360002EDFD041F2BA
:108DE000A02A41F2C82E41F27C20C2F2000EC2F24B
:108DF0000000C2F2000A0025DAF80010DEF80020B8
:108E000003689648B9607A603B60322401F0F4F957
:108E100005950425B3E69248FFF72EFA8C48FFF734
:108E20002BFA41F2A02EC2F2000E8E4BDEF800208B
:108E3000162A00F28C841A6801321A6041F27C20F2
:108E4000C2F2000000230360A6E78748FFF714FA88
:108E50007F48FFF711FAFAF721FB41F2A826C2F288
:108E600000060025059532243060042587E67F48FA
:108E7000FFF702FA7648FFF7FFF941F2A026C2F2A7
:108E80000006784B3268002A00F065841A68013ABF
:108E90001A6041F27C2AC2F2000A0023CAF80030AC
:108EA0007AE77348FFF7E8F96948FFF7E5F9FAF759
:108EB000E9FAD2E76F48FFF7DFF96548FFF7DCF919
:108EC00040F27413C2F200031D68D5F1010538BFEA
:108ED000002500261D6032240596B5420CBF1425DE
:108EE0000C254CE66448FFF7C7F95948FFF7C4F969
:108EF000FAF78EFA41F27825C2F2000500262860C2
:108F00003224059604253AE65C48FFF7B5F9504847
:108F1000FFF7B2F900240594FBF75CF83224059DB5
:108F20002DE65748FFF7A8F94948FFF7A5F9FAF7E2
:108F30005DFA41F2782AC2F2000A00250595322432
:108F4000CAF8000004251AE6059E002E7FF4A5ADA0
:108F5000089E002E3FF4C9AD41F2BC2AC2F2000ABD
:108F6000DAF80030B342FFF4C0AD059E0425089640
:108F700041F2782A4348C2F2000AFFF77DF93448EB
:108F8000FFF77AF9DAF80030112B40F0BA8240F29C
:108F90008C4EC2F2000EDEF80030002B40F0B5839C
:108FA000D9F80030002B00F0A78301F073FA364B9C
:108FB000364A064616F0010F4FEA5601344818BFEC
:108FC0001A46FFF711FAA6F114012A4641F2C0250C
:108FD000C2F200050020FAF7DDF82B68002B3FF401
:108FE0008FAD40F27416C2F2000641F2702A294B8E
:108FF0003068C2F2000A00221A60FAF745FBDAF87C
:109000000030002B3FF485AD234B41F27C2E002233
:10901000C2F2000E1A60DEF80000FAF775FA41F2AB
:109020009C20C2F200000368002B3FF47AAD1B4B7A
:1090300000221A60F8F77EF900F0FEFEFF280546D0
:109040007FF475AD00260596354698E588F700084B
:109050007CE10008C812002070F700088862002038
:1090600058F70008A012002000F7000840F7000899
:1090700020F70008A0F60008C0F60008B0F60008C7
:10908000E0F6000890F6000874E9000804E1000822
:1090900050F60008C0120020701200209C12002020
:1090A00041F2C42AC2F2000ADAF8003023B9DBF830
:1090B0000430002B40F0FB820126C7480696F8F7E3
:1090C000CBF800283FF460AC012001460022FAF7FB
:1090D00031F8D9F80030002B40F0BF8241F2A02ACD
:1090E000C2F2000ABC68DAF80030BB4A9C4200F0C9
:1090F000D282D2F804E0042540F21000B9693E693A
:10910000D7F800C07A69C2F2000041F2742A50F820
:109110002130F868CDF80CC0C2F2000A8DE8114089
:10912000CAF80010194641F2C82A731C41F2A02661
:10913000C2F20006C2F2000A3460CAF800E041F24E
:109140007C2EC2F2000EA548CEF800C002F26C726E
:10915000FFF74AF9322417E4A14B00221A6041F2CA
:10916000742041F2A022C2F20000C2F2000241F2D9
:10917000C825C2F20005016813682A68994D40F2BB
:109180007416C2F20006C3EB0313306802EB8302CD
:1091900000F096FC002800F0148241F2A02A41F26F
:1091A000C82E2968DFF860C28F48C2F2000AC2F2F6
:1091B000000EDAF80020DEF80030D1F1010E38BFE1
:1091C0004FF0000E8949C5F800E0BEF1000F08BF5E
:1091D00061460CBF14250C25FFF706F93CE48448D2
:1091E000FFF74AF88348FFF747F800F067FE0028CA
:1091F00040F07A813224FFF7ADBB159B40F2B414E6
:10920000C3F56E63C2F2000402332360D9F8003064
:10921000002B40F0018341F2A026C2F20006179C09
:1092200033689C4200F0FC82DDF858E0042540F2EF
:1092300010001B9B189ADDF854C0C2F2000041F2E6
:10924000A02650F82310009241F2C82A41F274225D
:10925000C2F20002C2F20006C2F2000A0194CDF886
:1092600008E0CDF80CC013603460CAF800E041F2A9
:109270007C2E1A9A199B6048C2F2000E02F26C72A0
:109280000133CEF800C03224FFF7AEF8FFF762BB1F
:1092900015A8FAF73DFC594815A9FFF7A5F80425CC
:1092A0003224FFF757BB1598FAF75CF8014654488B
:1092B000FFF79AF804253224FFF74CBBFAF78AFE31
:1092C0005048FEF7D9FF4B48FEF7D6FF3224FFF790
:1092D00041BB40F27410C2F20000159B0268934239
:1092E00088D0404A41491360002B474B474808BF8C
:1092F000194614BF0C2514253224FFF775F8FFF723
:1093000029BB41F29421C2F20001012340480B60C5
:10931000FEF7B2FF3748FEF7AFFF3224FFF71ABB64
:1093200015A8FAF76DFB3B489DF854109DF85520A1
:109330009DF85630FFF758F83224FFF70BBB15980D
:10934000FAF7A4FB34481599FFF74EF802253224AA
:10935000FFF700BB3148FEF78FFF2648FEF78CFF72
:109360003224FAF79FFBFFF7F5BA2D48FEF784FF8A
:1093700001242048FEF780FF05943224FFF7EABA63
:10938000159B002B00F0588241F2802AC2F2000A9D
:1093900024480123CAF80030FEF76EFF1548FEF797
:1093A0006BFF41F28021C2F2000140F2BC12C2F216
:1093B0000002FF23086813603224FAF73FF8FFF732
:1093C000C9BA1598F9F7AAFF17481599FFF70CF8CD
:1093D00004253224FFF7BEBA88620020B0F50008E9
:1093E000841200207401002008F60008DCF8000850
:1093F00004F500087CE10008ACF400083CF5000826
:10940000F4F200081CF50008F0F80008B8F20008B3
:10941000E4F400088CF20008DCF3000890F4000883
:1094200068F3000808F4000868F4000841F27821A5
:10943000C2F2000115980B6898423FF4DBAEF9F7D1
:10944000C7FFCE4A03460146CD4813600425FEF708
:10945000CBFF3224FFF77EBA15A8FAF7ADFAC94858
:1094600062E741F28025C2F200052B68002B40F034
:10947000F0811598FAF7E2FAC3481599FEF7B4FFA0
:1094800002253224FFF766BA41F2A822C2F2000296
:109490001598136898423FF4ADAEF9F7EBFF41F22F
:1094A000C024BA4B0146C2F200041960B848002338
:1094B00023600425FEF798FF3224FFF74BBA41F2F0
:1094C0009826C2F200061598336898423FF492AE8F
:1094D000FAF708F8AF4A03460146AF481360322452
:1094E000FEF782FFFFF736BA00F0E2FD3224FFF705
:1094F00031BAAA48FEF7C0FEA948FEF7BDFEFFF745
:10950000F4BA41F2A02E41F2C822C2F2000EC2F219
:109510000002DEF8000011682A46F9F73BFEFFF76B
:10952000E7BAA048FEF7A8FE01269D48FEF7A4FE74
:109530000696FFF723BADFF884A2504600F0E8FE53
:1095400000283FF42CAA41F2A021C2F20001DAF86F
:1095500008E00B689E4500F00681DAF804C0042597
:1095600040F21006B969F868C2F2000641F27422AE
:1095700056F821307E69CDF808C08DE80140C2F26E
:109580000002386841F2C82A0390116006F26C723A
:1095900041F2A026C2F20006C2F2000AC6F800E0BC
:1095A000CAF800C041F27C2A19463E683B697E48F1
:1095B000C2F2000A0133CAF80060FEF715FFFFF798
:1095C000EEB90425FFF748BA0AA8FEF71BFC0028ED
:1095D0003FF4CBA940F2BC13C2F200030A9A196807
:1095E000531C8B4203D34B1C9A427FF6BEA96F4893
:1095F000FEF7FAFE40F2BC150A9BC2F200051846BF
:109600002B60FAF71BFA0225FFF7AFB941F2B4213C
:10961000C2F2000101230B6001F0D2F841F2B42A3A
:109620000646634B634A644816F0010FC2F2000A13
:1096300018BF1A464FEA56010023CAF80030FEF759
:10964000D3FEFFF745BA002001460122F9F772FD6B
:10965000322401F0ADF9FFF7C5B9584800F0CCFD50
:109660003CE55748FEF708FE4D48FEF705FE41F27F
:10967000C42E4FF0000AC2F2000ECBF804A08BF803
:109680003CA050495048CEF800A0CDF81CA0FBF7F4
:1096900089FAFFF77ABA41F2C82EC2F2000EDEF85C
:1096A0000030D2F804E09E457FF425AD24E5474B19
:1096B00047484FF0010AC3F800A0FEF7DDFD384827
:1096C000FEF7DAFD4349099A0DA801F0CBFE0DA87B
:1096D000FAF71EFA41F2942EC2F2000E0425CEF8DB
:1096E00000A0CDF818A0FFF749B9FEF789FB3A4B67
:1096F00000221A60FFF76BB92848FEF7BDFD284825
:10970000FEF7BAFD6FF013015FE441F2B420C2F23C
:1097100000000123036001F053F841F2B42A064629
:10972000234B244A244816F0010FC2F2000A4FEAE4
:10973000560118BF1A460023CAF80030FEF754FE3F
:10974000A6F1140141E400221A60FFF71FBB0022BA
:109750001A60FFF773BB17221A60FFF79ABB3B2210
:109760001A60FFF732BB41F2C822C2F20002DAF8F7
:1097700004C013689C457FF4F2AEF1E67812002035
:10978000D0F2000860F2000884F30008A81200205C
:1097900018F30008981200203CF3000874F6000843
:1097A0007CE1000884F50008DCF5000858F50008A5
:1097B00074E9000804E1000828F600088862002027
:1097C0000CF2000854F2000848F20008C41200200D
:1097D00094F50008A8F50008A4120020814A40F280
:1097E000BC1A0023C2F2000A18461360FF23CAF80D
:1097F0000030F9F723FEFFF746BA7A4A40F2BC1A66
:109800000023C2F2000A18461360FF23CAF8003092
:10981000F9F714FEFFF722BA15A800F0EDFCFAE400
:1098200041F2C82AC2F2000ADDF858E0DAF8003046
:109830009E457FF4FBACFAE441F2802EC2F2000EAA
:109840006948CEF80030FEF717FD6848FEF714FDB2
:10985000A7E5644A40F2BC160023C2F2000618468F
:109860001360FF233360F9F7E9FD02E66048614CBD
:10987000FEF702FD5D48FEF7FFFCFEF7AABF5E485B
:10988000FEF7FAFC5948FEF7F7FCFEF768BF132D08
:1098900053D801A252F825F0C18E0008158F000898
:1098A000F18E00082F8F0008578E0008AF8E000839
:1098B0007B8E0008238E0008B38D0008758D00088C
:1098C000238D0008098D0008EF8C0008D58C000856
:1098D000A18C0008BB8C0008778C00084D8C000818
:1098E000F7980008778B0008002042490422FAF715
:1098F000B1FDFEF745BF41F2802AC2F2000A40F2F4
:10990000BC1EDAF80030D3F1010338BF0023C2F2E5
:10991000000E1846CAF800300025FF23CEF80030AC
:109920003224F9F78BFD05950225FFF728B9F7F7E3
:109930003BFCFBF769F9FEF7F0BE00240594002517
:109940003224FFF71CB92D48FEF796FC2748FEF796
:1099500093FCFEF7A0BF2A48FEF78EFC2348FEF7D3
:109960008BFC00F05BF8FEF725BF2648FEF784FC71
:109970001E48FEF781FC00F071FB2348FEF77CFCDB
:109980001A48FEF779FC2068FAF78CF91F48FEF7B1
:1099900073FC1648FEF770FC00F076FFFEF702BF7E
:1099A0001B48FEF769FC1148FEF766FCFEF76EBF28
:1099B0001848FEF761FC0D48FEF75EFCFEF761BF3C
:1099C0001548FEF759FC0948FEF756FCFEF754BF50
:1099D000304639460422FAF757FD00287EF447AF97
:1099E000FEF73FBF8012002038F400087CE1000839
:1099F000F8F00008B8010020F4EF0008C4F10008F6
:109A0000ACF000083CF000085CF0000888F00008AA
:109A100098F1000878F1000854F1000830B5104BB7
:109A20001B6887B013B9002007B030BDBF2069465E
:109A30001822FAF70FFD0028F5D00A486A460023DD
:109A40001478517895781C50C1EB01111C1808331B
:109A500005EB81010332402B6160F1D10120E3E786
:109A6000A0040020AC62002070B548F6890686B0DC
:109A7000114C6A460023C8F688061819195940681F
:109A80001170A6FB00514909C1EB0115A0EB85003F
:109A90000833517090700332402BEED1074B186899
:109AA00038B1BF2018226946FAF7EEFC003018BF23
:109AB000012006B070BD00BFAC620020A0040020F1
:109AC000F0B400231B4D02E00833402B22D05C5938
:109AD00014F0800F03EB0506F6D076689642F3D1BA
:109AE000C4F3C20604F0070704F0400418B1D4F12F
:109AF000010438BF0024002CE6D0BE420DD8B1428C
:109B000034BF00260126B94288BF0026002EDBD0D4
:109B1000012000E00020F0BC7047B9428CBF002754
:109B20000127B14234BF3E4647F00106002ECBD09C
:109B3000EEE700BFAC620020704700BF70B54FF485
:109B40004064C4F2020404266420F7F763FE6683CF
:109B50004FF40C70F7F75EFE284D26831420F7F7BC
:109B600059FE00264FF496732B60344603E004B987
:109B70002C682B68ABB14FF440600421C4F20200A2
:109B8000F6F772FED6F1010338BF0023002C08BFA0
:109B900000230028EBD0002BEBD02E682B68002B85
:109BA000E9D13220002E18BF002C0CBF0025012562
:109BB00015D0F7F72FFE4FF440600421C4F20200E5
:109BC000F6F752FE05467820F7F724FE6B1E584242
:109BD000C6EB040458411E2C98BF002070BDF7F757
:109BE00019FE4FF440600421C4F20200F6F73CFE77
:109BF0007820F7F70FFE284670BD00BF586100209F
:109C000038B54FF44064C4F202040425052065838E
:109C1000F7F700FE25830A20F7F7FCFD29462046CA
:109C2000F6F722FE04463220F7F7F4FD621E50429A
:109C3000504138BD70B5082401250026FFF7E0FF2C
:109C40006B0000B12E43013CDDB2F7D1304670BD50
:109C500038B54D1E0446EDB239B101354519FFF74F
:109C6000E9FF04F8010BAC42F9D138BD2DE9F04110
:109C70004FF44066804608250124C4F202060427FA
:109C80000AE00520F7F7C6FD502037836400F7F798
:109C9000C1FD013DE4B20ED0502014EA080F7783D5
:109CA000EFD1F7F7B7FD052037836400F7F7B2FD72
:109CB000013DE4B2F0D1BDE8F08100BF38B54D1EE2
:109CC0000446EDB239B10135451914F8010BFFF71F
:109CD000CDFFAC42F9D138BD10B50446FFF72EFFD9
:109CE000024680B9234603F8012B0133627003F862
:109CF000012B03F8012B03F8012B03F8012B03F8C8
:109D0000012B1A7010BD3320FFF7B0FF2046082149
:109D1000FFF79EFFFFF712FF012010BD70B5124B39
:109D20001A6882B00AB102B070BD012468464FF4CF
:109D300040651C60C4F20205F6F78CFD0820214640
:109D4000F6F736FF042602232846694600968DF86A
:109D500004408DF806408DF807408DF80530F6F781
:109D60001DFD2E83DFE700BFCC12002000B583B0BD
:109D70006846F6F76FFD04200121F6F719FF4FF44E
:109D800080724FF40060002369460092C4F2020022
:109D900001228DF805308DF804208DF806308DF8FD
:109DA0000730F6F7FBFC4FF6B800C0F60000FEF7F0
:109DB00063FA4EF27C10C0F60000FEF75DFA03B0C5
:109DC00000BD00BF10B50B4C2368012B10D04FF421
:109DD00000604FF480710122C4F20200F6F74AFDE0
:109DE0000548FEF749FA0548FEF746FA01232360C5
:109DF00010BD00BFC4010020CCF800087CE10008C1
:109E000010B50A4C236883B14FF400604FF48071A1
:109E10000022C4F20200F6F72DFD0548FEF72CFAE9
:109E20000448FEF729FA0023236010BDC401002076
:109E3000E0F800087CE10008F0B583B06846FDF763
:109E4000D3FC60B31A4A1B4B1068196801301060CC
:109E50009DF8052031B302F001021749BDF80170E9
:109E6000BDF803C01A6000239DF8004018460E4656
:109E700002E00130782B12D0CA5C0633A242F8D13E
:109E800000EB400206EB4202B2F80150BD42F0D1B5
:109E9000B2F80320624503D00130782BECD1FF20CB
:109EA00003B0F0BD12F00102D7D001221A60F6E72C
:109EB000D4120020D0120020D81200202DE9F04F3B
:109EC000DFF894814E4D002783B001263C46C24600
:109ED0002846F9F71DFE2846FEF7CEF94948FEF759
:109EE000CBF96846FDF780FC04EB440908EB49090F
:109EF0000AEB07054846FDF777FC0028FAD06A7997
:109F000012F00102F6D1D4B399F80010134602E022
:109F10000133A34231D018F80200884202F1060250
:109F2000F6D103EB430C0AEB4C0CB9F80100BCF87A
:109F300001E08645ECD1B9F803E0BCF803C0F44574
:109F4000E6D1FF2B19D00022134602E00133A342D1
:109F5000D0D018F802C08C4502F10602F6D103EB0E
:109F6000430C0AEB4C0CBCF801B08345EED1BCF8B5
:109F700003C0F445EAD1002BBCD1142E37D0731E98
:109F8000122B3BD8DFE803F02F2D2B292725232187
:109F90001F1D1B19171513110F0A31001A4D01341B
:109FA0000136063794E7194DF9E7194DF7E7194DD2
:109FB000F5E7194DF3E7194DF1E7194DEFE7194DA5
:109FC000EDE7194DEBE7194DE9E7194DE7E7194DB5
:109FD000E5E7194DE3E7194DE1E7194DDFE7194DC5
:109FE000DDE7194DDBE7194DD9E7194DD7E71948DA
:109FF000F9F78EFD012003B0BDE8F08F004DCEE7EC
:10A0000008F900087CE10008D0FA0008B0FA00085E
:10A0100090FA000874FA000858FA000838FA0008A4
:10A0200018FA0008FCF90008E0F90008CCF900086B
:10A03000B8F90008A4F9000890F9000874F90008BC
:10A0400058F900083CF9000820F9000818F9000840
:10A05000F4F80008ECFA0008D8120020F0B5124B12
:10A06000186883B0E8B10025104F04262C4605225D
:10A0700030466946FAF7EEF99DF800C0BDF80110C8
:10A08000BDF8032007F805C004EB440307EB4303C6
:10A09000013405360635142CA3F80110A3F803206B
:10A0A000E5D103B0F0BD00BFA0040020D81200200D
:10A0B000F0B5114B186883B0E0B100250F4F0426AE
:10A0C0002C4604EB440307EB43037A5DB3F801E04D
:10A0D000B3F803308DF8002030460522694601347C
:10A0E000ADF801E0ADF80330B6180635FAF7CCF953
:10A0F000142CE6D103B0F0BDA0040020D81200203B
:10A1000010B582B004460B460092D02000222146B2
:10A11000FDF710FAD0F1010038BF002002B010BDE9
:10A1200010B582B004460B460092D0200022214692
:10A13000FDF77EFAD0F1010038BF002002B010BD5B
:10A1400030B583B0FDF7A2F93F200DF107010122E0
:10A15000FFF7D6FF054620B301240720244B0DEB63
:10A16000000122461C60FFF7CBFF10B39DF80730BB
:10A17000002B29D100200DF107010122FFF7C0FFBC
:10A180000446B0B19DF807301A0619D503F07F03D5
:10A1900000200DF1070101228DF80730FFF7C0FF05
:10A1A0000EE00E200DF107010122FFF7A9FF044682
:10A1B00018B90024204603B030BD9DF807306BB9B4
:10A1C0000C4B01221A60F5E7072000230DEB00017C
:10A1D00022468DF80730FFF7A3FFCBE70E200DF1E5
:10A1E000070101228DF80750FFF79AFFE8E700BF4B
:10A1F00058130020501300202DE9F04F434B1B68EB
:10A2000089B01BB9184609B0BDE8F08F83680269B0
:10A210000193C36841690293466807688069013207
:10A2200046F26763C6F2666303926439049183FB66
:10A2300006B90199DDF80CB0019A059083FB078AF5
:10A2400083FB0BBC83FB0118DDF810B00299DDF82D
:10A250000CE0D017FD1783FB0121029A009183FBCC
:10A260000BB3DDF810B0C5EBAA05D1174FEAEE72BB
:10A270004FEAEB7E05EB850BC0EBA800F417DDF889
:10A280000080A7EB4B0B019FC4EBA90400EB8009F6
:10A29000C1EBA801A7EB4909029F01EB8108C2EBC2
:10A2A000AC02A7EB4808039F04EB840A02EB820C84
:10A2B000CEEBA303A6EB4A06A7EB4C0C049F06EBE0
:10A2C000041603EB830E059C8DF81960A7EB4E0E68
:10A2D00009EB001908EB01180CEB021C0BEB05173E
:10A2E00001340EEB031E002006A907228DF818701A
:10A2F0008DF81A908DF81B408DF81C808DF81DC0CC
:10A300008DF81EE0FFF70CFF7DE700BF5013002023
:10A310002DE9F04F394B1B688BB004461BB9002068
:10A320000BB0BDE8F08F002008A90722FFF7E8FE78
:10A330000028F4D09DF825A09DF820709DF8268077
:10A340009DF823909DF82430CDF818904FEA1A1B01
:10A350004FEA171C0BEB8B0B4FEA1819CDF81CB00A
:10A360000CEB8C0C9DF82220CDF800C009EB89097C
:10A3700008F00F08DDF81CC005930AF00F0ACDF8AD
:10A380000890CDF804809DF82150DDF81490DDF898
:10A390000480CDF80CA011090AEB4C0ADDF808C0C6
:10A3A00002F00F0201EB81012E091B0909F00F0BCE
:10A3B00002EB410108EB4C09069ADDF8008004939A
:10A3C00005F00F0507F00F0706EB860603EB830386
:10A3D00005EB460602F1FF3C07EB48070BEB430396
:10A3E0000AF1FF3509F1640227606660A160C4F8D4
:10A3F00018C0E3602561626192E700BF501300203E
:10A4000000B50E4B1B6883B053B1FF23C0F20203AB
:10A41000984207D800220120094B1A6003B000BD02
:10A420001846FBE70122DF200DF10701FAF712F8C9
:10A430009DF807200A2A88BF0022EDE7A00400202B
:10A440005413002000B5094B094A1B68106883B0FB
:10A450008DF8073040B1DF2001220DF10701FAF736
:10A4600013F8003018BF012003B000BD54130020C2
:10A47000A004002041F25433C2F200031868704770
:10A4800010B541F25434C2F200042060FFF7DAFF45
:10A49000206810BD00B50D4B1B6883B0FF200BB9C1
:10A4A00003B000BD112001A90222FFF729FE0028F8
:10A4B000F6D09DF80500064B9DF804201B68C0F3FC
:10A4C000400040EA4200C01AEAE700BF50130020F3
:10A4D000541300200649074A074B9A42BEBF51F861
:10A4E000040B42F8040BF8E704488047044800478F
:10A4F000D0FC000800000020A4020020DDA5000818
:10A50000DD0100083349344A002301E041F8043BEF
:10A510009142FBD3FEF7DEF8FEE7FEE7FEE7FEE73B
:10A52000FEE7FEE7FEE7FEE7FEE7FEE7FEE7FEE703
:10A53000FEE7FEE7FEE7FEE7FEE7FEE7FEE7FEE7F3
:10A54000FEE7FEE7FEE7FEE7FEE7FEE7FEE7FEE7E3
:10A55000FEE7FEE7FEE7FEE7FEE7FEE7FEE7FEE7D3
:10A56000FEE7FEE7FEE7FEE7FEE7FEE7FEE7FEE7C3
:10A57000FEE7FEE7FEE7FEE7FEE7FEE7FEE7FEE7B3
:10A58000FEE7FEE7FEE7FEE7FEE7FEE7FEE7FEE7A3
:10A59000FEE7FEE7FEE7FEE7FEE7FEE7FEE7FEE793
:10A5A000FEE7FEE7FEE7FEE7FEE7FEE7FEE7FEE783
:10A5B000FEE7FEE7FEE7FEE7FEE7FEE7FEE7FEE773
:10A5C000FEE7FEE7FEE7FEE7FEE7FEE7FEE7FEE763
:10A5D000FEE70000A4020020F06200204FF46D426C
:10A5E000CEF200024FF46053D2F88810C4F2020396
:10A5F00041F47001C2F888101968002241F001018D
:10A6000019609A60186843F2100120F08470C2F259
:10A61000004120F4803018605960196882B021F43C
:10A6200080211960DA60009201921A6842F4803247
:10A630001A6003E0009AB2F5C06F09D01A6802F4FC
:10A6400000320192009A01320092019A002AF1D060
:10A650004FF46053C4F202031B6813F4003308BFC5
:10A66000019301D001230193019B012B00D0FEE750
:10A670004FF46053C4F202034FF4E042196CC4F289
:10A68000000241F080511964116841F48041116069
:10A690009A6822F0F0029A609A6822F460429A6006
:10A6A0009A6842F480529A601A6822F080721A60A6
:10A6B00019684FF460528801C4F20202F8D445F2DE
:10A6C0000843C0F241735360136843F08073136012
:10A6D00011684FF460538901C4F20203F8D54FF4B6
:10A6E0007052C4F20202116841F4407141F002015B
:10A6F0001160126802F00702022A00D0FEE79A6891
:10A7000022F003029A609A6842F002029A609A6804
:10A7100002F00C02082AFAD14FF46D43CEF2000386
:10A720004FF000629A6002B0704700BF4FF4605370
:10A73000C4F202039A6802F00C02042A14D0082A18
:10A740001CBF4FF41052C0F2F40212D04FF4605309
:10A75000C4F2020318499B68C3F30313CB5C22FACB
:10A7600003F2164B1A6070474FF49052C0F27A020F
:10A77000ECE75868596810F4800F586815BF4FF41B
:10A7800090534FF41053C0F27A03C0F2F40301F077
:10A790003F01B3FBF1F24FF46053C4F20203C0F384
:10A7A00088105B68C3F30143013302FB00F25B00D6
:10A7B000B2FBF3F2CAE700BFC8010020D8010020B5
:10A7C00000B585B001A802A903AAF9F735FD10B9B3
:10A7D000FF2005B000BD029B002BF9D1024B186889
:10A7E000039B181AF5E700BF5C13002000B50E4B61
:10A7F0001B6883B053B1FF23C0F20203984207D80D
:10A8000000220120094B1A6003B000BD1846FBE787
:10A810000122DF200DF10701F9F71CFE9DF807204A
:10A820000A2A88BF0022EDE7A00400205C13002064
:10A8300000B5094B094A1B68106883B08DF80730D2
:10A8400040B1DF2001220DF10701F9F71DFE0030B4
:10A8500018BF012003B000BD5C130020A00400203D
:10A8600041F25C33C2F200031868704710B541F240
:10A870005C34C2F200042060FFF7DAFF206810BDEC
:10A880000920F9F74BBD00BF00B5144B1B6883B01E
:10A890002BB1AA2012491022F9F7DCFD50B9102281
:10A8A0000F48104900F042FE0F4B01221A600020B1
:10A8B00003B000BDBA2001A90222F9F7CBFD0028A0
:10A8C000EDD09DF804109DF80520074B01202D299F
:10A8D0001A60EDD152421A600120E9E7A00400207D
:10A8E000E0010020FCFA0008DC01002000B5134B59
:10A8F0001B68002B83B01ADB2B228DF804208DF807
:10A9000005300F4B1B6813B9002003B000BDAA200F
:10A910000C491022F9F7B8FD0028F5D0BA20022220
:10A9200001A9F9F7B1FD003018BF0120EDE75B4246
:10A930002D228DF804208DF80530E2E7DC0100209F
:10A94000A0040020E001002040F2DC13C2F200036A
:10A950001868704710B5014604460A48FDF744FDE3
:10A9600004F10C03182B0AD8074B1A68A24204D032
:10A970001C60FFF7BBFF012010BD012010BD0020AF
:10A9800010BD00BF0CFB0008DC01002040F2E0100D
:10A99000C2F20000704700BF014608B540F2E01067
:10A9A000C2F2000000F099FDBDE80840FFF79EBF2D
:10A9B00040F2E010C2F20000FAF70CB970B5284A74
:10A9C00048F28013126882B0C7F65543CB1802AE26
:10A9D0004FF4616101FB023346F8043D0546304601
:10A9E00000F038FA0369DA1E052A04460CD9022B56
:10A9F0002BD0092B10D18369C268D21A182A03DD23
:10AA000053B98368022B07DC019B304603F5616371
:10AA1000019300F01FFA044663696B6123692B619F
:10AA2000E36804F10C00EB6007C8013102F26C72BC
:10AA3000F6F756FBA861236A2B62A368AB606368D4
:10AA40006B6023682B6002B070BD8369C268D21A44
:10AA5000182AE1DD002BD7D18368012BD4DCDBE79A
:10AA6000DC01002046F2700048F2200108B5C4F273
:10AA70000200C2F20001F5F749FE60B146F2700033
:10AA800048F22001C4F20200C2F20001F5F76AFEAA
:10AA9000014B00221A6008BD601300202DE9F04729
:10AAA000DFF834E10646DEF80030002BFBD1002E43
:10AAB00000F08A80464D4748770007EB060CAC440F
:10AAC0004FF0FF3415F802AC631C00EB440104F1B5
:10AAD0000909802212EA0A0F0CBF4FF027084FF035
:10AAE0004308013352084B4521F8028FF2D104F19B
:10AAF000080115F803AC00EB410104F111098022B3
:10AB000012EA0A0F0CBF4FF027084FF04308013339
:10AB100052084B4521F8028FF2D104F1100115F8CB
:10AB200001AC00EB410104F11909802212EA0A0F7D
:10AB30000CBF4FF027084FF04308013352084B4534
:10AB400021F8028FF2D1033518346545BAD10022BD
:10AB500000EB4303114699520232602AFBD14FF4B5
:10AB6000806001240021C4F20000CEF80040F6F716
:10AB7000BBF846F270000021C4F20200F5F79AFD1E
:10AB8000BB19DB00303346F270004FF6F871194004
:10AB9000C4F20200F5F798FD46F27000102122463B
:10ABA000C4F20200F5F792FD46F270002146C4F2AD
:10ABB0000200F5F77FFD4FF48060C4F200002146EB
:10ABC000BDE8F047F6F790B8334602483746BEE78F
:10ABD00067130020F417002060130020B0F5C27F37
:10ABE00010B409D80C78054A00EB4000131814542F
:10ABF0004A785A708A789A7010BC704764130020A3
:10AC0000F0B469B10A4D01EB410700230478EC541C
:10AC1000EC184678667086780333BB42A670F5D18F
:10AC20000AB9F0BC70470846F0BCFFF737BF00BF59
:10AC3000641300202DE9F041654D9AB0002401A86D
:10AC40004FF40066C4F202062C60F5F703FE042000
:10AC50000121F5F7ADFF022703234FF040083046EE
:10AC600001A98DF809308DF80870CDF804808DF8B1
:10AC70000A408DF80B40F5F791FD3A460621304623
:10AC8000A6F81A80F5F7FCFD03A8F6F715F806A854
:10AC9000F6F780F838460121F5F798FF4FF40010D9
:10ACA0000121F5F785FF4FF480606A23C4F20000AC
:10ACB00003A90493ADF80C40ADF81440ADF80E4074
:10ACC000F5F7AEFF4FF4806060230126C4F2000068
:10ACD00006A9ADF81830ADF81A600894ADF8244014
:10ACE000F6F710F84FF48060C4F200000821F6F780
:10ACF0005BF84FF48060C4F200003146F5F7E6FFE0
:10AD00004FF48060C4F200003146F6F755F84FF476
:10AD100080604FF400713246C4F20000F6F76AF822
:10AD20000F2268468DF800208DF801408DF8024012
:10AD30008DF80360F5F78CFA0BA8F5F7A9FC46F23D
:10AD400070002146C4F20200F5F7B4FC46F2700030
:10AD5000C4F20200F5F774FB40F23443C4F200037E
:10AD60000C934FF4006312934FF40053139303F5C5
:10AD700095630F934FF4806311934FF44033159311
:10AD80004FF020630B9346F27000124B1494C4F200
:10AD900002000BA91094CDF838800D9316941796E5
:10ADA000189419942746F5F73FFC8DF82C408DF840
:10ADB0002D408DF82E402B68002BFCD10BA840F2C3
:10ADC00085110122FFF71CFF1AB0BDE8F08100BF1A
:10ADD00060130020F417002000210A2200F046BC76
:10ADE00008B5074B044613B10021AFF30080054BB3
:10ADF0001868836A03B19847204601F071F800BFD4
:10AE00000000000024FB000870B50E4B0E4DED1A3B
:10AE1000AD1000241E4603E056F82420904701346C
:10AE2000AC42F9D101F05EF8084D094BED1AAD10B6
:10AE300000241E4603E056F8242090470134AC421B
:10AE4000F9D170BD9C0200209C020020A0020020CD
:10AE50009C02002038B5074B1C68E36B05461BB904
:10AE6000242000F00DF8E063E16B2846BDE838408F
:10AE700000F002B854020020002200F0C3B8000025
:10AE8000024B0146186800F047BA00BF5402002088
:10AE900010B5002302E0CC5CC45401339342FAD1D4
:10AEA00010BD8218034601E003F8011B9342FBD159
:10AEB000704700002DE9F74F064600F09FFF40F273
:10AEC000B1739E42024640F396806FF4F663F31826
:10AED000A6F2B2719B1040F26D1505FB0135A6F28A
:10AEE0006D716FF0630391FBF3F36FF4C861ED18BC
:10AEF00071184FF4C87391FBF3F16D18642196FB40
:10AF0000F1FC01FB1C6C96FBF3F103FB1161D1F129
:10AF10000101466006F0030638BF00210196034692
:10AF2000022407261F7A4A2F11D15F69019805EB89
:10AF3000070810B9BCF1000F00D121B13B2FD4BFDD
:10AF40000027012700E00F464744013F3FE0442F20
:10AF500002D15F69EF193AE0019F37B9BCF1000FE8
:10AF60000CBF89464FF0010900E089462348D3F819
:10AF70000CA04FF0300808FB09090127A84605E09E
:10AF800009EB870B01375BF804BCD8445745F7DB66
:10AF900008F1040797FBF6FB06FB1B7B5F6918694A
:10AFA000BAF1010FB8BF4FF0010A0AF1FF3AB7EB4F
:10AFB0000B0748BF073700F1FF3B072000FB0B776B
:10AFC00059F82A9000E0073F4F45FCDA474498695A
:10AFD000DFF82C8008FB0707186A013C074443F898
:10AFE0001C7F9FD1936BD1699942ACBF0023012391
:10AFF0001360012000E00020BDE8FE8F28FB000860
:10B00000805101002DE9F84380460C46174600F0B8
:10B01000F5FED8F800109B4A91FBF2F3064602FBBE
:10B02000131104E001F5A83101F5C071013B0029BD
:10B03000F8DB4FF4616091FBF0F200FB12113C2051
:10B04000A26091FBF0F200FB1211626021601A1DF8
:10B05000072192FBF1F001FB1022002AB8BF073252
:10B06000002BA26140F2B2754FF4C8704FF0640C2F
:10B07000DFF81C9217DBA90704D195FBFCF20CFB4F
:10B08000125242B995FBF0F100FB1151D1F10101CF
:10B0900038BF002100E0012159F82120934218DB3C
:10B0A00001359B1AE7E7013DAA0704D195FBFCF2A5
:10B0B0000CFB125242B995FBF0F100FB1151D1F19A
:10B0C000010138BF002100E0012159F821209B181F
:10B0D000E9D4A5F26C7262616B4AE3614FF030090A
:10B0E00009FB01290022226102E001319B1A216142
:10B0F000216959F821209342F7DA0133E360002FE8
:10B1000040F0BA8000F0A6FC604B1B681BB373686C
:10B110009D4205D13168D8F80030F26931B90CE0B0
:10B120002846FFF7C7FE0028F4D110E093420CDB5D
:10B13000B26B934209DA01230BE09342FBDAB26B64
:10B140009342ACBF0023012303E0002301E04FF052
:10B15000FF33236200E02762236A2568012B0CBFBE
:10B16000F36B336A4FF4616093FBF0F200FB123330
:10B170003C2093FBF0F100FB11336068411AA0689A
:10B180006160EB1A821A3B2B2360A26003DD013160
:10B1900061603C3B04E0002B03DA013961603C3321
:10B1A000236063683B2B03DD0132A2603C3B04E07B
:10B1B000002B03DA013AA2603C336360A368172BCB
:10B1C0001FDDE2690132E261A2690132062AC8BFCD
:10B1D0000022A261E268183B0132A3602369E260A9
:10B1E00059F823108A4244DD0133521A0C2BE260D5
:10B1F00023613ED162690023013223616261E36110
:10B2000037E0002B35DAE269013AE261A269013ADE
:10B2100048BF0622A261E2681833013AE260A360E7
:10B220003ABB2369013B01D423611EE00B23236158
:10B2300063695A1E12F0030F626103F26B7305D14A
:10B24000642293FBF2F102FB113252B94FF4C8723F
:10B2500093FBF2F102FB1133D3F1010338BF00235A
:10B2600000E0012303F5B673E361236959F8233045
:10B27000E36000F0F0FB01E0002323622046BDE81C
:10B28000F88300BF8051010028FB00084C610020BA
:10B2900088FB000830B500293BD051F8042C0B1F67
:10B2A0001C49002AB8BF9B180A6812B95A600B6083
:10B2B00030BD93420CD219685818904203D15A58A5
:10B2C0008918426819605A60124A136030BD0A46F4
:10B2D000516809B19942FAD9146815199D420AD1E9
:10B2E0001B68E318D0188842136012D108681B1835
:10B2F00013604B680CE002D90C23036030BD186862
:10B300001C188C4203D10C684968001918605960F8
:10B31000536030BD48610020F8B5CD1C25F0030511
:10B3200008350C2D38BF0C25002D064645DB8D4217
:10B3300000D242E0234B1B681C4612E02268521BDD
:10B340000DD40B2A02D92260A4181EE0A34203D117
:10B3500063681C4A136021E062685A601EE023465D
:10B360006468002CEAD123E03046214600F06AF8F8
:10B3700038602946304600F065F8431C01461CD071
:10B38000C41C24F00304844201D1256006E0304649
:10B39000611A00F057F80130F7D10EE004F10B000C
:10B3A000231D20F00700C31A0AD05A42E250F8BD0C
:10B3B000054F3B68002BDCD1D6E70C23336000201F
:10B3C000F8BD00BF48610020446100201A4B10B551
:10B3D0001C68A36BD3B91820FFF752FD43F20E335C
:10B3E000A06303804AF6CD33438041F23423838047
:10B3F0004EF26D63C3804DF6EC63038105234381F8
:10B400000B23838101220023C0E90423A46B0B4991
:10B41000206962690A4B414303FB0212A0FB03014E
:10B42000511801220023121843EB0103C4E904233D
:10B4300023F0004010BD00BF540200202DF45158ED
:10B440002D7F954C38B5064C0023054608462360F1
:10B4500000F02CFD431C02D1236803B12B6038BDE2
:10B46000EC6200200EB400B59CB04FF40271ADF850
:10B4700014106FF000411DAB049107914FF6FF715E
:10B48000ADF81610084953F8042B0290069008688E
:10B49000019302A900F0E6F9029B00221A701CB089
:10B4A0005DF804EB03B0704754020020C9B20346B4
:10B4B00010F8012B12B18A42F9D102E0002918BF1D
:10B4C00000231846704710F8012B11F8013B012AA0
:10B4D00028BF9A42F7D0D01A7047034611F8012BC3
:10B4E00003F8012B002AF9D17047034613F8012B0A
:10B4F000002AFBD1181A0138704770B5A2B108E0D4
:10B50000012A03D128781B78C01A70BD013A002C9B
:10B51000F8D00B460546002AF4D010F8016B1C78D1
:10B520000131B442ECD0EDE7104670BD30B50139C1
:10B53000034609E011F8015F03F8015B013A1C467C
:10B5400015B99B18002205E01C46002AF2D1F8E745
:10B5500004F8012B9C42FBD130BD00002DE9F74FD0
:10B5600001904148D0F800900846044614F8015B69
:10B5700009EB05062046777807F00807FFB2002F91
:10B58000F3D12D2D03D114F8015B012704E02B2DFD
:10B5900004BF244614F8015B002B5ED0102B08D1A9
:10B5A00058E02078782801D058284ED165781023AB
:10B5B0000234002F0CBF6FF000404FF00040B0FB92
:10B5C000F3FA002603FB1A08304609EB050C9CF839
:10B5D00001C00CF0040B5FFA8BFBBBF1000F01D034
:10B5E000303D0BE01CF0030C1BD0BCF1010F14BF6D
:10B5F0004FF0570C4FF0370CCCEB05059D4210DA9D
:10B60000B6F1FF3F0AD0504506D801D1454503DCCD
:10B6100003FB0050012601E04FF0FF3614F8015BF8
:10B62000D3E7731C0AD1002F01990CBF6FF00040C3
:10B630004FF0004022230B6022B912E007B14042D4
:10B640007AB106B1611E11600BE03025002BB0D13C
:10B650000823AEE7302DACD1A3E7302DA1D00A23CB
:10B66000A7E7BDE8FE8F00BF5802002030B51346A3
:10B67000044A05460C46106829462246BDE830407B
:10B68000FFF76CBF540200202DE9F74F01903D48B1
:10B69000D0F800900846044614F8015B09EB050653
:10B6A0002046777807F00807FFB2002FF3D12D2D41
:10B6B00003D114F8015B012704E02B2D04BF2446BD
:10B6C00014F8015B002B57D0102B08D151E02078E3
:10B6D000782801D0582847D16578102302344FF0DC
:10B6E000FF3ABAFBF3FA03FB0AF000266FEA000800
:10B6F000304609EB050C9CF801C00CF0040B5FFA16
:10B700008BFBBBF1000F01D0303D0BE01CF0030CB4
:10B710001BD0BCF1010F14BF4FF0570C4FF0370C8A
:10B72000CCEB05059D4210DAB6F1FF3F0AD050453B
:10B7300006D801D1454503DC03FB0050012601E09A
:10B740004FF0FF3614F8015BD3E7731C05D1019964
:10B7500022230B60304622B912E007B140427AB191
:10B7600006B1611E11600BE03025002BB7D1082314
:10B77000B5E7302DB3D1AAE7302DA8D00A23AEE724
:10B78000BDE8FE8F5802002030B51346044A054636
:10B790000C46106829462246BDE83040FFF774BFCA
:10B7A000540200202DE9F0478D68AB4281460C46DB
:10B7B00092461F463FD38A8912F4906F39D026688B
:10B7C00009696369C1EB060803265E43022508F197
:10B7D000010302F4806296FBF5F6DB1912B29E4279
:10B7E00038BF1E4682B13146FFF796FD054600B9C7
:10B7F00013E021694246FFF74BFBA38923F49063D2
:10B8000043F08003A3810CE0324600F022FB0546A2
:10B8100038B948462169FFF73DFD0C23C9F80030CF
:10B8200018E0256166614544C8EB06062560A66000
:10B830003D46AF4200D23D462A462068514600F0C0
:10B84000EFFAA3685B1BA36023685D1925600020E5
:10B85000BDE8F087A38943F04003A3814FF0FF3098
:10B86000BDE8F0872DE9F04F9DB0064603938B8924
:10B8700003F080031BB20D46144663B10B6953B944
:10B880004021FFF749FD2860286110B90C2333607F
:10B89000D0E040236B610023099320238DF82930E9
:10B8A000DFF89C81DFF89C9130238DF82A30234605
:10B8B0009A4613F8012B1AB9BAEB040B0FD002E029
:10B8C000252AF5D1F8E73046294622465B46FFF7A0
:10B8D00069FF013000F0A780099B5B4409939AF847
:10B8E0000030002B00F09F8000234FF0FF320493C4
:10B8F0000793059206938DF853301A930AF1010AC3
:10B900004FF0010B05E0C8EB00000BFA00F0034319
:10B91000049354464A482178052200F073FA0AF14C
:10B92000010A049B0028EED1D90602D520228DF809
:10B9300053201A0702D52B228DF8532022782A2A69
:10B9400003D0079B21460A2010E0039A111D1268BC
:10B950000391002A01DB079204E0524243F0020304
:10B9600007920493013408E000FB03230C460131E5
:10B970002278303A092AF7D9079323782E2B19D148
:10B9800063782A2B09D1039B1A1D1B68039202348A
:10B99000002BB8BF4FF0FF330BE0611C00230A20DF
:10B9A00001E000FB03230C4601312278303A092ADA
:10B9B000F7D9059323482178032200F023FA40B1F8
:10B9C0004023C9EB000003FA00F0049B03430493F7
:10B9D000013414F8011B1C488DF82810062200F0D1
:10B9E00011FA88B1194B33B9039B073323F00703CE
:10B9F0000833039313E003AB0093304604A92A46AF
:10BA0000134BAFF3008007E003AB0093304604A96B
:10BA10002A460F4B00F092F8431C074603D0099BBF
:10BA2000DB19099343E7AB8903F040031BB20BB961
:10BA3000099801E04FF0FF301DB0BDE8F08F00BF66
:10BA400090FB000896FB00089AFB0008000000002D
:10BA5000A5B70008704770472DE9F04715461F4607
:10BA60008A680B69DDF820809A42A8BF13462B60D4
:10BA700091F8432006460C460AB101332B60236837
:10BA8000990602D52B6802332B60236813F0060950
:10BA900016D094F843302268003318BF0123920671
:10BAA00016D41EE00123304639465246C0470130C5
:10BAB00003D14FF0FF30BDE8F08709F1010901E043
:10BAC00004F1190AE1682B68CB1A9945EADBE0E733
:10BAD000E218302182F8431094F84510023382F8BE
:10BAE00044103046394604F14302C0470130E0D0EB
:10BAF00023682A68E16803F00603042B08BFC2EB41
:10BB000001052369A2680CBF25EAE57500259A4264
:10BB1000C4BFC3EB0203ED184FF000091A3408E06C
:10BB20000123304639462246C0470130C1D009F1D1
:10BB30000109A945F4DB0020BDE8F0872DE9FF47A6
:10BB40000E7E0C9D6E2E914680460C469A4601F163
:10BB5000430200F0AF800FD8632E1DD006D8002E10
:10BB600000F0C080582E40F0D0804FE0642E1CD0F2
:10BB7000692E40F0CA8018E0732E00F0B78005D817
:10BB80006F2E2BD0702E40F0C08043E0752E25D054
:10BB9000782E40F0BA8041E02B681A1D1B682A609D
:10BBA00001F1420781F84230B3E021682B6811F0BF
:10BBB000800F02D0191D296008E011F0400F03F139
:10BBC0000401296002D0B3F9005000E01D68002D87
:10BBD00045DA2D236D4284F8433040E021682B681C
:10BBE00011F0800F02D0191D296007E011F0400FFD
:10BBF00003F10401296001D01D8800E01D68237E47
:10BC00005F486F2B14BF0A23082324E081F84560A6
:10BC10005B4807E00B6843F020030B60782359482A
:10BC200084F8453021682B6811F0800F03F1040679
:10BC30002E6000D003E04F0601D51D8800E01D688E
:10BC4000CE0744BF41F0200121601DB9236823F0D5
:10BC5000200323601023002184F8431001E04848AA
:10BC60000A236668002EA66003DB216821F0040128
:10BC7000216005B96EB104F14201B5FBF3F603FB97
:10BC800016550F46455D01F801593546002EF4D191
:10BC900000E01746082B0AD12368DB0707D5616847
:10BCA0002369994203DC302307F8013C013FD21B92
:10BCB000226133E009682B6811F0800F05D0191D4F
:10BCC0002960196863690B600CE011F0400F03F103
:10BCD0000401296003D0196863690B8002E061697F
:10BCE0001B68196000232361174617E02B681A1D93
:10BCF0002A601F683846FFF7F8FB636820619842A6
:10BD000088BF23612369636005E004F1420784F87A
:10BD1000426001232361002384F84330CDF800A062
:10BD20004046214603AA4B46FFF796FE013002D15A
:10BD30004FF0FF3021E0404649463A462369D0475C
:10BD40000130F5D0236898070ED4E068039B984231
:10BD5000B8BF184611E00123404649463246D04755
:10BD60000130E5D0013502E0002504F11906E16853
:10BD7000039BCB1A9D42EEDBE7E704B0BDE8F087FA
:10BD8000A1FB0008B2FB000830B5141E9BB00546AD
:10BD900004DA8B2303604FF0FF301DE04FF4027292
:10BDA000ADF80C200091049101D0611E00E0214605
:10BDB0004FF6FF7202910591ADF80E2028461A4603
:10BDC00069461E9BFFF74EFD431C01DA8B232B6057
:10BDD00014B1009B00221A701BB030BD73B50093E4
:10BDE000054B06460D461446186831462A4623463A
:10BDF000FFF7CAFF7CBD00BF540200200048704717
:10BE00005C02002010B5C9B20346821803E0047832
:10BE100001338C4203D093421846F8D1002010BD64
:10BE2000814210B511D28C18A0420ED25342811813
:10BE3000E418CB1801E0A15C995412F1FF32FAD258
:10BE400010BDCC5CC454013300E000239342F8D110
:10BE500010BDF8B5064615460C4621B91146BDE899
:10BE6000F840FFF759BA1AB9FFF714FA2C4612E056
:10BE700000F013F8A8420ED230462946FFF74CFADC
:10BE8000074638B121462A46FFF702F830462146D8
:10BE9000FFF700FA3C462046F8BD51F8040C002894
:10BEA00002DA04390B58C01804387047094A13687D
:10BEB00063B118186946884298BF106004D9064BD0
:10BEC0000C221A604FF0FF3318467047034B136083
:10BED000EFE700BF50610020EC620020F06200201C
:10BEE000FEE700BFF8B500BFF8BC08BC9E4670472F
:10BEF000F8B500BFF8BC08BC9E4670476561737416
:10BF0000657220646174653A20253034642D2530D3
:10BF100032642D253032640D0A000000536F00009A
:10BF20004D6F0000446900004D690000446F00003F
:10BF30004672000053610000537500005475000004
:10BF40005765000054680000444346373720457267
:10BF5000726F723A20486967682070756C7365204B
:10BF60003C3D2035000000004443463737204572F1
:10BF7000726F723A20486967682070756C7365202B
:10BF80003E3D20323500000044434637372045729D
:10BF9000726F723A20706172697479205031206931
:10BFA0006E636F727265637400000000444346372D
:10BFB00037204572726F723A20706172697479200D
:10BFC000503220696E636F72726563740000000006
:10BFD0004443463737204572726F723A207061725F
:10BFE00069747920503320696E636F72726563746F
:10BFF0000000000000000000000000003C42423C45
:10C0000000000000241824427E42420024003C42EA
:10C0100042423C002400424242423C007C427C427C
:10C020007C40400000000000000000000000000014
:10C030000000000000000000000000000000000000
:10C0400000000000000000000000000000000000F0
:10C0500000000000000000000000000000000000E0
:10C0600000000000000000000000000000000000D0
:10C0700000000000000000000000000000000000C0
:10C0800000000000000000000000000000000000B0
:10C0900000000000000000000000000000000000A0
:10C0A0000000000000000000000000000000000090
:10C0B0000000000000000000000000000000000080
:10C0C0000000000000000000000000000000000070
:10C0D0000000000000000000000000000000000060
:10C0E0000000000000000000000000000000000050
:10C0F0000000000000000000000000003838381088
:10C1000000383800EEEE4400000000002828FE2829
:10C11000FE2828007C92907C12927C00E2A4E81019
:10C120002E4A8E00304830708A847A0038381020C9
:10C13000000000001820404040201800300804048F
:10C1400004083000004428EE284400000010107C51
:10C150001010000000000038381020000000007CA3
:10C160000000000000000000383838000204081009
:10C17000204080003844A2928A4438001030501089
:10C1800010107C007C82027C8080FE007C82027C1D
:10C1900002827C00808484FE04040400FE80807C93
:10C1A00002827C007C8280FC82827C00FE840810FB
:10C1B000202020007C82827C82827C007C82827EA5
:10C1C00002827C0010281000102810003838003837
:10C1D00038102000081020402010080000007C00CB
:10C1E0007C00000020100804081020007C82020C53
:10C1F000100010007C82BAAABC827C001028448205
:10C20000FE828200FC8282FC8282FC007C82808032
:10C2100080827C00FC8282828282FC00FE8080F828
:10C220008080FE00FE8080F8808080007C82809E7E
:10C2300082827C00828282FE82828200381010100C
:10C24000101038000202020282827C00848890E092
:10C2500090888400808080808080FE0082C6AA92C0
:10C260008282820082C2A2928A8682007C8282823C
:10C2700082827C00FC8282FC808080007C828282C0
:10C280008A847A00FC8282FC888482007C82807CA2
:10C2900002827C00FE101010101010008282828238
:10C2A00082827C0082828282442810008292929252
:10C2B00092926C0082442810284482008244281004
:10C2C00010101000FE0408102040FE007C4040408A
:10C2D00040407C0080402010080402007C040404DC
:10C2E00004047C001028440000000000000000004E
:10C2F0000000FE003838100800000000001824423A
:10C300007E424200007C427C42427C00003C424033
:10C3100040423C00007C424242427C00007E407C25
:10C3200040407E00007E407C40404000003C424057
:10C330004E423C000042427E424242000008080851
:10C34000080808000002020202423C000042447851
:10C35000484442000040404040407E000042665A4F
:10C3600042424200004262524A464200003C42427F
:10C3700042423C00007C42427C404000003C424241
:10C380004A443A00007C42427C444200003C403C2B
:10C3900002423C00003E08080808080000424242F1
:10C3A00042423C00004242424224180000424242C3
:10C3B0005A66420000422418182442000022140841
:10C3C00008080800007E040810207E00384040C0A5
:10C3D00040403800101010001010100038040406FF
:10C3E0000404380060920C0000000000000000000F
:10C3F0000000000000000100010002000200030034
:10C400000300040004000500050006000700080002
:10C4100009000B000D000E001000120014001700A0
:10C4200019001C001F002100240028002B002E00F2
:10C430003200360039003D00420046004A004F00FD
:10C44000540059005E00630069006E0074007A00B9
:10C45000800086008C0093009900A000A700AE0029
:10C46000B600BD00C500CD00D500DD00E500EE0042
:10C47000F600FF004E6F6E65000000005261696EAD
:10C48000626F77004661646500000000526F6C6C5B
:10C49000000000004578706C6F64650052616E6446
:10C4A0006F6D0000536E616B6500000054656C6534
:10C4B000747970650000000043756265000000003B
:10C4C0004D6174726978000044726F700000000062
:10C4D00053717565657A65004E6F726D616C000011
:10C4E000436C6F636B320000080809090A0A0B0BE2
:10C4F0000C0C0D0D0E0E0F000000000000000000DF
:10C5000000052200000000000015220000000000CD
:10C5100000072200000000000012220000000000BE
:10C520000010220000000000000C220000000000AB
:10C53000000E220000000000001322000000000096
:10C54000001122000000000000172200000000007F
:10C55000000F220000000000001622000000000072
:10C560000007172200000000001217220000000040
:10C570000010172200000000000B1722000000002E
:10C58000000D172200000000001317220000000019
:10C590000011172200000000001922000000000016
:10C5A00000041819220000000015181922000000CC
:10C5B00000071819220000000012181922000000BC
:10C5C0000010181922000000000C181922000000A9
:10C5D000000E181922000000001318192200000094
:10C5E0000011181922000000001B220000000000AA
:10C5F0000004181B220000000015181B2200000078
:10C600000007181B220000000012181B2200000067
:10C610000010181B22000000000C181B2200000054
:10C62000000E181B220000000013181B220000003F
:10C630000011181B22000000001A22000000000058
:10C640000004181A220000000015181A2200000029
:10C650000007181A220000000012181A2200000019
:10C660000010181A22000000000C181A2200000006
:10C67000000E181A220000000013181A22000000F1
:10C680000011181A22000000001C22000000000007
:10C690000004181C220000000015181C22000000D5
:10C6A0000007181C220000000012181C22000000C5
:10C6B0000010181C22000000000C181C22000000B2
:10C6C000000E181C220000000013181C220000009D
:10C6D0000011181C220000000000000000000000F3
:10C6E00000091E220000000000151F2200000000AB
:10C6F00000071F220000000000121F22000000009F
:10C7000000101F2200000000000C1F22000000008B
:10C71000000E1F220000000000131F220000000076
:10C7200000111F220000000000171F22000000005F
:10C73000000F1F220000000000161F220000000052
:10C740000007171F220000000012171F2200000020
:10C750000010171F22000000000B171F220000000E
:10C76000000D171F220000000013171F22000000F9
:10C770000011171F2200000000191F2200000000F6
:10C78000000418191F220000001518191F220000AC
:10C79000000718191F220000001218191F2200009C
:10C7A000001018191F220000000C18191F22000089
:10C7B000000E18191F220000001318191F22000074
:10C7C000001118191F220000001B1F22000000008A
:10C7D0000004181B1F2200000015181B1F22000058
:10C7E0000007181B1F2200000012181B1F22000048
:10C7F0000010181B1F220000000C181B1F22000035
:10C80000000E181B1F2200000013181B1F2200001F
:10C810000011181B1F220000001A1F220000000038
:10C820000004181A1F2200000015181A1F22000009
:10C830000007181A1F2200000012181A1F220000F9
:10C840000010181A1F220000000C181A1F220000E6
:10C85000000E181A1F2200000013181A1F220000D1
:10C860000011181A1F220000001C1F2200000000E7
:10C870000004181C1F2200000015181C1F220000B5
:10C880000007181C1F2200000012181C1F220000A5
:10C890000010181C1F220000000C181C1F22000092
:10C8A000000E181C1F2200000013181C1F2200007D
:10C8B0000011181C1F2200000041000000000000B1
:10C8C00000091E220000000000151F2200000000C9
:10C8D00000071F220000000000121F2200000000BD
:10C8E00000101F2200000000000C1F2200000000AA
:10C8F000000E1F220000000000131F220000000095
:10C9000000111F220000000000171F22000000007D
:10C91000000F1F220000000000161F220000000070
:10C920000007171F220000000012171F220000003E
:10C930000103000000000000000B171F2200000090
:10C94000000D171F220000000013171F2200000017
:10C950000011171F2200000001171F2026000000F1
:10C9600001111F202600000001131F2026000000D7
:10C97000010E1F2026000000010C1F2026000000D1
:10C9800001101F202600000001121F2026000000B9
:10C9900001071F202600000001151F2026000000AF
:10C9A00001091F20260000000126000000000000F1
:10C9B00001091E222600000001151F22260000008A
:10C9C00001071F222600000001121F22260000007E
:10C9D00001101F2226000000010C1F22260000006B
:10C9E000010E1F222600000001131F222600000056
:10C9F00001111F222600000001171F22260000003F
:10CA0000010F1F222600000001161F222600000031
:10CA10000107171F222600000112171F22260000FF
:10CA200001240000000000000112171F2000000078
:10CA30000107171F2000000001161F200000000042
:10CA4000010F1F200000000001171F200000000040
:10CA500001111F200000000001131F200000000032
:10CA6000010E1F2000000000010C1F20000000002C
:10CA700001101F200000000001121F200000000014
:10CA800001071F200000000001151F20000000000A
:10CA900001091E200000000000410000000000000D
:10CAA00000091E220000000000151F2200000000E7
:10CAB00000071F220000000000121F2200000000DB
:10CAC00000101F2200000000000C1F2200000000C8
:10CAD000000E1F220000000000131F2200000000B3
:10CAE00000111F220000000000171F22000000009C
:10CAF000000F1F220000000000161F22000000008F
:10CB00000007171F220000000012171F220000005C
:10CB10000003220000000000000B171F220000008D
:10CB2000000D171F220000000013171F2200000035
:10CB30000011171F2200000000191F220000000032
:10CB400001111F202600000001131F2026000000F5
:10CB5000010E1F2026000000010C1F2026000000EF
:10CB600001101F202600000001121F2026000000D7
:10CB700001071F202600000001151F2026000000CD
:10CB800001091E2026000000012600000000000010
:10CB900001091E222600000001151F2226000000A8
:10CBA00001071F222600000001121F22260000009C
:10CBB00001101F2226000000010C1F222600000089
:10CBC000010E1F222600000001131F222600000074
:10CBD00001111F222600000001191F200000000083
:10CBE0000111171F200000000113171F2000000073
:10CBF000010D171F20000000010B171F200000006F
:10CC000001240000000000000112171F2000000096
:10CC10000107171F2000000001161F200000000060
:10CC2000010F1F200000000001171F20000000005E
:10CC300001111F200000000001131F200000000050
:10CC4000010E1F2000000000010C1F20000000004A
:10CC500001101F200000000001121F200000000032
:10CC600001071F200000000001151F200000000028
:10CC700001091E200000000000410000000000002B
:10CC800000091E220000000000151F220000000005
:10CC900000071F220000000000121F2200000000F9
:10CCA00000101F2200000000000C1F2200000000E6
:10CCB000000E1F220000000000131F2200000000D1
:10CCC00000111F220000000000171F2200000000BA
:10CCD000000F1F220000000000161F2200000000AD
:10CCE0000007171F220000000012171F220000007B
:10CCF0000003220000000000000B171F22000000AC
:10CD0000000D171F220000000013171F2200000053
:10CD10000011171F2200000000191F220000000050
:10CD200001111F202600000001131F202600000013
:10CD3000010E1F2026000000010C1F20260000000D
:10CD400001101F202600000001121F2026000000F5
:10CD500001071F202600000001151F2026000000EB
:10CD600001091E202600000001260000000000002E
:10CD700001091E222600000001151F2226000000C6
:10CD800001071F222600000001121F2226000000BA
:10CD900001101F2226000000010C1F2226000000A7
:10CDA000010E1F222600000001131F222600000092
:10CDB00001111F222600000001191F2000000000A1
:10CDC0000111171F200000000113171F2000000091
:10CDD000010D171F20000000010B171F200000008D
:10CDE00001032000000000000112171F20000000B6
:10CDF0000107171F2000000001161F20000000007F
:10CE0000010F1F200000000001171F20000000007C
:10CE100001111F200000000001131F20000000006E
:10CE2000010E1F2000000000010C1F200000000068
:10CE300001101F200000000001121F200000000050
:10CE400001071F200000000001151F200000000046
:10CE500001091E2000000000004100000000000049
:10CE600000091E220000000000151F220000000023
:10CE700000071F220000000000121F220000000017
:10CE800000101F2200000000000C1F220000000004
:10CE9000000E1F220000000000131F2200000000EF
:10CEA00000111F220000000000171F2200000000D8
:10CEB000000F1F220000000000161F2200000000CB
:10CEC0000007171F220000000012171F2200000099
:10CED0000103000000000000000B171F22000000EB
:10CEE000000D171F220000000013171F2200000072
:10CEF0000011171F2200000000191F22000000006F
:10CF000001111F202600000001131F202600000031
:10CF1000010E1F2026000000010C1F20260000002B
:10CF200001101F202600000001121F202600000013
:10CF300001071F202600000001151F202600000009
:10CF400001091E202600000001260000000000004C
:10CF500001091E222600000001151F2226000000E4
:10CF600001071F222600000001121F2226000000D8
:10CF700001101F2226000000010C1F2226000000C5
:10CF8000010E1F222600000001131F2226000000B0
:10CF900001111F222600000001191F2000000000BF
:10CFA0000111171F200000000113171F20000000AF
:10CFB000010D171F20000000010B171F20000000AB
:10CFC00001240000000000000112171F20000000D3
:10CFD0000107171F2000000001161F20000000009D
:10CFE000010F1F200000000001171F20000000009B
:10CFF00001111F200000000001131F20000000008D
:10D00000010E1F2000000000010C1F200000000086
:10D0100001101F200000000001121F20000000006E
:10D0200001071F200000000001151F200000000064
:10D0300001091E2000000000004100000000000067
:10D0400000091E220000000000151F220000000041
:10D0500000071F220000000000121F220000000035
:10D0600000101F2200000000000C1F220000000022
:10D07000000E1F220000000000131F22000000000D
:10D0800000111F220000000000171F2200000000F6
:10D09000000F1F220000000000161F2200000000E9
:10D0A0000007171F220000000012171F22000000B7
:10D0B0000003220000000000000B171F22000000E8
:10D0C000000D171F220000000013171F2200000090
:10D0D0000011171F2200000001171F20260000006A
:10D0E00001111F202600000001131F202600000050
:10D0F000010E1F2026000000010C1F20260000004A
:10D1000001101F202600000001121F202600000031
:10D1100001071F202600000001151F202600000027
:10D1200001091E202600000001260000000000006A
:10D1300001091E222600000001151F222600000002
:10D1400001071F222600000001121F2226000000F6
:10D1500001101F2226000000010C1F2226000000E3
:10D16000010E1F222600000001131F2226000000CE
:10D1700001111F222600000001171F2226000000B7
:10D18000010F1F222600000001161F2226000000AA
:10D190000107171F222600000112171F2226000078
:10D1A00001032000000000000112171F20000000F2
:10D1B0000107171F2000000001161F2000000000BB
:10D1C000010F1F200000000001171F2000000000B9
:10D1D00001111F200000000001131F2000000000AB
:10D1E000010E1F2000000000010C1F2000000000A5
:10D1F00001101F200000000001121F20000000008D
:10D2000001071F200000000001151F200000000082
:10D2100001091E20000000000000000000000000C6
:10D220000035000000000000002B0000000000009E
:10D230000033000000000000003200000000000089
:10D24000002E000000000000003000000000000080
:10D250000028000000000000003100000000000075
:10D26000002900000000000000380000000000005D
:10D270000037000000000000003D0000000000003A
:10D2800000333800000000000032380000000000C9
:10D29000002E380000000000002F380000000000C1
:10D2A00000273800000000000031380000000000B6
:10D2B00000293800000000000039000000000000D4
:10D2C000002C363900000000002B36390000000029
:10D2D000003336390000000000323639000000000B
:10D2E000002E363900000000003036390000000002
:10D2F00000283639000000000031363900000000F7
:10D300000029363900000000003B0000000000004A
:10D31000002C363B00000000002B363B00000000D4
:10D320000033363B000000000032363B00000000B6
:10D33000002E363B000000000030363B00000000AD
:10D340000028363B000000000031363B00000000A2
:10D350000029363B00000000003C000000000000F7
:10D36000002C363C00000000002B363C0000000082
:10D370000033363C000000000032363C0000000064
:10D38000002E363C000000000030363C000000005B
:10D390000028363C000000000031363C0000000050
:10D3A0000029363C00000000003E000000000000A4
:10D3B000002C363E00000000002B363E000000002E
:10D3C0000033363E000000000032363E0000000010
:10D3D000002E363E000000000030363E0000000007
:10D3E0000028363E000000000031363E00000000FC
:10D3F0000029363E00000000000000000000000090
:10D4000000212D3F0000000000212B400000000003
:10D4100000213340000000000021324000000000E5
:10D4200000212E40000000000021304000000000DC
:10D4300000212840000000000021314000000000D1
:10D4400000212940000000000021384000000000B9
:10D45000002137400000000000213D400000000096
:10D460000021333840000000002132384000000025
:10D4700000212E384000000000212F38400000001D
:10D480000021273840000000002131384000000012
:10D490000021293840000000002139400000000030
:10D4A00000212C363940000000212B363940000085
:10D4B0000021333639400000002132363940000067
:10D4C00000212E363940000000213036394000005E
:10D4D0000021283639400000002131363940000053
:10D4E000002129363940000000213B4000000000A7
:10D4F00000212C363B40000000212B363B40000031
:10D50000002133363B400000002132363B40000012
:10D5100000212E363B400000002130363B40000009
:10D52000002128363B400000002131363B400000FE
:10D53000002129363B40000000213C400000000053
:10D5400000212C363C40000000212B363C400000DE
:10D55000002133363C400000002132363C400000C0
:10D5600000212E363C400000002130363C400000B7
:10D57000002128363C400000002131363C400000AC
:10D58000002129363C40000000213E400000000000
:10D5900000212C363E40000000212B363E4000008A
:10D5A000002133363E400000002132363E4000006C
:10D5B00000212E363E400000002130363E40000063
:10D5C000002128363E400000002131363E40000058
:10D5D000002129363E40000000000000000000004D
:10D5E0000111181C1F2000000113181C1F2000002F
:10D5F000010E181C1F200000010C181C1F20000029
:10D600000110181C1F2000000112181C1F20000010
:10D610000107181C1F2000000115181C1F20000006
:10D620000104181C1F200000011C1F200000000026
:10D630000111181A1F2000000113181A1F200000E2
:10D64000010E181A1F200000010C181A1F200000DC
:10D650000110181A1F2000000112181A1F200000C4
:10D660000107181A1F2000000115181A1F200000BA
:10D670000104181A1F20000001191F2000000000DB
:10D680000111181B1F2000000113181B1F20000090
:10D69000010E181B1F200000010C181B1F2000008A
:10D6A0000110181B1F2000000112181B1F20000072
:10D6B0000107181B1F2000000115181B1F20000068
:10D6C0000104181B1F200000011B1F200000000088
:10D6D000011118191F200000011318191F20000044
:10D6E000010E18191F200000010C18191F2000003E
:10D6F000011018191F200000011218191F20000026
:10D70000010718191F200000011518191F2000001B
:10D71000010418191F20000001191F20000000003B
:10D720000111171F200000000113171F2000000027
:10D73000010D171F20000000010C171F2000000022
:10D740000110171F200000000112171F2000000009
:10D750000107171F2000000001161F200000000015
:10D76000010F1F200000000001171F200000000013
:10D7700001111F200000000001131F200000000005
:10D78000010E1F2000000000010C1F2000000000FF
:10D7900001101F200000000001121F2000000000E7
:10D7A00001071F200000000001151F2000000000DD
:10D7B00001091E200000000000173A0000000000D0
:10D7C000001723263A000000000F3A000000000076
:10D7D000000F23263A00000000163A000000000067
:10D7E000001623263A0000000007173A0000000048
:10D7F00000071723263A00000012173A0000000025
:10D8000000121723263A00000010173A000000000B
:10D8100000101723263A0000000B173A0000000002
:10D82000000B1723263A0000000D173A00000000F5
:10D83000000D1723263A00000013173A00000000DD
:10D8400000131723263A00000011173A00000000C9
:10D8500000111723263A000000193A0000000000CA
:10D86000001923263A000000000418193A000000AD
:10D870000004181923263A00001518193A49000027
:10D880000015181923263A49000718193A490000CB
:10D890000007181923263A49001218193A490000BE
:10D8A0000012181923263A49001018193A490000A5
:10D8B0000010181923263A49000C18193A4900009B
:10D8C000000C181923263A49000E18193A4900008D
:10D8D000000E181923263A49001318193A49000076
:10D8E0000013181923263A49001118193A49000063
:10D8F0000011181923263A49001B3A49000000007C
:10D90000001B23263A4900000004181B3A49000076
:10D910000004181B23263A490015181B3A49000039
:10D920000015181B23263A490007181B3A49000026
:10D930000007181B23263A490012181B3A49000019
:10D940000012181B23263A490010181B3A49000000
:10D950000010181B23263A49000C181B3A490000F6
:10D96000000C181B23263A49000E181B3A490000E8
:10D97000000E181B23263A490013181B3A490000D1
:10D980000013181B23263A490011181B3A490000BE
:10D990000011181B23263A49000000000000000077
:10D9A0000000000000000000000000000000000077
:10D9B0000000000000000000000000000000000067
:10D9C0000000000000000000000000000000000057
:10D9D0000000000000000000000000000000000047
:10D9E0000000000000000000000000000000000037
:10D9F0000000000000000000000000003D000000EA
:10DA0000350000002B000000330000003200000051
:10DA10002E0000003000000028000000310000004F
:10DA20002900000038000000370000003D00000021
:10DA3000350000002B000000330000003200000021
:10DA40002E0000003000000028000000310000001F
:10DA50002900000038000000370000003D000000F1
:10DA60003D4100002C4100002B41000033410000EB
:10DA7000324100002E4100003041000028410000EA
:10DA800031410000294100003841000037410000C9
:10DA90003D4100002C4100002B41000033410000BB
:10DAA000324100002E4100003041000028410000BA
:10DAB0003141000029410000384100003741000099
:10DAC0003D4100003D4147002C4147002B414700AC
:10DAD00033414700324142482E41424830414800DC
:10DAE0002841480031414800294148003841434A13
:10DAF0003741434A3D414A002C414A002B41464AA6
:10DB00003341464A3241464A2E41464A304144005A
:10DB10002841440031414400294144003841440037
:10DB2000374147003D4147002A4100002C41000099
:10DB30002B41000033410000324100002E41000023
:10DB4000304100002841000031410000294100001F
:10DB500038410000374100003D41000033384100AA
:10DB6000323841002E3841002F384100273841001B
:10DB70003138410029384100394100002C36394103
:10DB80002B3639413336394132363941141D0000C4
:10DB9000041D0000151D0000071D0000121D0000DF
:10DBA000101D00000C1D00000E1D0000131D0000C4
:10DBB000111D0000171D00000F1D0000161D0000A4
:10DBC000041D0000151D0000071D0000121D0000AF
:10DBD000101D00000C1D00000E1D0000131D000094
:10DBE000111D0000171D00000F1D0000161D000074
:10DBF000141D0000041D0000151D0000071D00007D
:10DC0000121D0000101D00000C1D00000E1D000064
:10DC1000131D0000111D0000171D00000F1D000046
:10DC2000161D000007171D0012171D0010171D00FC
:10DC30000B171D000D171D0013171D0011171D00D8
:10DC4000191D00000418191D1518191D0718191D94
:10DC50001218191D4500000000000000000000001F
:10DC600000000000000000000000000000000000B4
:10DC700000000000000000000000000000000000A4
:10DC80000000000000000000000000000000000094
:10DC90000000000000000000000000000000000084
:10DCA0000000000000000000000000000000000074
:10DCB00000000000450000006868206D6D202831DC
:10DCC000322900006868206D6D2028323429000058
:10DCD000686820756E64206D6D202831322900003F
:10DCE000686820756E64206D6D202832342900002C
:10DCF0006D6D206E616368206868202831322B29A1
:10DD0000000000006D6D206E616368206868202847
:10DD1000323429004F7373692F4265726C696E202B
:10DD200028313229000000004F7373692F42657259
:10DD30006C696E202831322B290000004F65736911
:10DD400020283132290000004F65736920283132C4
:10DD50002B290000526865696E2F52756872202861
:10DD600031322900526865696E2F52756872202819
:10DD700031322B2900000000536368776162656EC1
:10DD80002028313229000000536368776162656E94
:10DD9000202831322B290000576573736920283100
:10DDA000322900005765737369202831322B29000E
:10DDB000436F756E74646F776E00000054656D700C
:10DDC00065726174757200000000000000020003BB
:10DDD00003000707000E03000E04000F02010004F9
:10DDE0000102030102040102050107040107050104
:10DDF0000B04010B06020003020204020604020ADD
:10DE000004020E04030004030404030905030E04C2
:10DE1000040003040407040B0705000805080705B0
:10DE20000F03060006060007060803060B03060E8E
:10DE30000407000307030B070707070E0408000485
:10DE4000080006080504080804080C04080E030866
:10DE50000E04090004090404090405090A04090E52
:10DE6000040A00040A02030A02040A06030A0A0357
:10DE70000A0E040B00070B07040B0A080C00070C22
:10DE800007050C0B070D00060D00070D07030D0B12
:10DE9000040D0F030E00060E060B0E0C040E0C06EE
:10DEA0000F00070F07040F0B070000000705000015
:10DEB000B8DC000807060000C4DC00080805000004
:10DEC000D0DC000808060000E0DC000801030000C8
:10DED000F0DC00080104000004DD0008020100007D
:10DEE00014DD00080203000028DD00080301000023
:10DEF0003CDD00080303000048DD000804010000C9
:10DF000054DD00080403000064DD00080502000081
:10DF100078DD00080503000088DD00080601000028
:10DF200098DD000806030000A4DD000809070000D2
:10DF3000B0DD00080A000000BCDD00082800000079
:10DF400054696D656F757400290D0A004F4B000010
:10DF50004552524F520000002D20000049504144CC
:10DF60004452455353200000415020004D4F44453A
:10DF7000200000006170000054494D452000000061
:10DF80004649524D5741524520000000434D442020
:10DF90000000000048545450204745542000000021
:10DFA0002D2D3E20000000003C30643E3C30613EA0
:10DFB0000D0A00003C253032783E0000636170207D
:10DFC000222573222C22257322000000617020225A
:10DFD0002573222C222573220000000074696D65D0
:10DFE0002022257322000000455350383236362057
:10DFF0004C4F474745520D0A00000000ACED0008A9
:10E00000B4ED0008BCED0008C4ED0008C8ED000840
:10E01000CCED0008D0ED0008D4ED0008E4E60008DF
:10E02000ECE60008F4E600089CF90008F8E60008B1
:10E0300004E1000804E1000804E1000804E100082C
:10E0400004E10008040000000200000002000000DB
:10E050000200000002000000DCED0008E8ED00080E
:10E06000ACED0008B4ED0008D4ED0008E0EA0008CB
:10E07000E4EA0008ECEA000848EA0008ECED0008D1
:10E08000F0ED00089CEB00089CEB00089CEB0008FE
:10E09000F4ED0008F4ED0008F4ED0008ACED000824
:10E0A000F8ED000888E4000808EE0008D4ED000848
:10E0B000ACED0008F8ED000888E40008D4ED000895
:10E0C00014EE00081CEE000824EE000828EE0008FC
:10E0D00030EE000834EE00084CEA0008D4ED0008E9
:10E0E0006163746976650000257325640000000093
:10E0F000485454502F312E3020323030204F4B00B6
:10E100000D0A0D0A000000003C68746D6C3E0D0A9B
:10E11000000000003C686561643E0D0A00000000DC
:10E120003C7469746C653E003C2F7469746C653E88
:10E130000D0A00003C2F686561643E0D0A00000076
:10E140003C626F64793E0D0A000000003C48313E9D
:10E150000D0A00003C2F48313E0D0A003C6120684A
:10E160007265663D222F0000223E00003C2F613E7A
:10E17000266E6273703B266E6273703B0D0A000060
:10E180004D61696E000000006E6574776F726B0000
:10E190004E6574776F726B0054656D706572617453
:10E1A000757265006C6472004C445200446973706F
:10E1B0006C617900616E696D6174696F6E730000E6
:10E1C000416E696D6174696F6E730000616D6269A3
:10E1D0006C69676874000000416D62696C6967680A
:10E1E0007400000074696D657273000054696D6598
:10E1F000727300003C503E003C7472206267636F93
:10E200006C6F723D236630663066303E0D0A00004A
:10E210003C74723E0D0A00003C74643E0000000035
:10E220003C2F74643E0000003C696E70757420746D
:10E230007970653D2274657874222069643D2200FE
:10E2400022206E616D653D22000000002220766173
:10E250006C75653D2200000022206D61786C656E52
:10E260006774683D22000000222073697A653D22B0
:10E27000000000003C74643E3C627574746F6E2054
:10E28000747970653D227375626D697422206E61C8
:10E290006D653D22616374696F6E222076616C75D5
:10E2A000653D227361766500223E5365743C2F62A2
:10E2B0007574746F6E3E00003C2F74643E0D0A004E
:10E2C0003C7461626C6520626F726465723D303EC1
:10E2D0000D0A00003C2F74723E0D0A003C74683E2B
:10E2E0003C666F6E7420636F6C6F723D626C756517
:10E2F0003E0000003C2F666F6E743E3C2F74683EFB
:10E300000D0A00003C2F7461626C653E3C503E0D6E
:10E310000A0000003C627574746F6E207479706539
:10E320003D227375626D697422206E616D653D22B8
:10E33000616374696F6E222076616C75653D2200A1
:10E340003C2F627574746F6E3E266E6273703B0074
:10E350003C2F626F64793E0D0A0000003C2F687408
:10E360006D6C3E0D0A0000003C73656C65637420A3
:10E3700069643D2200000000223E0D0A00000000FA
:10E380003C2F73656C6563743E0D0A003C6F7074BE
:10E39000696F6E2076616C75653D22002073656C37
:10E3A00065637465640000003C2F6F7074696F6E64
:10E3B0003E0D0A00266E6273703B3C696E70757488
:10E3C00020747970653D22636865636B626F7822A3
:10E3D000206E616D653D2200222076616C75653D81
:10E3E00022616374697665222000000063686563BA
:10E3F0006B6564003C696E70757420747970653D5E
:10E400002272616E6765222069643D22000000006F
:10E4100022206D696E3D220022206D61783D220030
:10E4200022207374796C653D2277696474683A00C0
:10E4300070783B0022206F6E696E7075743D22000B
:10E440005F6F75747075742E76616C75653D000034
:10E450002E76616C7565223E000000003C6F75747D
:10E46000707574206E616D653D2200005F6F75747C
:10E47000707574223E0000003C2F6F7574707574C7
:10E480003E0000002E0D0A0044656661756C740044
:10E49000313500003C666F726D206D6574686F6485
:10E4A0003D224745542220616374696F6E3D222FDF
:10E4B000000000003C2F666F726D3E0D0A000000E8
:10E4C000436F6C6F727300003C74643E0D0A000071
:10E4D00036340000266E6273703B266E6273703BAA
:10E4E000266E6273703B0D0A000000004C6561727D
:10E4F0006E696E672049522072656D6F7465206386
:10E500006F6E74726F6C2E2E2E000000537769743C
:10E510006368696E6720706F776572206F6E2E2E4C
:10E520002E000000537769746368696E6720706F0E
:10E53000776572206F66662E2E2E00006F66666C01
:10E54000696E65004D696E696D756D206C656E67ED
:10E550007468206F66206B657920697320313021E3
:10E560000000000054696D657365727665722073F2
:10E5700075636365737366756C6C79206368616E2F
:10E580006765642E0000000053657474696E67202F
:10E590006F66206E65772074696D65736572766548
:10E5A00072206661696C65642E00000054696D65B7
:10E5B0007A6F6E65207375636365737366756C6CD3
:10E5C00079206368616E6765642E0000536574741A
:10E5D000696E67206F66206E65772074696D657A55
:10E5E0006F6E65206661696C65642E0047657474A2
:10E5F000696E67206E65742074696D6500000000A7
:10E60000446973706C6179696E672074656D7065BB
:10E610007261747572652E2E2E00000053746F7235
:10E620006564206D696E696D756D2076616C7565C8
:10E630000000000054657374696E6720646973702C
:10E640006C61792E2E2E0000536176696E672073FF
:10E65000657474696E6773207065726D616E656E46
:10E66000746C792E2E2E00006874747020706174A2
:10E67000683A20272573270D0A000000687474701B
:10E6800020706172616D65746572733A202725731D
:10E69000270D0A002F000000253032642E2530326D
:10E6A000640000002534640025303264000000005E
:10E6B000616374696F6E00006C6561726E697200EF
:10E6C000706F7765726F6E00706F7765726F6666D8
:10E6D00000000000736176656461746574696D653E
:10E6E0000000000079656172000000006D6F6E74BB
:10E6F00068000000646179006D696E007361766581
:10E700007469636B65720000576F7264436C6F636A
:10E710006B00000056657273696F6E00454550527C
:10E720004F4D0000454550524F4D2056657273695C
:10E730006F6E00005469636B65720000506F7765FF
:10E7400072204F6E00000000506F776572204F6698
:10E75000660000004C6561726E2049522072656D42
:10E760006F746520636F6E74726F6C006565707294
:10E770006F6D64756D700000454550524F4D2064BB
:10E78000756D70003C503E0D0A3C666F6E742063E0
:10E790006F6C6F723D677265656E3E003C5052450E
:10E7A0003E000000253034780000000020200000EA
:10E7B0003C2F5052453E0000202020002F6E6574F3
:10E7C000776F726B0000000073617665776C616E25
:10E7D00000000000776C616E6D6F646500000000E2
:10E7E0007373696400000000576F7264436C6F6359
:10E7F0006B204E6574776F726B0000003C423E43A5
:10E800006F6E6E656374696E6720746F2041636319
:10E8100065737320506F696E742C20747279206157
:10E820006761696E206C617465722E3C2F423E00F8
:10E830003C423E53746174696E672061732041638A
:10E840006365737320506F696E742C207472792025
:10E85000616761696E206C617465722E3C2F423E67
:10E86000000000007361766574696D65736572768A
:10E87000657200007361766574696D657A6F6E65A7
:10E88000000000006E657474696D65004950206178
:10E890006464726573730000455350383236362015
:10E8A0006669726D7761726500000000574C414ED9
:10E8B000000000005353494400000000266E6273BC
:10E8C000703B266E6273703B266E6273703B000075
:10E8D0004B65790054696D652073657276657200C9
:10E8E00054696D65207A6F6E652028474D54202B42
:10E8F00029000000476574206E65742074696D6599
:10E90000000000003C503E0D0A3C666F6E742063B0
:10E910006F6C6F723D7265643E3C423E00000000C9
:10E920003C2F423E3C2F666F6E743E0D0A00000085
:10E930002F74656D706572617475726500000000FA
:10E940007361766574636F727272746300000000A5
:10E950007361766574636F727264733138787800AE
:10E96000646973706C617974656D706572617475DA
:10E97000726500002E350000266465673B43000089
:10E98000576F7264436C6F636B2054656D70657272
:10E9900061747572650000005254432074656D7097
:10E9A000657261747572650044533138787800007F
:10E9B00054656D7020636F7272656374696F6E2049
:10E9C0005254432028756E697473206F6620302E70
:10E9D00035B043290000000054656D7020636F72EC
:10E9E00072656374696F6E204453313878782028DB
:10E9F000756E697473206F6620302E35B043290020
:10EA0000446973706C61792074656D7065726174AE
:10EA1000757265002F6C6472000000006C64726D8A
:10EA2000696E00006C64726D6178000073617665D8
:10EA30006175746F0000000025750000576F7264E7
:10EA4000436C6F636B204C44520000004D696E00B4
:10EA50004D6178004175746F6D61746963206272F5
:10EA6000696768746E6573730000000053657420F5
:10EA70006173206D696E696D756D2076616C756569
:10EA800000000000536574206173206D6178696D2A
:10EA9000756D2076616C7565000000002F646973E8
:10EAA000706C617900000000736176656974697348
:10EAB000000000007361766573796E63616D626951
:10EAC00000000000736176656272696768746E6544
:10EAD0007373000073617665636F6C6F727300000F
:10EAE00072656400677265656E000000626C756532
:10EAF0000000000073617665646973706C61796D04
:10EB00006F6465007361766574696E7465727661B1
:10EB10006C00000074657374646973706C617900D3
:10EB200073617665616C6C00576F7264436C6F63E0
:10EB30006B20446973706C61790000004553204973
:10EB4000535400005065726D616E656E7420646987
:10EB500073706C6179206F662022455320495354AD
:10EB600022000000446973706C6179204D6F646508
:10EB70000000000055736520646973706C61792032
:10EB8000636F6C6F727300004272696768746E65C0
:10EB900073732028312D313529000000300000002A
:10EBA00054656D7020646973706C617920696E744E
:10EBB000657276616C00000054657374206469733B
:10EBC000706C6179000000005361766520616C6CA7
:10EBD000000000002F616E696D6174696F6E7300D3
:10EBE00073617665616E696D6174696F6E000000B6
:10EBF00073617665636F6C6F72616E696D61746964
:10EC00006F6E00006465660073617665616E00007A
:10EC100073702564000000006661762564000000C2
:10EC20007361766563616E00637370256400000034
:10EC30006364656600000000576F7264436C6F6325
:10EC40006B20416E696D6174696F6E730000000026
:10EC5000416E696D6174696F6E000000436F6C6F87
:10EC60007220416E696D6174696F6E00616E25641A
:10EC700000000000646566256400000031000000AB
:10EC800063616E25640000006364656625640000AE
:10EC90002F616D62696C69676874000073617665E5
:10ECA000616D62696D6F6465000000007361766577
:10ECB000616D62696C656473000000007361766564
:10ECC000616D62696F666673657400007361766575
:10ECD00061616E00617370256400000061646566A7
:10ECE00000000000576F7264436C6F636B20416DCE
:10ECF00062696C6967687400234C454473000000C6
:10ED00004F6666736574206F66207365636F6E640B
:10ED1000203D203000000000416D62696C69676829
:10ED200074204D6F6465000061616E256400000011
:10ED300061646566256400002F74696D65727300F7
:10ED40007361766569640000610000006F00000077
:10ED50006625640074256400576F7264436C6F63AA
:10ED60006B2054696D65727300000000696425644E
:10ED700000000000612564006F25640068256400C0
:10ED80006D256400485454502F312E3020343034D7
:10ED9000204E6F7420466F756E640000343034204E
:10EDA0004E6F7420466F756E640D0A004E616D657E
:10EDB0000000000056616C756500000059595959F2
:10EDC000000000004D4D0000444400006868000051
:10EDD0006D6D0000416374696F6E0000574C414EC9
:10EDE00020436C69656E74004150000047000000CC
:10EDF0004200000036330000446563656C65726153
:10EE000074696F6E000000004661766F75726974F8
:10EE100065000000536C6F7400000000416374696A
:10EE2000766500004F6E000046726F6D00000000B6
:10EE3000546F0000486F7572000000000100000070
:10EE40000F00000015000000070000000B0000008C
:10EE5000070000000B000000070000000B0000008E
:10EE60000F00000014000000000000000F00000070
:10EE7000140000000000000001000000000000007D
:10EE800005000000020000000B0000000C00000064
:10EE90001A000000020000000B0000000200000049
:10EEA0000B00000000000000100000001C0000002B
:10EEB00028000000300000000100000001000000F8
:10EEC0000000000002000000050000000C0000002F
:10EED0001100000022000000050000000C000000EE
:10EEE000050000000C000000000000001000000001
:10EEF00010000000200000002000000001000000C1
:10EF000001000000000000000200000005000000F9
:10EF10000C000000110000002200000005000000AD
:10EF20000C000000050000000C00000000000000C4
:10EF300000000000000000000000000000000000D1
:10EF400001000000010000000000000003000000BC
:10EF5000050000000C0000000F0000001E00000073
:10EF6000050000000C000000040000000B00000081
:10EF70000000000010000000150000002500000047
:10EF8000250000000100000001000000000000005A
:10EF9000322E302E360000000D0A57656C636F6DFF
:10EFA0006520746F20576F7264436C6F636B204CE5
:10EFB0006F676765722100002D2D2D2D2D2D2D2DB4
:10EFC0002D2D2D2D2D2D2D2D2D2D2D2D2D2D2D2D71
:10EFD0002D2D2D2D0000000056657273696F6E3A5D
:10EFE00020000000727463206973206F6E6C696E7C
:10EFF00065000000727463206973206F66666C6937
:10F000006E650000656570726F6D206973206F6EAC
:10F010006C696E650000000063757272656E742025
:10F02000656570726F6D2076657273696F6E3A20D8
:10F030003078253038780D0A000000007265616470
:10F04000696E6720697220636F6465732066726FF2
:10F050006D20656570726F6D0000000072656164FF
:10F06000696E6720646973706C617920636F6E6686
:10F07000696775726174696F6E2066726F6D206565
:10F080006570726F6D00000072656164696E672063
:10F0900074696D6573657276657220646174612050
:10F0A00066726F6D20656570726F6D007265616468
:10F0B000696E67206E696768742074696D65727324
:10F0C0002066726F6D20656570726F6D00000000C4
:10F0D00072656164696E672074656D7020636F6E20
:10F0E00066696775726174696F6E2066726F6D20F4
:10F0F000656570726F6D0000656570726F6D206977
:10F1000073206F66666C696E6500000075706461DF
:10F1100074696E6720454550524F4D20746F2076BC
:10F12000657273696F6E203078253038780D0A006B
:10F1300077726974696E672076657273696F6E2085
:10F14000746F20454550524F4D206661696C65646F
:10F150000000000077726974696E6720495220636D
:10F160006F64657320746F20454550524F4D206683
:10F1700061696C656400000077726974696E67206C
:10F18000636F6E66696720746F20454550524F4D1E
:10F19000206661696C65640077726974696E6720C6
:10F1A00074696D657365727665722064617461203F
:10F1B000746F20454550524F4D206661696C6564FF
:10F1C0000000000077726974696E67206E69676875
:10F1D000742074696D65206461746120746F2045CA
:10F1E0004550524F4D206661696C65640000000017
:10F1F00063616C6C696E67204952206C6561726E48
:10F200002066756E6374696F6E00000075736572B9
:10F2100020627574746F6E20707265737365643AE2
:10F2200020636F6E6669677572696E6720657370BB
:10F2300038323636206173206163636573732070E2
:10F240006F696E7400000000776F7264636C6F63A7
:10F250006B00000031323334353637383930000036
:10F26000636F6D6D616E643A2073657420646973B9
:10F27000706C617920636F6C6F727320746F2025DE
:10F28000642025642025640D0A000000636F6D6D05
:10F29000616E643A2073657420616D62696C6967A0
:10F2A000687420636F6C6F727320746F2025642004
:10F2B00025642025640D0A00636F6D6D616E643AEC
:10F2C0002073657420706F776572202573000000CD
:10F2D000636F6D6D616E643A207365742064697349
:10F2E000706C6179206D6F646520746F2025640DEA
:10F2F0000A000000636F6D6D616E643A207365747F
:10F3000020616D62696C69676874206D6F64652047
:10F31000746F2025640D0A00636F6D6D616E643A31
:10F320002073657420616E696D6174696F6E206D04
:10F330006F646520746F2025640D0A00636F6D6D26
:10F34000616E643A2073657420636F6C6F72206124
:10F350006E696D6174696F6E206D6F646520746F86
:10F360002025640D0A000000636F6D6D616E643AC4
:10F370002073686F772074656D7065726174757243
:10F3800065000000636F6D6D616E643A2073657493
:10F3900020646973706C6179206272696768746E49
:10F3A00065737320746F2025642C20646973616217
:10F3B0006C65206175746D6F6D6174696320627234
:10F3C000696768746E65737320636F6E74726F6CB7
:10F3D00020706572204C44520D0A0000636F6D6D01
:10F3E000616E643A2073657420616D62696C69674F
:10F3F0006874206272696768746E65737320746FD5
:10F400002025640D0A000000636F6D6D616E643A23
:10F4100020656E61626C65206175746F6D617469E1
:10F4200063206272696768746E65737320636F6EC0
:10F4300074726F6C00000000636F6D6D616E643AF2
:10F440002064697361626C65206175746F6D6174AD
:10F450006963206272696768746E65737320636F95
:10F460006E74726F6C000000636F6D6D616E643A54
:10F470002073657420646973706C617920666C61B7
:10F48000677320746F2030782530327800000000D8
:10F49000636F6D6D616E643A207374617274206481
:10F4A0006973706C6179207465737400636F6D6D3E
:10F4B000616E643A207365742074696D6520746FA1
:10F4C000202573202534642D253032642D253032DB
:10F4D0006420253032643A253032643A2530326473
:10F4E0000D0A0000636F6D6D616E643A2073746184
:10F4F0007274206E65742074696D65207265717513
:10F5000065737400636F6D6D616E643A206C656144
:10F51000726E20495220636F64657300636F6D6D76
:10F52000616E643A207361766520646973706C6102
:10F53000792073657474696E67730000636F6D6D15
:10F54000616E643A207072696E74207469636B65D1
:10F55000723A2027257327006C64723A206F6C641E
:10F56000206272696768746E65733A202564206E44
:10F570006577206272696768746E6573733A2025D7
:10F58000640D0A0065737038323636206E6F77204E
:10F590007570000065737038323636206E6F7720D4
:10F5A0006F6E6C696E650000202049502025730045
:10F5B00064636637373A202573202534642D25305F
:10F5C00032642D2530326420253032643A253032C1
:10F5D000643A253032640D0A0000000072656164EF
:10F5E000207274633A202573202534642D2530322F
:10F5F000642D2530326420253032643A253032645F
:10F600003A253032640D0A00466F756E64205469E5
:10F610006D65723A20257320617420253032643A7A
:10F62000253032640D0A0000676F742074656D70B8
:10F63000657261747572652066726F6D2044533116
:10F64000387878783A20256425730D0A0000000088
:10F65000676F742074656D70657261747572652072
:10F6600066726F6D205254433A20256425730D0A4B
:10F67000000000006E6F2074656D706572617475B6
:10F68000726520617661696C61626C6500000000E2
:10F6900075706461746520646973706C61790000D1
:10F6A00049524D503A20504F574552206B657900D2
:10F6B00049524D503A204F4B206B657900000000B5
:10F6C00049524D503A2064656372656D656E7420D1
:10F6D000646973706C6179206D6F6465000000006F
:10F6E00049524D503A20696E6372656D656E7420A3
:10F6F000646973706C6179206D6F6465000000004F
:10F7000049524D503A2064656372656D656E742090
:10F71000616E696D6174696F6E206D6F6465000064
:10F7200049524D503A20696E6372656D656E742062
:10F73000616E696D6174696F6E206D6F6465000044
:10F7400049524D503A2064656372656D656E742050
:10F75000686F75720000000049524D503A20696E82
:10F760006372656D656E7420686F757200000000CD
:10F7700049524D503A2064656372656D656E742020
:10F780006D696E757465000049524D503A20696E7E
:10F790006372656D656E74206D696E7574650000C9
:10F7A00049524D503A2064656372656D656E7420F0
:10F7B000726564206272696768746E6573730000B5
:10F7C00049524D503A20696E6372656D656E7420C2
:10F7D000726564206272696768746E657373000095
:10F7E00049524D503A2064656372656D656E7420B0
:10F7F000677265656E206272696768746E6573739F
:10F800000000000049524D503A20696E6372656DE8
:10F81000656E7420677265656E20627269676874D0
:10F820006E6573730000000049524D503A206465C4
:10F830006372656D656E7420626C756520627269B5
:10F840006768746E6573730049524D503A20696E53
:10F850006372656D656E7420626C75652062726995
:10F860006768746E6573730049524D503A20646541
:10F870006372656D656E74206272696768746E6527
:10F880007373000049524D503A20696E6372656D82
:10F89000656E74206272696768746E6573730000C8
:10F8A00049524D503A206765742074656D706572D9
:10F8B0006174757265000000706F7765725F696EC4
:10F8C000697428292063616C6C65640073776974BE
:10F8D0006368696E6720706F776572206F6E0000D5
:10F8E000737769746368696E6720706F77657220DB
:10F8F0006F66660020206765742074656D706572A0
:10F9000061747572650000002020706F7765722049
:10F910006F66662F6F6E000020206F6B0000000086
:10F92000202064656372656D656E74206469737010
:10F930006C6179206D6F6465000000002020696EA5
:10F940006372656D656E7420646973706C61792093
:10F950006D6F646500000000202064656372656D52
:10F96000656E7420616E696D6174696F6E206D6F74
:10F97000646500002020696E6372656D656E742099
:10F98000616E696D6174696F6E206D6F64650000F2
:10F99000202064656372656D656E7420686F757292
:10F9A000000000002020696E6372656D656E742032
:10F9B000686F757200000000202064656372656DD9
:10F9C000656E74206D696E75746500002020696E27
:10F9D0006372656D656E74206D696E757465000087
:10F9E000202064656372656D656E742072656420A5
:10F9F0006272696768746E65737300002020696EB7
:10FA00006372656D656E74207265642062726967E9
:10FA100068746E6573730000202064656372656DA1
:10FA2000656E7420677265656E20627269676874BE
:10FA30006E657373000000002020696E6372656D4F
:10FA4000656E7420677265656E206272696768749E
:10FA50006E65737300000000202064656372656D3D
:10FA6000656E7420626C7565206272696768746E79
:10FA7000657373002020696E6372656D656E742016
:10FA8000626C7565206272696768746E6573730075
:10FA9000202064656372656D656E7420676C6F62AB
:10FAA000616C206272696768746E65737300000030
:10FAB0002020696E6372656D656E7420676C6F627D
:10FAC000616C206272696768746E65737300000010
:10FAD0002020746F67676C65206175746F20627297
:10FAE000696768746E6573730000000020205468B5
:10FAF000616E6B20796F7521000000003139322E64
:10FB000035332E3130332E31303300004E657720BF
:10FB100074696D657A6F6E653A2025640D0A000080
:10FB200043000000F40100201F0000001C00000042
:10FB30001F0000001E0000001F0000001E0000004B
:10FB40001F0000001F0000001E0000001F0000003A
:10FB50001E0000001F0000001F0000001D0000002C
:10FB60001F0000001E0000001F0000001E0000001B
:10FB70001F0000001F0000001E0000001F0000000A
:10FB80001E0000001F0000006D0100006E0100005B
:10FB9000232D302B2000686C4C0065666745464776
:10FBA00000303132333435363738394142434445F9
:10FBB0004600303132333435363738396162636468
:10FBC00065660000202020202020202020282828D2
:10FBD0002828202020202020202020202020202015
:10FBE000202020208810101010101010101010105D
:10FBF000101010100404040404040404040410107D
:10FC00001010101010414141414141010101010119
:10FC100001010101010101010101010101010110C5
:10FC200010101010104242424242420202020202EE
:10FC30000202020202020202020202020202021096
:10FC40001010102000000000000000000000000064
:10FC500000000000000000000000000000000000A4
:10FC60000000000000000000000000000000000094
:10FC70000000000000000000000000000000000084
:10FC80000000000000000000000000000000000074
:10FC90000000000000000000000000000000000064
:10FCA0000000000000000000000000000000000054
:10FCB0000000000000000000000000000000000044
:08FCC00000000000000000003C
:08FCC8001405FF7F010000009C
:10FCD00000000000010203040102030406070809F2
:10FCE00038BF000820BF00083CBF000840BF000824
:10FCF00044BF000830BF000834BF0008FF00000008
:10FD0000FF000000E80300000100000020000000E8
:10FD1000200000000300000005000000200000009B
:10FD200074C40008B51D00080200000002000000B5
:10FD30000000000084C40008291E00080400000020
:10FD400004000000030000008CC40008E52800083F
:10FD500002000000020000000300000094C400083C
:10FD600099260008020000000200000003000000C5
:10FD70009CC40008091A00080200000002000000EC
:10FD800000000000A4C40008B12B0008020000001D
:10FD90000200000003000000ACC40008E9250008D0
:10FDA000040000000400000003000000B8C40008C4
:10FDB0002D240008020000000200000003000000E3
:10FDC000C0C40008092F0008020000000200000063
:10FDD00003000000C8C4000855220008020000000B
:10FDE0000200000003000000D0C40008D520000875
:10FDF000040000000400000003000000D8C4000854
:10FE00000000000000000000000000000CE70008F7
:10FE1000000000000000000000000000E0C4000836
:10FE20000000000000000000000000007CC400088A
:10FE30000400000004000000010000000F000000AA
:10FE400020000000010000003C00000074C4000815
:10FE50000100000001000000000000007CC4000858
:10FE60000400000004000000010000000500000084
:10FE7000010000000F00000016000000FFFF00005E
:10FE8000FFFF0000D80E0000FFFFFFFFFF00000093
:10FE9000FF000000FF000000000000000000000064
:10FEA0000102030406070809007A030A01000000A2
:10FEB0003139322E35332E3130332E31303300008C
:10FEC0000000000000000000000000000000000032
:10FED0000000000000000000000000000000000022
:10FEE0000000000020FB00080000000000000000EF
:10FEF0000000000000000000000000000000000002
:10FF000000000000000000000000000000000000F1
:10FF100000000000000000000000000000000000E1
:10FF200000000000F4010020C3FB000801000000F5
:10FF3000000000004A000000000000000000000077
:10FF400000000000000000000000000000000000B1
:10FF50004A00000000000000000000000000000057
:10FF6000000000000000000000000000AD010008DB
:04FF700089010008FB
:0400000508000000EF
:00000001FF
